LX51 LINKER/LOCATER V4.66.97.0                                                          06/12/2025  17:35:51  PAGE 1


LX51 LINKER/LOCATER V4.66.97.0, INVOKED BY:
D:\KEIL_V5\C51\BIN\LX51.EXE .\Out_Files\STARTUP.obj, .\Out_Files\system_um800y.obj, .\Out_Files\common.obj, .\Out_Files\
>> uart0.obj, .\Out_Files\gpio.obj, .\Out_Files\lptimer.obj, .\Out_Files\radio.obj, .\Out_Files\um2006A.obj, .\Out_Files
>> \um2006A_hal.obj, .\Out_Files\main.obj, .\Out_Files\app.obj, .\Out_Files\app_um2006A.obj, .\Out_Files\app_ev1527.obj 
>> TO .\Out_Files\UM2006A_RX_DIRECT PRINT (.\Out_Files\UM2006A_RX_DIRECT.map) REMOVEUNUSED CLASSES (XDATA (X:0X0-X:0X7FF
>> ), HDATA (X:0X0-X:0X7FF), ECODE (C:0X0-C:0XFFFF), HCONST (C:0X0-C:0XFFFF))


CPU MODE:     8051 MODE
MEMORY MODEL: LARGE WITH FLOATING POINT ARITHMETIC


INPUT MODULES INCLUDED:
  .\Out_Files\STARTUP.obj (?C_STARTUP)
         COMMENT TYPE 1: A51 / ASM51 Assembler
  .\Out_Files\system_um800y.obj (SYSTEM_UM800Y)
         COMMENT TYPE 0: C51 V9.60.0.0
  .\Out_Files\common.obj (COMMON)
         COMMENT TYPE 0: C51 V9.60.0.0
  .\Out_Files\uart0.obj (UART0)
         COMMENT TYPE 0: C51 V9.60.0.0
  .\Out_Files\gpio.obj (GPIO)
         COMMENT TYPE 0: C51 V9.60.0.0
  .\Out_Files\lptimer.obj (LPTIMER)
         COMMENT TYPE 0: C51 V9.60.0.0
  .\Out_Files\radio.obj (RADIO)
         COMMENT TYPE 0: C51 V9.60.0.0
  .\Out_Files\um2006A.obj (UM2006A)
         COMMENT TYPE 0: C51 V9.60.0.0
  .\Out_Files\um2006A_hal.obj (UM2006A_HAL)
         COMMENT TYPE 0: C51 V9.60.0.0
  .\Out_Files\main.obj (MAIN)
         COMMENT TYPE 0: C51 V9.60.0.0
  .\Out_Files\app.obj (APP)
         COMMENT TYPE 0: C51 V9.60.0.0
  .\Out_Files\app_um2006A.obj (APP_UM2006A)
         COMMENT TYPE 0: C51 V9.60.0.0
  .\Out_Files\app_ev1527.obj (APP_EV1527)
         COMMENT TYPE 0: C51 V9.60.0.0
  D:\KEIL_V5\C51\LIB\C51FPL.LIB (?C?FPADD)
         COMMENT TYPE 1: A51 / ASM51 Assembler
  D:\KEIL_V5\C51\LIB\C51FPL.LIB (?C?FPMUL)
         COMMENT TYPE 1: A51 / ASM51 Assembler
  D:\KEIL_V5\C51\LIB\C51FPL.LIB (?C?FPDIV)
         COMMENT TYPE 1: A51 / ASM51 Assembler
  D:\KEIL_V5\C51\LIB\C51FPL.LIB (?C?FPCMP)
         COMMENT TYPE 1: A51 / ASM51 Assembler
  D:\KEIL_V5\C51\LIB\C51FPL.LIB (?C?FPNEG)
         COMMENT TYPE 1: A51 / ASM51 Assembler
  D:\KEIL_V5\C51\LIB\C51FPL.LIB (?C?FCAST)
         COMMENT TYPE 1: A51 / ASM51 Assembler
  D:\KEIL_V5\C51\LIB\C51FPL.LIB (?C?CASTF)
         COMMENT TYPE 1: A51 / ASM51 Assembler
  D:\KEIL_V5\C51\LIB\C51FPL.LIB (PRINTF)
         COMMENT TYPE 1: A51 / ASM51 Assembler
  D:\KEIL_V5\C51\LIB\C51FPL.LIB (FABS)
         COMMENT TYPE 1: A51 / ASM51 Assembler
  D:\KEIL_V5\C51\LIB\C51FPL.LIB (?C?FPGETOPN)
         COMMENT TYPE 1: A51 / ASM51 Assembler
  D:\KEIL_V5\C51\LIB\C51FPL.LIB (?C?FPROUND)
         COMMENT TYPE 1: A51 / ASM51 Assembler
  D:\KEIL_V5\C51\LIB\C51FPL.LIB (?C?FPCONVERT)
         COMMENT TYPE 1: A51 / ASM51 Assembler
  D:\KEIL_V5\C51\LIB\C51FPL.LIB (?C?FTNPWR)
         COMMENT TYPE 1: A51 / ASM51 Assembler
  D:\KEIL_V5\C51\LIB\C51L.LIB (?C_INIT)
LX51 LINKER/LOCATER V4.66.97.0                                                        06/12/2025  17:35:51  PAGE 2


         COMMENT TYPE 1: A51 / ASM51 Assembler
  D:\KEIL_V5\C51\LIB\C51L.LIB (?C?COPY)
         COMMENT TYPE 1: A51 / ASM51 Assembler
  D:\KEIL_V5\C51\LIB\C51L.LIB (?C?CLDPTR)
         COMMENT TYPE 1: A51 / ASM51 Assembler
  D:\KEIL_V5\C51\LIB\C51L.LIB (?C?CLDOPTR)
         COMMENT TYPE 1: A51 / ASM51 Assembler
  D:\KEIL_V5\C51\LIB\C51L.LIB (?C?CSTPTR)
         COMMENT TYPE 1: A51 / ASM51 Assembler
  D:\KEIL_V5\C51\LIB\C51L.LIB (?C?CSTOPTR)
         COMMENT TYPE 1: A51 / ASM51 Assembler
  D:\KEIL_V5\C51\LIB\C51L.LIB (?C?IMUL)
         COMMENT TYPE 1: A51 / ASM51 Assembler
  D:\KEIL_V5\C51\LIB\C51L.LIB (?C?LADD)
         COMMENT TYPE 1: A51 / ASM51 Assembler
  D:\KEIL_V5\C51\LIB\C51L.LIB (?C?LMUL)
         COMMENT TYPE 1: A51 / ASM51 Assembler
  D:\KEIL_V5\C51\LIB\C51L.LIB (?C?ULDIV)
         COMMENT TYPE 1: A51 / ASM51 Assembler
  D:\KEIL_V5\C51\LIB\C51L.LIB (?C?SLDIV)
         COMMENT TYPE 1: A51 / ASM51 Assembler
  D:\KEIL_V5\C51\LIB\C51L.LIB (?C?LOR)
         COMMENT TYPE 1: A51 / ASM51 Assembler
  D:\KEIL_V5\C51\LIB\C51L.LIB (?C?LNEG)
         COMMENT TYPE 1: A51 / ASM51 Assembler
  D:\KEIL_V5\C51\LIB\C51L.LIB (?C?SLCMP)
         COMMENT TYPE 1: A51 / ASM51 Assembler
  D:\KEIL_V5\C51\LIB\C51L.LIB (?C?ULCMP)
         COMMENT TYPE 1: A51 / ASM51 Assembler
  D:\KEIL_V5\C51\LIB\C51L.LIB (?C?ULSHR)
         COMMENT TYPE 1: A51 / ASM51 Assembler
  D:\KEIL_V5\C51\LIB\C51L.LIB (?C?LSHL)
         COMMENT TYPE 1: A51 / ASM51 Assembler
  D:\KEIL_V5\C51\LIB\C51L.LIB (?C?LLDOPTR)
         COMMENT TYPE 1: A51 / ASM51 Assembler
  D:\KEIL_V5\C51\LIB\C51L.LIB (?C?LLDXDATA)
         COMMENT TYPE 1: A51 / ASM51 Assembler
  D:\KEIL_V5\C51\LIB\C51L.LIB (?C?LLDXDATA0)
         COMMENT TYPE 1: A51 / ASM51 Assembler
  D:\KEIL_V5\C51\LIB\C51L.LIB (?C?LLDIXDATA)
         COMMENT TYPE 1: A51 / ASM51 Assembler
  D:\KEIL_V5\C51\LIB\C51L.LIB (?C?LSTXDATA)
         COMMENT TYPE 1: A51 / ASM51 Assembler
  D:\KEIL_V5\C51\LIB\C51L.LIB (?C?LSTKXDATA)
         COMMENT TYPE 1: A51 / ASM51 Assembler
  D:\KEIL_V5\C51\LIB\C51L.LIB (?C?PLDXDATA)
         COMMENT TYPE 1: A51 / ASM51 Assembler
  D:\KEIL_V5\C51\LIB\C51L.LIB (?C?PLDIXDATA)
         COMMENT TYPE 1: A51 / ASM51 Assembler
  D:\KEIL_V5\C51\LIB\C51L.LIB (?C?PSTXDATA)
         COMMENT TYPE 1: A51 / ASM51 Assembler
  D:\KEIL_V5\C51\LIB\C51L.LIB (?C?CCASE)
         COMMENT TYPE 1: A51 / ASM51 Assembler
  D:\KEIL_V5\C51\LIB\C51L.LIB (?C?LCASE)
         COMMENT TYPE 1: A51 / ASM51 Assembler
  D:\KEIL_V5\C51\LIB\C51L.LIB (?C?ICALL)
         COMMENT TYPE 1: A51 / ASM51 Assembler
  D:\KEIL_V5\C51\LIB\C51L.LIB (?C?MEMSET)
         COMMENT TYPE 1: A51 / ASM51 Assembler
  D:\KEIL_V5\C51\LIB\C51L.LIB (?C?LLDIDATA)
         COMMENT TYPE 1: A51 / ASM51 Assembler
  D:\KEIL_V5\C51\LIB\C51L.LIB (?C?LLDPDATA)
         COMMENT TYPE 1: A51 / ASM51 Assembler
  D:\KEIL_V5\C51\LIB\C51L.LIB (?C?LLDCODE)
         COMMENT TYPE 1: A51 / ASM51 Assembler
LX51 LINKER/LOCATER V4.66.97.0                                                        06/12/2025  17:35:51  PAGE 3




ACTIVE MEMORY CLASSES OF MODULE:  .\Out_Files\UM2006A_RX_DIRECT (?C_STARTUP)

BASE        START       END         USED      MEMORY CLASS
==========================================================
X:000000H   X:000000H   X:0007FFH   000332H   XDATA
X:000000H   X:000000H   X:0007FFH             HDATA
C:000000H   C:000000H   C:00FFFFH             ECODE
C:000000H   C:000000H   C:00FFFFH             HCONST
C:000000H   C:000000H   C:00FFFFH   001F25H   CODE
I:000000H   I:000000H   I:0000FFH   000001H   IDATA
C:000000H   C:000000H   C:00FFFFH   0001ADH   CONST
I:000000H   I:000000H   I:00007FH   000015H   DATA
I:000020H.0 I:000020H.0 I:00002FH.7 000001H.1 BIT


MEMORY MAP OF MODULE:  .\Out_Files\UM2006A_RX_DIRECT (?C_STARTUP)


START     STOP      LENGTH    ALIGN  RELOC    MEMORY CLASS   SEGMENT NAME
=========================================================================

* * * * * * * * * * *   D A T A   M E M O R Y   * * * * * * * * * * * * *
000000H   000007H   000008H   ---    AT..     DATA           "REG BANK 0"
000008H   00000CH   000005H   BYTE   UNIT     DATA           _DATA_GROUP_
00000DH   000017H   00000BH   ---    ---      **GAP**
000018H   00001FH   000008H   ---    AT..     DATA           "REG BANK 3"
000020H.0 000021H.0 000001H.1 BIT    UNIT     BIT            _BIT_GROUP_
000021H.1 000021H   000000H.7 ---    ---      **GAP**
000022H   000022H   000001H   BYTE   UNIT     IDATA          ?STACK

* * * * * * * * * * *   C O D E   M E M O R Y   * * * * * * * * * * * * *
000000H   000002H   000003H   ---    OFFS..   CODE           ?CO??C_STARTUP?0
000003H   000005H   000003H   BYTE   OFFS..   CODE           ?APP_EV1527?00003
000006H   00001BH   000016H   BYTE   UNIT     CODE           ?PR?_UART0_SEND_BYTE?UART0
00001CH   000022H   000007H   BYTE   UNIT     CODE           ?PR?UM2006A_HAL_IRQ?UM2006A_HAL
000023H   000025H   000003H   BYTE   OFFS..   CODE           ?UART0?00023
000026H   00005CH   000037H   BYTE   UNIT     CODE           ?PR?_UART0_INIT?UART0
00005DH   000062H   000006H   BYTE   UNIT     CODE           ?PR?APP_UM2006A_INIT?APP_UM2006A
000063H   000065H   000003H   BYTE   OFFS..   CODE           ?LPTIMER?00063
000066H   000AAFH   000A4AH   BYTE   UNIT     CODE           ?C?LIB_CODE
000AB0H   000F32H   000483H   BYTE   UNIT     CODE           ?PR?PRINTF?PRINTF
000F33H   00112FH   0001FDH   BYTE   UNIT     CODE           ?C_INITSEG
001130H   00125DH   00012EH   BYTE   UNIT     CODE           ?PR?_CLOCK_INIT?SYSTEM_UM800Y
00125EH   001357H   0000FAH   BYTE   UNIT     CODE           ?PR?GPIO_IRQHANDLER?APP_EV1527
001358H   00141FH   0000C8H   BYTE   UNIT     CODE           ?PR?LPTIMER_IRQHANDLER?LPTIMER
001420H   0014E2H   0000C3H   BYTE   UNIT     CODE           ?PR?_GPIO_IRQ_SET?GPIO
0014E3H   0015A1H   0000BFH   BYTE   UNIT     CODE           ?PR?_GPIO_IN_ENABLE?GPIO
0015A2H   00163CH   00009BH   BYTE   UNIT     CODE           ?PR?UM2006A_CAL_RC32K?UM2006A
00163DH   0016C8H   00008CH   BYTE   UNIT     CODE           ?C_C51STARTUP
0016C9H   001752H   00008AH   BYTE   UNIT     CODE           ?PR?_APP_EV1527_RECV_DATA?APP_EV1527
001753H   0017D3H   000081H   BYTE   UNIT     CODE           ?PR?_GPIO_DIR_SET?GPIO
0017D4H   001854H   000081H   BYTE   UNIT     CODE           ?PR?_GPIO_PU_SET?GPIO
001855H   0018D5H   000081H   BYTE   UNIT     CODE           ?PR?_GPIO_PD_SET?GPIO
0018D6H   001956H   000081H   BYTE   UNIT     CODE           ?PR?_GPIO_IO_SET?GPIO
001957H   0019D6H   000080H   BYTE   UNIT     CODE           ?PR?APP_UM2006A_RUN?APP_UM2006A
0019D7H   001A4DH   000077H   BYTE   UNIT     CODE           ?PR?_UART0_SET_BAUD_RATE?UART0
001A4EH   001AB5H   000068H   BYTE   UNIT     CODE           ?PR?UM2006A_INIT?UM2006A
001AB6H   001B19H   000064H   BYTE   UNIT     CODE           ?PR?SPI_READ_BYTE?UM2006A_HAL
001B1AH   001B7AH   000061H   BYTE   UNIT     CODE           ?PR?APP_INIT?APP
001B7BH   001BD5H   00005BH   BYTE   UNIT     CODE           ?PR?_SPI_WRITE_BYTE?UM2006A_HAL
001BD6H   001C25H   000050H   BYTE   UNIT     CODE           ?PR?SPI_INIT?UM2006A_HAL
001C26H   001C6FH   00004AH   BYTE   UNIT     CODE           ?PR?UART0_IRQHANDLER?UART0
001C70H   001CB6H   000047H   BYTE   UNIT     CODE           ?PR?_DELAY_MS?COMMON
LX51 LINKER/LOCATER V4.66.97.0                                                        06/12/2025  17:35:51  PAGE 4


001CB7H   001CFCH   000046H   BYTE   UNIT     CODE           ?PR?_GPIO_IRQ_CLR?GPIO
001CFDH   001D40H   000044H   BYTE   UNIT     CODE           ?C?LDIV
001D41H   001D80H   000040H   BYTE   UNIT     CODE           ?PR?_GPIO_IO_GET?GPIO
001D81H   001DC0H   000040H   BYTE   UNIT     CODE           ?PR?APP_EV1527_INIT?APP_EV1527
001DC1H   001DF5H   000035H   BYTE   UNIT     CODE           ?PR?_GPIO_INIT?GPIO
001DF6H   001E2AH   000035H   BYTE   UNIT     CODE           ?PR?_UM2006A_WRITE_REG?UM2006A
001E2BH   001E5AH   000030H   BYTE   UNIT     CODE           ?PR?_LPTIMER_INIT?LPTIMER
001E5BH   001E8AH   000030H   BYTE   UNIT     CODE           ?PR?UM2006A_HAL_INIT?UM2006A_HAL
001E8BH   001EB8H   00002EH   BYTE   UNIT     CODE           ?PR?_UM2006A_READ_REG?UM2006A
001EB9H   001EC6H   00000EH   BYTE   UNIT     CODE           ?PR?UM2006A_INTO_RX_BPFCAL?UM2006A
001EC7H   001ED4H   00000EH   BYTE   UNIT     CODE           ?PR?UM2006A_RESET_DIGIT?UM2006A
001ED5H   001EE2H   00000EH   BYTE   UNIT     CODE           ?PR?SPI_CS_DISABLE?UM2006A_HAL
001EE3H   001EEEH   00000CH   BYTE   UNIT     CODE           ?PR?RADIO_INIT?RADIO
001EEFH   001EF9H   00000BH   BYTE   UNIT     CODE           ?PR?SYSTEM_INIT?SYSTEM_UM800Y
001EFAH   001F04H   00000BH   BYTE   UNIT     CODE           ?PR?MAIN?MAIN
001F05H   001F0DH   000009H   BYTE   UNIT     CODE           ?PR?_LPTIMER_SET_TIME?LPTIMER
001F0EH   001F15H   000008H   BYTE   UNIT     CODE           ?PR?LPTIMER_START?LPTIMER
001F16H   001F1CH   000007H   BYTE   UNIT     CODE           ?PR?SPI_CS_ENABLE?UM2006A_HAL
001F1DH   001F21H   000005H   BYTE   UNIT     CODE           ?PR?_PUTCHAR?UART0
001F22H   001F24H   000003H   BYTE   UNIT     CODE           ?PR?APP_RUN?APP
001F25H   002071H   00014DH   BYTE   UNIT     CONST          ?CO?APP
002072H   0020D1H   000060H   BYTE   UNIT     CONST          ?CO?APP_UM2006A

* * * * * * * * * * *  X D A T A   M E M O R Y  * * * * * * * * * * * * *
000000H   000157H   000158H   BYTE   UNIT     XDATA          ?XD?UM2006A
000158H   00025EH   000107H   BYTE   UNIT     XDATA          ?XD?APP_EV1527
00025FH   0002D0H   000072H   BYTE   UNIT     XDATA          _XDATA_GROUP_
0002D1H   000318H   000048H   BYTE   UNIT     XDATA          ?XD?GPIO
000319H   000324H   00000CH   BYTE   UNIT     XDATA          ?XD?LPTIMER
000325H   00032CH   000008H   BYTE   UNIT     XDATA          ?XD?SYSTEM_UM800Y
00032DH   000330H   000004H   BYTE   UNIT     XDATA          ?XD?UART0
000331H   000331H   000001H   BYTE   UNIT     XDATA          ?XD?UM2006A_HAL

* * * * * * * * *   R E M O V E D     S E G M E N T S   * * * * * * * *
   *DEL*:           000015H   BYTE   UNIT     CODE           ?PR?_DELAY?COMMON
   *DEL*:           000004H   BYTE   UNIT     XDATA          ?XD?_DELAY?COMMON
   *DEL*:           00006CH   BYTE   UNIT     CODE           ?PR?_PRINTF_BUFF_BYTE?COMMON
   *DEL*:           00000BH   BYTE   UNIT     XDATA          ?XD?_PRINTF_BUFF_BYTE?COMMON
   *DEL*:           000077H   BYTE   UNIT     CODE           ?PR?_PRINTF_BUFF_WORD?COMMON
   *DEL*:           00000BH   BYTE   UNIT     XDATA          ?XD?_PRINTF_BUFF_WORD?COMMON
   *DEL*:           000010H   BYTE   UNIT     CONST          ?CO?COMMON
   *DEL*:           000012H   BYTE   UNIT     CODE           ?PR?_UART0_IRQ_INIT?UART0
   *DEL*:           00002EH   BYTE   UNIT     CODE           ?PR?_UART0_SEND_BYTES?UART0
   *DEL*:           000007H   BYTE   UNIT     XDATA          ?XD?_UART0_SEND_BYTES?UART0
   *DEL*:           000003H   BYTE   UNIT     CODE           ?PR?UART0_RECV_BYTE?UART0
   *DEL*:           000081H   BYTE   UNIT     CODE           ?PR?_GPIO_OD_SET?GPIO
   *DEL*:           000081H   BYTE   UNIT     CODE           ?PR?_GPIO_CS_SET?GPIO
   *DEL*:           000081H   BYTE   UNIT     CODE           ?PR?_GPIO_DR_SET?GPIO
   *DEL*:           0000BFH   BYTE   UNIT     CODE           ?PR?_GPIO_SR_SET?GPIO
   *DEL*:           000040H   BYTE   UNIT     CODE           ?PR?_GPIO_IRQ_GET?GPIO
   *DEL*:           000098H   BYTE   UNIT     CODE           ?PR?_LPTIMER_IRQ_INIT?LPTIMER
   *DEL*:           000003H   BYTE   UNIT     XDATA          ?XD?_LPTIMER_IRQ_INIT?LPTIMER
   *DEL*:           000036H   BYTE   UNIT     CODE           ?PR?_LPTIMER_PWM_INIT?LPTIMER
   *DEL*:           000109H   BYTE   UNIT     CODE           ?PR?_LPTIMER_PWM_SET?LPTIMER
   *DEL*:           000007H   BYTE   UNIT     XDATA          ?XD?_LPTIMER_PWM_SET?LPTIMER
   *DEL*:           000030H   BYTE   UNIT     CODE           ?PR?_LPTIMER_PWM_CHANNEL_CONFIG?LPTIMER
   *DEL*:           00002DH   BYTE   UNIT     CODE           ?PR?_LPTIMER_CAPTURE_INIT?LPTIMER
   *DEL*:           000021H   BYTE   UNIT     CODE           ?PR?_LPTIMER_GET_LPTCMP?LPTIMER
   *DEL*:           000008H   BYTE   UNIT     CODE           ?PR?LPTIMER_STOP?LPTIMER
   *DEL*:           000010H   BYTE   UNIT     CODE           ?PR?_LPTIMER_TRIGGER_EDGE_SET?LPTIMER
   *DEL*:           000010H   BYTE   UNIT     CODE           ?PR?_LPTIMER_LPTIN_EDGE_SET?LPTIMER
   *DEL*:           000012H   BYTE   UNIT     CODE           ?PR?LPTIM_GET_CNT_VALUE?LPTIMER
   *DEL*:           00003FH   BYTE   UNIT     CODE           ?PR?_LPTIMER_IO_CONFIG?LPTIMER
   *DEL*:           000078H   BYTE   UNIT     CODE           ?PR?_RADIO_RECV_DATA?RADIO
   *DEL*:           000007H   BYTE   UNIT     XDATA          ?XD?_RADIO_RECV_DATA?RADIO
LX51 LINKER/LOCATER V4.66.97.0                                                        06/12/2025  17:35:51  PAGE 5


   *DEL*:           00004AH   BYTE   UNIT     CODE           ?PR?_UM2006A_WRITE_REGS?UM2006A
   *DEL*:           000006H   BYTE   UNIT     XDATA          ?XD?_UM2006A_WRITE_REGS?UM2006A
   *DEL*:           00005BH   BYTE   UNIT     CODE           ?PR?_UM2006A_READ_REGS?UM2006A
   *DEL*:           000007H   BYTE   UNIT     XDATA          ?XD?_UM2006A_READ_REGS?UM2006A
   *DEL*:           00000AH   BYTE   UNIT     CODE           ?PR?_UM2006A_READ_FIFO?UM2006A
   *DEL*:           000007H   BYTE   UNIT     CODE           ?PR?UM2006A_INTO_IDLE?UM2006A
   *DEL*:           00000EH   BYTE   UNIT     CODE           ?PR?UM2006A_INTO_SLEEP?UM2006A
   *DEL*:           00000EH   BYTE   UNIT     CODE           ?PR?UM2006A_INTO_RX?UM2006A
   *DEL*:           00000EH   BYTE   UNIT     CODE           ?PR?UM2006A_INTO_RX_VCOCAL?UM2006A
   *DEL*:           00000EH   BYTE   UNIT     CODE           ?PR?UM2006A_INTO_RX_RC32KCAL?UM2006A
   *DEL*:           00001DH   BYTE   UNIT     CODE           ?PR?_UM2006A_SET_SDO_SEL?UM2006A
   *DEL*:           000001H   BYTE   UNIT     XDATA          ?XD?_UM2006A_SET_SDO_SEL?UM2006A
   *DEL*:           000019H   BYTE   UNIT     CODE           ?PR?_UM2006A_SET_GPIO0_SEL?UM2006A
   *DEL*:           000001H   BYTE   UNIT     XDATA          ?XD?_UM2006A_SET_GPIO0_SEL?UM2006A
   *DEL*:           00001DH   BYTE   UNIT     CODE           ?PR?_UM2006A_SET_GPIO1_SEL?UM2006A
   *DEL*:           000001H   BYTE   UNIT     XDATA          ?XD?_UM2006A_SET_GPIO1_SEL?UM2006A
   *DEL*:           000019H   BYTE   UNIT     CODE           ?PR?_UM2006A_SET_CLKOUT?UM2006A
   *DEL*:           000001H   BYTE   UNIT     XDATA          ?XD?_UM2006A_SET_CLKOUT?UM2006A
   *DEL*:           000126H   BYTE   UNIT     CODE           ?PR?_UM2006A_SET_FREQ?UM2006A
   *DEL*:           000014H   BYTE   UNIT     XDATA          ?XD?_UM2006A_SET_FREQ?UM2006A
   *DEL*:           000021H   BYTE   UNIT     CODE           ?PR?_UM2006A_SET_PAYLOAD_ENABLE?UM2006A
   *DEL*:           000001H   BYTE   UNIT     XDATA          ?XD?_UM2006A_SET_PAYLOAD_ENABLE?UM2006A
   *DEL*:           00001DH   BYTE   UNIT     CODE           ?PR?_UM2006A_SET_PAYLOAD_LENGTH?UM2006A
   *DEL*:           000001H   BYTE   UNIT     XDATA          ?XD?_UM2006A_SET_PAYLOAD_LENGTH?UM2006A
   *DEL*:           00001BH   BYTE   UNIT     CODE           ?PR?_UM2006A_SET_RSSITHR?UM2006A
   *DEL*:           000014H   BYTE   UNIT     CODE           ?PR?UM2006A_READ_RSSI?UM2006A
   *DEL*:           000007H   BYTE   UNIT     CODE           ?PR?UM2006A_CLEAR_VALIDALL?UM2006A
   *DEL*:           00001CH   BYTE   UNIT     CODE           ?PR?_UM2006A_SET_MODULATION?UM2006A
   *DEL*:           000001H   BYTE   UNIT     XDATA          ?XD?_UM2006A_SET_MODULATION?UM2006A
   *DEL*:           00004FH   BYTE   UNIT     CODE           ?PR?_UM2006A_SET_UART_ENABLE?UM2006A
   *DEL*:           000003H   BYTE   UNIT     XDATA          ?XD?_UM2006A_SET_UART_ENABLE?UM2006A
   *DEL*:           000046H   BYTE   UNIT     CODE           ?PR?_UM2006A_SET_WOR_EXTEND?UM2006A
   *DEL*:           000002H   BYTE   UNIT     XDATA          ?XD?_UM2006A_SET_WOR_EXTEND?UM2006A
   *DEL*:           00020FH   BYTE   UNIT     CODE           ?PR?_UM2006A_SET_WOR_CALCULATE?UM2006A
   *DEL*:           000021H   BYTE   UNIT     XDATA          ?XD?_UM2006A_SET_WOR_CALCULATE?UM2006A
   *DEL*:           0002A8H   BYTE   UNIT     CODE           ?PR?_FIND_MATCH_ROWS?UM2006A
   *DEL*:           000013H   BYTE   UNIT     XDATA          ?XD?_FIND_MATCH_ROWS?UM2006A
   *DEL*:           000027H   BYTE   UNIT     CODE           ?PR?_UM2006A_CLEAR_WOR_CONFIG?UM2006A
   *DEL*:           000041H   BYTE   UNIT     CODE           ?PR?_UM2006A_SET_WOR_SLEEP?UM2006A
   *DEL*:           000004H   BYTE   UNIT     XDATA          ?XD?_UM2006A_SET_WOR_SLEEP?UM2006A
   *DEL*:           000103H   BYTE   UNIT     CODE           ?PR?_UM2006A_SET_WOR_T1?UM2006A
   *DEL*:           000009H   BYTE   UNIT     XDATA          ?XD?_UM2006A_SET_WOR_T1?UM2006A
   *DEL*:           000028H   BYTE   UNIT     CODE           ?PR?_UM2006A_SET_WOR_T2_EXT_EN?UM2006A
   *DEL*:           000002H   BYTE   UNIT     XDATA          ?XD?_UM2006A_SET_WOR_T2_EXT_EN?UM2006A
   *DEL*:           000123H   BYTE   UNIT     CODE           ?PR?_UM2006A_SET_WOR_T2?UM2006A
   *DEL*:           000009H   BYTE   UNIT     XDATA          ?XD?_UM2006A_SET_WOR_T2?UM2006A
   *DEL*:           00002EH   BYTE   UNIT     CODE           ?PR?_UM2006A_SET_WOR_T3_EXT_MODE?UM2006A
   *DEL*:           000002H   BYTE   UNIT     XDATA          ?XD?_UM2006A_SET_WOR_T3_EXT_MODE?UM2006A
   *DEL*:           000162H   BYTE   UNIT     CODE           ?PR?_UM2006A_SET_WOR_T3?UM2006A
   *DEL*:           00000AH   BYTE   UNIT     XDATA          ?XD?_UM2006A_SET_WOR_T3?UM2006A
   *DEL*:           0002C0H   BYTE   UNIT     CODE           ?PR?_UM2006A_SET_FSK_SPEED?UM2006A
   *DEL*:           000010H   BYTE   UNIT     XDATA          ?XD?_UM2006A_SET_FSK_SPEED?UM2006A
   *DEL*:           0000F7H   BYTE   UNIT     CODE           ?PR?_UM2006A_SET_OOK_SPEED?UM2006A
   *DEL*:           000006H   BYTE   UNIT     XDATA          ?XD?_UM2006A_SET_OOK_SPEED?UM2006A
   *DEL*:           00004FH   BYTE   UNIT     CODE           ?PR?_UM2006A_SET_MANCHESTER_MODE?UM2006A
   *DEL*:           000003H   BYTE   UNIT     XDATA          ?XD?_UM2006A_SET_MANCHESTER_MODE?UM2006A
   *DEL*:           00000AH   BYTE   UNIT     CODE           ?PR?UM2006A_GET_PJDVALID?UM2006A
   *DEL*:           00000AH   BYTE   UNIT     CODE           ?PR?UM2006A_GET_RSSIVALID?UM2006A
   *DEL*:           00000AH   BYTE   UNIT     CODE           ?PR?UM2006A_GET_SYNCVALID?UM2006A
   *DEL*:           00000AH   BYTE   UNIT     CODE           ?PR?UM2006A_GET_RXBYTE_DONE?UM2006A
   *DEL*:           000046H   BYTE   UNIT     CODE           ?PR?_UM2006A_MASKDEM_SEL?UM2006A
   *DEL*:           000002H   BYTE   UNIT     XDATA          ?XD?_UM2006A_MASKDEM_SEL?UM2006A
   *DEL*:           000046H   BYTE   UNIT     CODE           ?PR?_UM2006A_SET_DUTYCYCLE_MODE?UM2006A
   *DEL*:           000002H   BYTE   UNIT     XDATA          ?XD?_UM2006A_SET_DUTYCYCLE_MODE?UM2006A
   *DEL*:           00002FH   BYTE   UNIT     CODE           ?PR?_UM2006A_SET_PJD_LEN?UM2006A
LX51 LINKER/LOCATER V4.66.97.0                                                        06/12/2025  17:35:51  PAGE 6


   *DEL*:           000001H   BYTE   UNIT     XDATA          ?XD?_UM2006A_SET_PJD_LEN?UM2006A
   *DEL*:           000072H   BYTE   UNIT     CODE           ?PR?_UM2006A_SET_SYNCWORD?UM2006A
   *DEL*:           000006H   BYTE   UNIT     XDATA          ?XD?_UM2006A_SET_SYNCWORD?UM2006A
   *DEL*:           000006H   BYTE   UNIT     CODE           ?PR?UM2006A_HAL_GET_FLAG?UM2006A_HAL
   *DEL*:           000006H   BYTE   UNIT     CODE           ?PR?UM2006A_HAL_CLEAR_FLAG?UM2006A_HAL
   *DEL*:           00000DH   BYTE   UNIT     CODE           ?PR?_FABS?FABS



OVERLAY MAP OF MODULE:   .\Out_Files\UM2006A_RX_DIRECT (?C_STARTUP)


FUNCTION/MODULE                            BIT_GROUP   DATA_GROUP   XDATA_GROUP
--> CALLED FUNCTION/MODULE                START  STOP  START  STOP  START  STOP
===============================================================================
?C_C51STARTUP                             ----- -----  ----- -----  ----- -----
  +--> MAIN/MAIN
  +--> ?C_INITSEG

MAIN/MAIN                                 ----- -----  ----- -----  ----- -----
  +--> SYSTEM_INIT/SYSTEM_UM800Y
  +--> APP_INIT/APP
  +--> APP_RUN/APP

SYSTEM_INIT/SYSTEM_UM800Y                 ----- -----  ----- -----  ----- -----
  +--> _CLOCK_INIT/SYSTEM_UM800Y

_CLOCK_INIT/SYSTEM_UM800Y                 ----- -----  ----- -----  025FH 0266H

APP_INIT/APP                              ----- -----  ----- -----  ----- -----
  +--> _UART0_INIT/UART0
  +--> PRINTF/PRINTF
  +--> APP_UM2006A_INIT/APP_UM2006A

_UART0_INIT/UART0                         ----- -----  ----- -----  025FH 0262H
  +--> _UART0_SET_BAUD_RATE/UART0

_UART0_SET_BAUD_RATE/UART0                ----- -----  ----- -----  0263H 026EH

PRINTF/PRINTF                             20H.0 21H.0  0008H 000CH  02A1H 02D0H
  +--> _PUTCHAR/UART0

_PUTCHAR/UART0                            ----- -----  ----- -----  ----- -----
  +--> _UART0_SEND_BYTE/UART0

_UART0_SEND_BYTE/UART0                    ----- -----  ----- -----  ----- -----

APP_UM2006A_INIT/APP_UM2006A              ----- -----  ----- -----  ----- -----
  +--> RADIO_INIT/RADIO
  +--> APP_EV1527_INIT/APP_EV1527

RADIO_INIT/RADIO                          ----- -----  ----- -----  ----- -----
  +--> UM2006A_HAL_INIT/UM2006A_HAL
  +--> UM2006A_INIT/UM2006A
  +--> UM2006A_INTO_RX_BPFCAL/UM2006A

UM2006A_HAL_INIT/UM2006A_HAL              ----- -----  ----- -----  ----- -----
  +--> _GPIO_INIT/GPIO
  +--> _GPIO_DIR_SET/GPIO
  +--> _GPIO_IN_ENABLE/GPIO
  +--> _GPIO_PD_SET/GPIO
  +--> UM2006A_HAL_IRQ/UM2006A_HAL
  +--> _GPIO_IRQ_SET/GPIO

_GPIO_INIT/GPIO                           ----- -----  ----- -----  0261H 0261H
LX51 LINKER/LOCATER V4.66.97.0                                                        06/12/2025  17:35:51  PAGE 7



_GPIO_DIR_SET/GPIO                        ----- -----  ----- -----  ----- -----

_GPIO_IN_ENABLE/GPIO                      ----- -----  ----- -----  ----- -----

_GPIO_PD_SET/GPIO                         ----- -----  ----- -----  ----- -----

UM2006A_HAL_IRQ/UM2006A_HAL               ----- -----  ----- -----  ----- -----

_GPIO_IRQ_SET/GPIO                        ----- -----  ----- -----  025FH 0260H
  +--> _GPIO_IRQ_CLR/GPIO

_GPIO_IRQ_CLR/GPIO                        ----- -----  ----- -----  ----- -----

UM2006A_INIT/UM2006A                      ----- -----  ----- -----  025FH 0260H
  +--> SPI_INIT/UM2006A_HAL
  +--> UM2006A_RESET_DIGIT/UM2006A
  +--> _DELAY_MS/COMMON
  +--> _UM2006A_WRITE_REG/UM2006A
  +--> UM2006A_CAL_RC32K/UM2006A

SPI_INIT/UM2006A_HAL                      ----- -----  ----- -----  ----- -----
  +--> _GPIO_INIT/GPIO
  +--> _GPIO_DIR_SET/GPIO
  +--> _GPIO_PU_SET/GPIO
  +--> _GPIO_IO_SET/GPIO
  +--> _GPIO_IN_ENABLE/GPIO

_GPIO_PU_SET/GPIO                         ----- -----  ----- -----  ----- -----

_GPIO_IO_SET/GPIO                         ----- -----  ----- -----  ----- -----

UM2006A_RESET_DIGIT/UM2006A               ----- -----  ----- -----  ----- -----
  +--> _UM2006A_WRITE_REG/UM2006A

_UM2006A_WRITE_REG/UM2006A                ----- -----  ----- -----  0268H 0269H
  +--> SPI_CS_ENABLE/UM2006A_HAL
  +--> _SPI_WRITE_BYTE/UM2006A_HAL
  +--> SPI_CS_DISABLE/UM2006A_HAL

SPI_CS_ENABLE/UM2006A_HAL                 ----- -----  ----- -----  ----- -----
  +--> _GPIO_IO_SET/GPIO

_SPI_WRITE_BYTE/UM2006A_HAL               ----- -----  ----- -----  026AH 026BH
  +--> _GPIO_DIR_SET/GPIO
  +--> _GPIO_IO_SET/GPIO

SPI_CS_DISABLE/UM2006A_HAL                ----- -----  ----- -----  ----- -----
  +--> _GPIO_IO_SET/GPIO
  +--> _GPIO_DIR_SET/GPIO

_DELAY_MS/COMMON                          ----- -----  ----- -----  0261H 0268H

UM2006A_CAL_RC32K/UM2006A                 ----- -----  ----- -----  0261H 0267H
  +--> _UM2006A_READ_REG/UM2006A
  +--> _UM2006A_WRITE_REG/UM2006A

_UM2006A_READ_REG/UM2006A                 ----- -----  ----- -----  0268H 0269H
  +--> SPI_CS_ENABLE/UM2006A_HAL
  +--> _SPI_WRITE_BYTE/UM2006A_HAL
  +--> SPI_READ_BYTE/UM2006A_HAL
  +--> SPI_CS_DISABLE/UM2006A_HAL

SPI_READ_BYTE/UM2006A_HAL                 ----- -----  ----- -----  026AH 026BH
  +--> _GPIO_DIR_SET/GPIO
LX51 LINKER/LOCATER V4.66.97.0                                                        06/12/2025  17:35:51  PAGE 8


  +--> _GPIO_IO_SET/GPIO
  +--> _GPIO_IO_GET/GPIO

_GPIO_IO_GET/GPIO                         ----- -----  ----- -----  ----- -----

UM2006A_INTO_RX_BPFCAL/UM2006A            ----- -----  ----- -----  ----- -----
  +--> _UM2006A_WRITE_REG/UM2006A

APP_EV1527_INIT/APP_EV1527                ----- -----  ----- -----  ----- -----
  +--> _GPIO_INIT/GPIO
  +--> _GPIO_IN_ENABLE/GPIO
  +--> _GPIO_DIR_SET/GPIO
  +--> _GPIO_PU_SET/GPIO
  +--> _GPIO_IRQ_SET/GPIO
  +--> _LPTIMER_INIT/LPTIMER
  +--> _LPTIMER_SET_TIME/LPTIMER
  +--> LPTIMER_START/LPTIMER

_LPTIMER_INIT/LPTIMER                     ----- -----  ----- -----  ----- -----

_LPTIMER_SET_TIME/LPTIMER                 ----- -----  ----- -----  ----- -----

LPTIMER_START/LPTIMER                     ----- -----  ----- -----  ----- -----

APP_RUN/APP                               ----- -----  ----- -----  ----- -----
  +--> APP_UM2006A_RUN/APP_UM2006A

APP_UM2006A_RUN/APP_UM2006A               ----- -----  ----- -----  025FH 02A0H
  +--> _APP_EV1527_RECV_DATA/APP_EV1527
  +--> PRINTF/PRINTF

_APP_EV1527_RECV_DATA/APP_EV1527          ----- -----  ----- -----  02A1H 02A7H

?C_INITSEG                                ----- -----  ----- -----  ----- -----

*** NEW ROOT ****************************

UART0_IRQHANDLER/UART0                    ----- -----  ----- -----  ----- -----

*** NEW ROOT ****************************

LPTIMER_IRQHANDLER/LPTIMER                ----- -----  ----- -----  ----- -----

*** NEW ROOT ****************************

GPIO_IRQHANDLER/APP_EV1527                ----- -----  ----- -----  ----- -----



PUBLIC SYMBOLS OF MODULE:  .\Out_Files\UM2006A_RX_DIRECT (?C_STARTUP)


      VALUE       CLASS    TYPE      PUBLIC SYMBOL NAME
      =================================================
      020002A1H   XDATA    BYTE      ?_app_ev1527_recv_data?BYTE
*DEL*:00000000H   XDATA    BYTE      ?_find_match_rows?BYTE
*DEL*:00000000H   XDATA    BYTE      ?_lptimer_pwm_set?BYTE
      020002A1H   XDATA    ---       ?_PRINTF?BYTE
*DEL*:00000000H   XDATA    BYTE      ?_radio_recv_data?BYTE
      020002A1H   XDATA    ---       ?_SPRINTF?BYTE
*DEL*:00000000H   XDATA    BYTE      ?_um2006A_read_regs?BYTE
*DEL*:00000000H   XDATA    BYTE      ?_um2006A_set_freq?BYTE
*DEL*:00000000H   XDATA    BYTE      ?_um2006A_set_syncword?BYTE
*DEL*:00000000H   XDATA    BYTE      ?_um2006A_write_regs?BYTE
      010003CCH   CODE     ---       ?C?CASTF
LX51 LINKER/LOCATER V4.66.97.0                                                        06/12/2025  17:35:51  PAGE 9


      010009F6H   CODE     ---       ?C?CCASE
      0100070EH   CODE     ---       ?C?CLDOPTR
      010006F5H   CODE     ---       ?C?CLDPTR
      00000000H   NUMBER   ---       ?C?CODESEG
      010006CFH   CODE     ---       ?C?COPY
      0100074DH   CODE     ---       ?C?CSTOPTR
      0100073BH   CODE     ---       ?C?CSTPTR
      01000398H   CODE     ---       ?C?FCASTC
      01000393H   CODE     ---       ?C?FCASTI
      0100038EH   CODE     ---       ?C?FCASTL
      0100006DH   CODE     ---       ?C?FPADD
      01000306H   CODE     ---       ?C?FPCMP
      01000304H   CODE     ---       ?C?FPCMP3
      0100048AH   CODE     ---       ?C?FPCONVERT
      01000267H   CODE     ---       ?C?FPDIV
      01000403H   CODE     ---       ?C?FPGETOPN2
      0100015EH   CODE     ---       ?C?FPMUL
      01000438H   CODE     ---       ?C?FPNANRESULT
      0100037DH   CODE     ---       ?C?FPNEG
      01000442H   CODE     ---       ?C?FPOVERFLOW
      0100041AH   CODE     ---       ?C?FPRESULT
      0100042EH   CODE     ---       ?C?FPRESULT2
      0100044DH   CODE     ---       ?C?FPROUND
      01000069H   CODE     ---       ?C?FPSUB
      0100043FH   CODE     ---       ?C?FPUNDERFLOW
      010005BFH   CODE     ---       ?C?FTNPWR
      01000A56H   CODE     ---       ?C?ICALL
      01000A5AH   CODE     ---       ?C?ICALL2
      0100076FH   CODE     ---       ?C?IMUL
      01000781H   CODE     ---       ?C?LADD
      01000A1CH   CODE     ---       ?C?LCASE
      01000AA0H   CODE     ---       ?C?LLDCODE
      01000A88H   CODE     ---       ?C?LLDIDATA
      01000964H   CODE     ---       ?C?LLDIXDATA
      0100095BH   CODE     ---       ?C?LLDIXDATA1
      0100095DH   CODE     ---       ?C?LLDIXDATA8
      01000913H   CODE     ---       ?C?LLDOPTR
      01000A94H   CODE     ---       ?C?LLDPDATA
      01000943H   CODE     ---       ?C?LLDXDATA
      0100094FH   CODE     ---       ?C?LLDXDATA0
      0100078EH   CODE     ---       ?C?LMUL
      010008B8H   CODE     ---       ?C?LNEG
      010008ABH   CODE     ---       ?C?LOR
      01000900H   CODE     ---       ?C?LSHL
      0100099CH   CODE     ---       ?C?LSTKXDATA
      01000990H   CODE     ---       ?C?LSTXDATA
      01000A5CH   CODE     ---       ?C?MEMSET
      010009D6H   CODE     ---       ?C?PLDIXDATA
      010009CDH   CODE     ---       ?C?PLDXDATA
      010009EDH   CODE     ---       ?C?PSTXDATA
      010008C6H   CODE     ---       ?C?SLCMP
      01001CFDH   CODE     ---       ?C?SLDIV
      010008DCH   CODE     ---       ?C?ULCMP
      01000819H   CODE     ---       ?C?ULDIV
      010008EDH   CODE     ---       ?C?ULSHR
      00000000H   NUMBER   ---       ?C?XDATASEG
      01001684H   CODE     ---       ?C_START
      01000000H   CODE     ---       ?C_STARTUP
      010016C9H   CODE     ---       _app_ev1527_recv_data
      01001130H   CODE     ---       _clock_init
*DEL*:00000000H   CODE     ---       _delay
      01001C70H   CODE     ---       _delay_ms
*DEL*:00000000H   CODE     ---       _FABS
*DEL*:00000008H   CODE     ---       _find_match_rows
*DEL*:00000000H   CODE     ---       _gpio_cs_set
LX51 LINKER/LOCATER V4.66.97.0                                                        06/12/2025  17:35:51  PAGE 10


      01001753H   CODE     ---       _gpio_dir_set
*DEL*:00000000H   CODE     ---       _gpio_dr_set
      010014E3H   CODE     ---       _gpio_in_enable
      01001DC1H   CODE     ---       _gpio_init
      01001D41H   CODE     ---       _gpio_io_get
      010018D6H   CODE     ---       _gpio_io_set
      01001CB7H   CODE     ---       _gpio_irq_clr
*DEL*:00000000H   CODE     ---       _gpio_irq_get
      01001420H   CODE     ---       _gpio_irq_set
*DEL*:00000000H   CODE     ---       _gpio_od_set
      01001855H   CODE     ---       _gpio_pd_set
      010017D4H   CODE     ---       _gpio_pu_set
*DEL*:00000000H   CODE     ---       _gpio_sr_set
*DEL*:00000000H   CODE     ---       _lptimer_capture_init
*DEL*:00000000H   CODE     ---       _lptimer_get_lptcmp
      01001E2BH   CODE     ---       _lptimer_init
*DEL*:00000000H   CODE     ---       _lptimer_io_config
*DEL*:00000000H   CODE     ---       _lptimer_irq_init
*DEL*:00000000H   CODE     ---       _lptimer_lptin_edge_set
*DEL*:00000000H   CODE     ---       _lptimer_pwm_channel_config
*DEL*:00000000H   CODE     ---       _lptimer_pwm_init
*DEL*:00000000H   CODE     ---       _lptimer_pwm_set
      01001F05H   CODE     ---       _lptimer_set_time
*DEL*:00000000H   CODE     ---       _lptimer_trigger_edge_set
      01000B1BH   CODE     ---       _PRINTF
*DEL*:00000000H   CODE     ---       _printf_buff_byte
*DEL*:00000000H   CODE     ---       _printf_buff_word
      01001F1DH   CODE     ---       _putchar
*DEL*:00000000H   CODE     ---       _radio_recv_data
      01001B7BH   CODE     ---       _spi_write_byte
      01000B15H   CODE     ---       _SPRINTF
      01000026H   CODE     ---       _uart0_init
*DEL*:00000000H   CODE     ---       _uart0_irq_init
      01000006H   CODE     ---       _uart0_send_byte
*DEL*:00000000H   CODE     ---       _uart0_send_bytes
*DEL*:00000004H   CODE     ---       _um2006A_clear_wor_config
*DEL*:00000000H   CODE     ---       _um2006A_maskdem_sel
*DEL*:00000000H   CODE     ---       _um2006A_read_fifo
      01001E92H   CODE     ---       _um2006A_read_reg
*DEL*:00000000H   CODE     ---       _um2006A_read_regs
*DEL*:00000000H   CODE     ---       _um2006A_set_clkout
*DEL*:00000000H   CODE     ---       _um2006A_set_dutycycle_mode
*DEL*:00000000H   CODE     ---       _um2006A_set_freq
*DEL*:00000000H   CODE     ---       _um2006A_set_fsk_speed
*DEL*:00000000H   CODE     ---       _um2006A_set_gpio0_sel
*DEL*:00000000H   CODE     ---       _um2006A_set_gpio1_sel
*DEL*:00000000H   CODE     ---       _um2006A_set_manchester_mode
*DEL*:00000000H   CODE     ---       _um2006A_set_modulation
*DEL*:00000000H   CODE     ---       _um2006A_set_ook_speed
*DEL*:00000000H   CODE     ---       _um2006A_set_payload_enable
*DEL*:00000000H   CODE     ---       _um2006A_set_payload_length
*DEL*:00000000H   CODE     ---       _um2006A_set_pjd_len
*DEL*:00000000H   CODE     ---       _um2006A_set_rssithr
*DEL*:00000000H   CODE     ---       _um2006A_set_sdo_sel
*DEL*:00000000H   CODE     ---       _um2006A_set_syncword
*DEL*:00000000H   CODE     ---       _um2006A_set_uart_enable
*DEL*:00000005H   CODE     ---       _um2006A_set_wor_calculate
*DEL*:00000000H   CODE     ---       _um2006A_set_wor_extend
*DEL*:00000000H   CODE     ---       _um2006A_set_wor_sleep
*DEL*:00000000H   CODE     ---       _um2006A_set_wor_t1
*DEL*:00000000H   CODE     ---       _um2006A_set_wor_t2
*DEL*:00000000H   CODE     ---       _um2006A_set_wor_t2_ext_en
*DEL*:00000000H   CODE     ---       _um2006A_set_wor_t3
*DEL*:00000000H   CODE     ---       _um2006A_set_wor_t3_ext_mode
      01001E0AH   CODE     ---       _um2006A_write_reg
LX51 LINKER/LOCATER V4.66.97.0                                                        06/12/2025  17:35:51  PAGE 11


*DEL*:00000000H   CODE     ---       _um2006A_write_regs
*SFR* 000000D0H.6 DATA     BIT       AC
*SFR* 000000E0H   DATA     BYTE      ACC
*SFR* 000000E0H.0 DATA     BIT       ACC0
*SFR* 000000E0H.1 DATA     BIT       ACC1
*SFR* 000000E0H.2 DATA     BIT       ACC2
*SFR* 000000E0H.3 DATA     BIT       ACC3
*SFR* 000000E0H.4 DATA     BIT       ACC4
*SFR* 000000E0H.5 DATA     BIT       ACC5
*SFR* 000000E0H.6 DATA     BIT       ACC6
*SFR* 000000E0H.7 DATA     BIT       ACC7
*SFR* 000000FEH   DATA     BYTE      ADCCDR0
*SFR* 000000FFH   DATA     BYTE      ADCCDR1
*SFR* 000000F6H   DATA     BYTE      ADCCSTAT
*SFR* 000000B6H   DATA     WORD      ADCDR
*SFR* 000000B6H   DATA     BYTE      ADCDR0
*SFR* 000000B7H   DATA     BYTE      ADCDR1
*SFR* 000000ACH   DATA     BYTE      ADCGCR0
*SFR* 000000ADH   DATA     BYTE      ADCGCR1
*SFR* 000000B4H   DATA     BYTE      ADCGCR2
*SFR* 000000B5H   DATA     BYTE      ADCGCR3
*SFR* 000000F5H   DATA     BYTE      ADCHL
*SFR* 00000093H   DATA     BYTE      ADCIER
*SFR* 000000F7H   DATA     BYTE      ADCSPW
*SFR* 000000FDH   DATA     BYTE      ADCVREF
      01001D81H   CODE     ---       app_ev1527_init
      01001B1AH   CODE     ---       app_init
      01001F22H   CODE     ---       app_run
      0100005DH   CODE     ---       app_um2006A_init
      01001957H   CODE     ---       app_um2006A_run
*SFR* 000000F0H   DATA     BYTE      B
*SFR* 000000F0H.0 DATA     BIT       B0
*SFR* 000000F0H.1 DATA     BIT       B1
*SFR* 000000F0H.2 DATA     BIT       B2
*SFR* 000000F0H.3 DATA     BIT       B3
*SFR* 000000F0H.4 DATA     BIT       B4
*SFR* 000000F0H.5 DATA     BIT       B5
*SFR* 000000F0H.6 DATA     BIT       B6
*SFR* 000000F0H.7 DATA     BIT       B7
*SFR* 00000086H   DATA     BYTE      BEEPCTR
*SFR* 000000F8H   DATA     BYTE      CLKCON
*SFR* 000000B1H   DATA     BYTE      CLKST
*SFR* 000000D0H.7 DATA     BIT       CY
      02000158H   XDATA    WORD      cycle
*SFR* 00000083H   DATA     BYTE      DPH
*SFR* 00000085H   DATA     BYTE      DPH1
*SFR* 00000082H   DATA     BYTE      DPL
*SFR* 00000084H   DATA     BYTE      DPL1
*SFR* 00000092H   DATA     BYTE      DPS
*SFR* 000000A8H.7 DATA     BIT       EA
*SFR* 000000A8H.6 DATA     BIT       EADC
*SFR* 000000B8H.3 DATA     BIT       EFCINTEN
*SFR* 000000A8H.5 DATA     BIT       EPWM
*SFR* 000000D8H.3 DATA     BIT       ERSTF
*SFR* 000000A8H.4 DATA     BIT       ES0
*SFR* 000000A8H.2 DATA     BIT       ES1
*SFR* 000000B2H   DATA     BYTE      ESTCR
*SFR* 000000A8H.1 DATA     BIT       ET0
*SFR* 000000A8H.3 DATA     BIT       ET1
*SFR* 0000009EH   DATA     BYTE      EUARTEN
*SFR* 000000A8H.0 DATA     BIT       EX0
*SFR* 000000D0H.5 DATA     BIT       F0
*SFR* 000000D0H.1 DATA     BIT       F1
      0200015FH   XDATA    ---       g_recv_data
      0200015EH   XDATA    BYTE      g_recv_index
LX51 LINKER/LOCATER V4.66.97.0                                                        06/12/2025  17:35:51  PAGE 12


      0100125EH   CODE     ---       GPIO_IRQHandler
      020002D1H   XDATA    ---       gpiofunc
*SFR* 000000B8H.0 DATA     BIT       GTIM0INTEN
*SFR* 000000B8H.2 DATA     BIT       GTIM1INTEN
*SFR* 000000B8H.6 DATA     BIT       GTIM2INTEN
      0200015CH   XDATA    WORD      high_time
*SFR* 000000B8H.5 DATA     BIT       I2CINTEN
*SFR* 000000A8H   DATA     BYTE      IEN0
*SFR* 000000B8H   DATA     BYTE      IEN1
*SFR* 0000009AH   DATA     BYTE      IEN2
*SFR* 000000A9H   DATA     BYTE      IP0
*SFR* 000000B9H   DATA     BYTE      IP1
*SFR* 000000BDH   DATA     BYTE      LDOTRIMH
*SFR* 00000091H   DATA     BYTE      LDOTRIML
*DEL*:00000000H   CODE     ---       lptim_get_cnt_value
      01001358H   CODE     ---       LPTIMER_IRQHandler
      01001F0EH   CODE     ---       lptimer_start
*DEL*:00000000H   CODE     ---       lptimer_stop
      02000319H   XDATA    ---       lptimfunc
*SFR* 000000B8H.4 DATA     BIT       LPTIMINTEN
*SFR* 000000DDH   DATA     BYTE      LVDCON
*SFR* 000000D8H.5 DATA     BIT       LVRF
      01001EFAH   CODE     ---       main
*SFR* 000000D1H   DATA     WORD      OADR
*SFR* 000000D2H   DATA     BYTE      OADRH
*SFR* 000000D1H   DATA     BYTE      OADRL
*SFR* 000000D4H   DATA     BYTE      OCTRL
*SFR* 000000D3H   DATA     BYTE      ODATA
*SFR* 000000A2H   DATA     BYTE      OINTEN
*SFR* 000000A3H   DATA     BYTE      OINTUS
*SFR* 000000A7H   DATA     BYTE      OPSET
*SFR* 000000A5H   DATA     BYTE      OSEC
*SFR* 000000A6H   DATA     BYTE      OSTATUS
*SFR* 000000A1H   DATA     BYTE      OUS
*SFR* 000000D0H.0 DATA     BIT       P
*SFR* 00000080H   DATA     BYTE      P0
*SFR* 00000080H.0 DATA     BIT       P00
*SFR* 00000080H.1 DATA     BIT       P01
*SFR* 00000080H.2 DATA     BIT       P02
*SFR* 00000080H.3 DATA     BIT       P03
*SFR* 00000080H.4 DATA     BIT       P04
*SFR* 00000080H.5 DATA     BIT       P05
*SFR* 000000ABH   DATA     BYTE      P0AH
*SFR* 000000A4H   DATA     BYTE      P0AL
*SFR* 000000D7H   DATA     BYTE      P0CS
*SFR* 00000097H   DATA     BYTE      P0DR
*SFR* 000000E9H   DATA     BYTE      P0IEN
*SFR* 000000E1H   DATA     BYTE      P0IRQ
*SFR* 000000D6H   DATA     BYTE      P0OD
*SFR* 000000F9H   DATA     BYTE      P0OEN
*SFR* 000000D5H   DATA     BYTE      P0PD
*SFR* 000000F1H   DATA     BYTE      P0PU
*SFR* 00000090H   DATA     BYTE      P1
*SFR* 00000090H.0 DATA     BIT       P10
*SFR* 00000090H.1 DATA     BIT       P11
*SFR* 00000090H.2 DATA     BIT       P12
*SFR* 00000090H.3 DATA     BIT       P13
*SFR* 00000090H.4 DATA     BIT       P14
*SFR* 00000090H.5 DATA     BIT       P15
*SFR* 000000B0H   DATA     BYTE      P1AH
*SFR* 000000AEH   DATA     BYTE      P1AL
*SFR* 000000DCH   DATA     BYTE      P1CS
*SFR* 000000E5H   DATA     BYTE      P1DR
*SFR* 000000EAH   DATA     BYTE      P1IEN
*SFR* 000000E2H   DATA     BYTE      P1IRQ
LX51 LINKER/LOCATER V4.66.97.0                                                        06/12/2025  17:35:51  PAGE 13


*SFR* 000000DBH   DATA     BYTE      P1OD
*SFR* 000000FAH   DATA     BYTE      P1OEN
*SFR* 000000DAH   DATA     BYTE      P1PD
*SFR* 000000F2H   DATA     BYTE      P1PU
*SFR* 000000A0H   DATA     BYTE      P2
*SFR* 000000A0H.0 DATA     BIT       P20
*SFR* 000000A0H.2 DATA     BIT       P22
*SFR* 000000A0H.3 DATA     BIT       P23
*SFR* 000000A0H.5 DATA     BIT       P25
*SFR* 000000A0H.6 DATA     BIT       P26
*SFR* 000000A0H.7 DATA     BIT       P27
*SFR* 000000E8H   DATA     BYTE      P2AH
*SFR* 000000C0H   DATA     BYTE      P2AL
*SFR* 000000F4H   DATA     BYTE      P2CS
*SFR* 000000FCH   DATA     BYTE      P2DR
*SFR* 000000EBH   DATA     BYTE      P2IEN
*SFR* 000000E3H   DATA     BYTE      P2IRQ
*SFR* 000000ECH   DATA     BYTE      P2OD
*SFR* 000000FBH   DATA     BYTE      P2OEN
*SFR* 000000E4H   DATA     BYTE      P2PD
*SFR* 000000F3H   DATA     BYTE      P2PU
*SFR* 000000DEH   DATA     BYTE      PCLK0
*SFR* 000000DFH   DATA     BYTE      PCLK1
*SFR* 00000087H   DATA     BYTE      PCON
*SFR* 0000008EH   DATA     BYTE      PDSEL
*SFR* 0000008FH   DATA     BYTE      POREN
*SFR* 000000D8H.4 DATA     BIT       PORF
*SFR* 000000E6H   DATA     BYTE      PRESET0
*SFR* 000000E7H   DATA     BYTE      PRESET1
*SFR* 000000D0H   DATA     BYTE      PSW
*SFR* 000000C8H   DATA     BYTE      PWM0CON
*SFR* 000000C4H   DATA     BYTE      PWM0DH
*SFR* 000000C3H   DATA     BYTE      PWM0DL
*SFR* 000000C8H.7 DATA     BIT       PWM0EN
*SFR* 000000C8H.2 DATA     BIT       PWM0IE
*SFR* 000000C8H.1 DATA     BIT       PWM0IF
*SFR* 000000CCH   DATA     BYTE      PWM0PH
*SFR* 000000CBH   DATA     BYTE      PWM0PL
*SFR* 000000C8H.6 DATA     BIT       PWM0S
*SFR* 000000C8H.0 DATA     BIT       PWM0SS
*SFR* 000000C9H   DATA     BYTE      PWM1CON
*SFR* 000000C6H   DATA     BYTE      PWM1DH
*SFR* 000000C5H   DATA     BYTE      PWM1DL
*SFR* 000000CEH   DATA     BYTE      PWM1PH
*SFR* 000000CDH   DATA     BYTE      PWM1PL
*SFR* 000000CAH   DATA     BYTE      PWM2CON
*SFR* 000000C7H   DATA     BYTE      PWM2DH
*SFR* 000000CFH   DATA     BYTE      PWM2DL
*SFR* 000000C2H   DATA     BYTE      PWM2PH
*SFR* 000000C1H   DATA     BYTE      PWM2PL
      01001EE3H   CODE     ---       radio_init
*SFR* 00000098H.2 DATA     BIT       RB80
*SFR* 000000F8H.2 DATA     BIT       RC16MEN
*SFR* 000000F8H.5 DATA     BIT       RC16MF
*SFR* 000000F8H.3 DATA     BIT       RC32KEN
*SFR* 000000F8H.6 DATA     BIT       RC32KF
      02000325H   XDATA    DWORD     rch24m
*SFR* 000000EEH   DATA     BYTE      RCHDIV
*SFR* 000000BEH   DATA     BYTE      RCHTRIMH
*SFR* 000000BFH   DATA     BYTE      RCHTRIML
*SFR* 0000009FH   DATA     BYTE      RCLTRIMH
*SFR* 000000BCH   DATA     BYTE      RCLTRIML
*SFR* 000000AFH   DATA     BYTE      REMAP
*SFR* 00000098H.4 DATA     BIT       REN0
      02000000H   XDATA    ---       rf_config
LX51 LINKER/LOCATER V4.66.97.0                                                        06/12/2025  17:35:51  PAGE 14


*SFR* 00000098H.0 DATA     BIT       RI0
*SFR* 000000D0H.3 DATA     BIT       RS0
*SFR* 000000D0H.4 DATA     BIT       RS1
*SFR* 000000D8H   DATA     BYTE      RSTSTAT
*SFR* 00000099H   DATA     BYTE      S0BUF
*SFR* 00000098H   DATA     BYTE      S0CON
*SFR* 000000BAH   DATA     BYTE      S0RELH
*SFR* 000000AAH   DATA     BYTE      S0RELL
*SFR* 0000009CH   DATA     BYTE      S1BUF
*SFR* 0000009BH   DATA     BYTE      S1CON
*SFR* 000000BBH   DATA     BYTE      S1RELH
*SFR* 0000009DH   DATA     BYTE      S1RELL
*SFR* 00000098H.7 DATA     BIT       SM0
*SFR* 00000098H.6 DATA     BIT       SM1
*SFR* 00000098H.5 DATA     BIT       SM20
*SFR* 00000081H   DATA     BYTE      SP
      01001ED5H   CODE     ---       spi_cs_disable
      01001F16H   CODE     ---       spi_cs_enable
      01001BD6H   CODE     ---       spi_init
      01001AB6H   CODE     ---       spi_read_byte
*SFR* 000000B8H.1 DATA     BIT       SPIINTEN
*SFR* 000000D9H   DATA     BYTE      SYSDIV
*SFR* 000000F8H.0 DATA     BIT       SYSSEL
      02000329H   XDATA    DWORD     system_core_clock
      01001EEFH   CODE     ---       system_init
*SFR* 00000098H.3 DATA     BIT       TB80
*SFR* 00000098H.1 DATA     BIT       TI0
      0200015AH   XDATA    WORD      time
      0200032DH   XDATA    BYTE      tx_flag
      0200032EH   XDATA    ---       uart0_func
      01001C26H   CODE     ---       UART0_IRQHandler
*DEL*:00000000H   CODE     ---       uart0_recv_byte
*SFR* 000000B8H.7 DATA     BIT       UART2INTEN
      010015A2H   CODE     ---       um2006A_cal_rc32K
*DEL*:00000000H   CODE     ---       um2006A_clear_validall
*DEL*:00000000H   CODE     ---       um2006A_get_pjdvalid
*DEL*:00000000H   CODE     ---       um2006A_get_rssivalid
*DEL*:00000000H   CODE     ---       um2006A_get_rxbyte_done
*DEL*:00000000H   CODE     ---       um2006A_get_syncvalid
*DEL*:00000000H   CODE     ---       um2006A_hal_clear_flag
*DEL*:00000000H   CODE     ---       um2006A_hal_get_flag
      01001E5BH   CODE     ---       um2006A_hal_init
      0100001CH   CODE     ---       um2006A_hal_irq
      01001A4EH   CODE     ---       um2006A_init
*DEL*:00000000H   CODE     ---       um2006A_into_idle
*DEL*:00000000H   CODE     ---       um2006A_into_rx
      01001EB9H   CODE     ---       um2006A_into_rx_bpfcal
*DEL*:00000000H   CODE     ---       um2006A_into_rx_rc32kcal
*DEL*:00000000H   CODE     ---       um2006A_into_rx_vcocal
*DEL*:00000000H   CODE     ---       um2006A_into_sleep
*DEL*:00000000H   CODE     ---       um2006A_read_rssi
      01001EC7H   CODE     ---       um2006A_reset_digit
*SFR* 000000D8H.6 DATA     BIT       WDEN
*SFR* 000000D8H.7 DATA     BIT       WDOF
*SFR* 000000D8H.0 DATA     BIT       WDT0
*SFR* 000000D8H.1 DATA     BIT       WDT1
*SFR* 000000D8H.2 DATA     BIT       WDT2
*SFR* 000000F8H.1 DATA     BIT       XCLKEN
*SFR* 000000F8H.4 DATA     BIT       XCLKF
*SFR* 000000B3H   DATA     BYTE      XTHCTR



SYMBOL TABLE OF MODULE:  .\Out_Files\UM2006A_RX_DIRECT (?C_STARTUP)

LX51 LINKER/LOCATER V4.66.97.0                                                        06/12/2025  17:35:51  PAGE 15


      VALUE       REP       CLASS    TYPE      SYMBOL NAME
      ====================================================
      ---         MODULE    ---      ---       ?C_STARTUP
      01000000H   PUBLIC    CODE     ---       ?C_STARTUP
      000000E0H   SYMBOL    DATA     ---       ACC
      000000F0H   SYMBOL    DATA     ---       B
      00000083H   SYMBOL    DATA     ---       DPH
      00000082H   SYMBOL    DATA     ---       DPL
      00000000H   SYMBOL    NUMBER   ---       IBPSTACK
      00000100H   SYMBOL    NUMBER   ---       IBPSTACKTOP
      000000A0H   SYMBOL    NUMBER   ---       IDATALEN
      01001640H   SYMBOL    CODE     ---       IDATALOOP
      00000000H   SYMBOL    NUMBER   ---       PBPSTACK
      00000100H   SYMBOL    NUMBER   ---       PBPSTACKTOP
      00000000H   SYMBOL    NUMBER   ---       PDATALEN
      00000000H   SYMBOL    NUMBER   ---       PDATASTART
      00000000H   SYMBOL    NUMBER   ---       PPAGE
      00000000H   SYMBOL    NUMBER   ---       PPAGEENABLE
      000000A0H   SYMBOL    DATA     ---       PPAGE_SFR
      00000081H   SYMBOL    DATA     ---       SP
      0100163DH   SYMBOL    CODE     ---       STARTUP1
      00000000H   SYMBOL    NUMBER   ---       XBPSTACK
      00000000H   SYMBOL    NUMBER   ---       XBPSTACKTOP
      00000000H   SYMBOL    NUMBER   ---       XDATALEN
      00000000H   SYMBOL    NUMBER   ---       XDATASTART
      01000000H   LINE      CODE     ---       #126
      0100163DH   LINE      CODE     ---       #134
      0100163FH   LINE      CODE     ---       #135
      01001640H   LINE      CODE     ---       #136
      01001641H   LINE      CODE     ---       #137
      01001643H   LINE      CODE     ---       #191
      01001646H   LINE      CODE     ---       #205

      ---         MODULE    ---      ---       SYSTEM_UM800Y
      02000329H   PUBLIC    XDATA    DWORD     system_core_clock
      02000325H   PUBLIC    XDATA    DWORD     rch24m
      01001EEFH   PUBLIC    CODE     ---       system_init
      01001130H   PUBLIC    CODE     ---       _clock_init
      00000098H.3 SFRSYM    DATA     BIT       TB80
      000000E0H.7 SFRSYM    DATA     BIT       ACC7
      00000080H   SFRSYM    DATA     BYTE      P0
      00000090H   SFRSYM    DATA     BYTE      P1
      000000A0H   SFRSYM    DATA     BYTE      P2
      00000098H.5 SFRSYM    DATA     BIT       SM20
      000000B2H   SFRSYM    DATA     BYTE      ESTCR
      000000B1H   SFRSYM    DATA     BYTE      CLKST
      000000D0H.6 SFRSYM    DATA     BIT       AC
      000000D8H.3 SFRSYM    DATA     BIT       ERSTF
      000000E6H   SFRSYM    DATA     BYTE      PRESET0
      000000D4H   SFRSYM    DATA     BYTE      OCTRL
      000000A8H.7 SFRSYM    DATA     BIT       EA
      0000008FH   SFRSYM    DATA     BYTE      POREN
      000000C8H   SFRSYM    DATA     BYTE      PWM0CON
      000000E7H   SFRSYM    DATA     BYTE      PRESET1
      000000C9H   SFRSYM    DATA     BYTE      PWM1CON
      00000086H   SFRSYM    DATA     BYTE      BEEPCTR
      000000CAH   SFRSYM    DATA     BYTE      PWM2CON
      000000B8H.4 SFRSYM    DATA     BIT       LPTIMINTEN
      000000ABH   SFRSYM    DATA     BYTE      P0AH
      000000B0H   SFRSYM    DATA     BYTE      P1AH
      000000E8H   SFRSYM    DATA     BYTE      P2AH
      000000F8H.6 SFRSYM    DATA     BIT       RC32KF
      000000A8H   SFRSYM    DATA     BYTE      IEN0
      000000A7H   SFRSYM    DATA     BYTE      OPSET
      000000A4H   SFRSYM    DATA     BYTE      P0AL
LX51 LINKER/LOCATER V4.66.97.0                                                        06/12/2025  17:35:51  PAGE 16


      000000B8H   SFRSYM    DATA     BYTE      IEN1
      000000A8H.6 SFRSYM    DATA     BIT       EADC
      00000085H   SFRSYM    DATA     BYTE      DPH1
      000000AEH   SFRSYM    DATA     BYTE      P1AL
      0000009AH   SFRSYM    DATA     BYTE      IEN2
      000000C0H   SFRSYM    DATA     BYTE      P2AL
      000000B6H   SFRSYM    DATA     BYTE      ADCDR0
      000000F8H.5 SFRSYM    DATA     BIT       RC16MF
      000000B7H   SFRSYM    DATA     BYTE      ADCDR1
      00000084H   SFRSYM    DATA     BYTE      DPL1
      000000D6H   SFRSYM    DATA     BYTE      P0OD
      000000DBH   SFRSYM    DATA     BYTE      P1OD
      000000D5H   SFRSYM    DATA     BYTE      P0PD
      00000098H.4 SFRSYM    DATA     BIT       REN0
      000000ECH   SFRSYM    DATA     BYTE      P2OD
      000000DAH   SFRSYM    DATA     BYTE      P1PD
      000000E4H   SFRSYM    DATA     BYTE      P2PD
      000000D7H   SFRSYM    DATA     BYTE      P0CS
      00000097H   SFRSYM    DATA     BYTE      P0DR
      0000009EH   SFRSYM    DATA     BYTE      EUARTEN
      000000DCH   SFRSYM    DATA     BYTE      P1CS
      000000E5H   SFRSYM    DATA     BYTE      P1DR
      000000F4H   SFRSYM    DATA     BYTE      P2CS
      000000FCH   SFRSYM    DATA     BYTE      P2DR
      000000D0H.7 SFRSYM    DATA     BIT       CY
      000000D8H.0 SFRSYM    DATA     BIT       WDT0
      000000D8H.1 SFRSYM    DATA     BIT       WDT1
      000000D8H.2 SFRSYM    DATA     BIT       WDT2
      00000081H   SFRSYM    DATA     BYTE      SP
      000000F1H   SFRSYM    DATA     BYTE      P0PU
      000000F2H   SFRSYM    DATA     BYTE      P1PU
      000000D1H   SFRSYM    DATA     WORD      OADR
      000000F3H   SFRSYM    DATA     BYTE      P2PU
      00000093H   SFRSYM    DATA     BYTE      ADCIER
      000000A5H   SFRSYM    DATA     BYTE      OSEC
      000000D8H.6 SFRSYM    DATA     BIT       WDEN
      000000BAH   SFRSYM    DATA     BYTE      S0RELH
      00000080H.0 SFRSYM    DATA     BIT       P00
      000000D8H.7 SFRSYM    DATA     BIT       WDOF
      000000BBH   SFRSYM    DATA     BYTE      S1RELH
      00000090H.0 SFRSYM    DATA     BIT       P10
      00000080H.1 SFRSYM    DATA     BIT       P01
      00000087H   SFRSYM    DATA     BYTE      PCON
      000000C4H   SFRSYM    DATA     BYTE      PWM0DH
      000000A0H.0 SFRSYM    DATA     BIT       P20
      00000090H.1 SFRSYM    DATA     BIT       P11
      00000080H.2 SFRSYM    DATA     BIT       P02
      000000C6H   SFRSYM    DATA     BYTE      PWM1DH
      00000090H.2 SFRSYM    DATA     BIT       P12
      00000080H.3 SFRSYM    DATA     BIT       P03
      000000C7H   SFRSYM    DATA     BYTE      PWM2DH
      000000C8H.2 SFRSYM    DATA     BIT       PWM0IE
      000000AAH   SFRSYM    DATA     BYTE      S0RELL
      000000A0H.2 SFRSYM    DATA     BIT       P22
      00000090H.3 SFRSYM    DATA     BIT       P13
      00000080H.4 SFRSYM    DATA     BIT       P04
      000000C8H.1 SFRSYM    DATA     BIT       PWM0IF
      0000009DH   SFRSYM    DATA     BYTE      S1RELL
      000000A0H.3 SFRSYM    DATA     BIT       P23
      00000090H.4 SFRSYM    DATA     BIT       P14
      00000080H.5 SFRSYM    DATA     BIT       P05
      000000C3H   SFRSYM    DATA     BYTE      PWM0DL
      00000090H.5 SFRSYM    DATA     BIT       P15
      000000A6H   SFRSYM    DATA     BYTE      OSTATUS
      000000C5H   SFRSYM    DATA     BYTE      PWM1DL
LX51 LINKER/LOCATER V4.66.97.0                                                        06/12/2025  17:35:51  PAGE 17


      000000A0H.5 SFRSYM    DATA     BIT       P25
      000000D8H.4 SFRSYM    DATA     BIT       PORF
      000000D8H   SFRSYM    DATA     BYTE      RSTSTAT
      000000CFH   SFRSYM    DATA     BYTE      PWM2DL
      000000A0H.6 SFRSYM    DATA     BIT       P26
      000000C8H.7 SFRSYM    DATA     BIT       PWM0EN
      000000A0H.7 SFRSYM    DATA     BIT       P27
      000000A8H.5 SFRSYM    DATA     BIT       EPWM
      000000D8H.5 SFRSYM    DATA     BIT       LVRF
      000000F8H   SFRSYM    DATA     BYTE      CLKCON
      000000CCH   SFRSYM    DATA     BYTE      PWM0PH
      000000CEH   SFRSYM    DATA     BYTE      PWM1PH
      000000B8H.5 SFRSYM    DATA     BIT       I2CINTEN
      000000C2H   SFRSYM    DATA     BYTE      PWM2PH
      000000F0H   SFRSYM    DATA     BYTE      B
      000000EEH   SFRSYM    DATA     BYTE      RCHDIV
      000000CBH   SFRSYM    DATA     BYTE      PWM0PL
      000000CDH   SFRSYM    DATA     BYTE      PWM1PL
      000000C1H   SFRSYM    DATA     BYTE      PWM2PL
      000000F7H   SFRSYM    DATA     BYTE      ADCSPW
      000000F8H.1 SFRSYM    DATA     BIT       XCLKEN
      000000E0H   SFRSYM    DATA     BYTE      ACC
      000000DDH   SFRSYM    DATA     BYTE      LVDCON
      000000A8H.4 SFRSYM    DATA     BIT       ES0
      000000A9H   SFRSYM    DATA     BYTE      IP0
      000000A8H.1 SFRSYM    DATA     BIT       ET0
      000000A8H.2 SFRSYM    DATA     BIT       ES1
      000000F6H   SFRSYM    DATA     BYTE      ADCCSTAT
      000000B9H   SFRSYM    DATA     BYTE      IP1
      000000A8H.3 SFRSYM    DATA     BIT       ET1
      00000098H.0 SFRSYM    DATA     BIT       RI0
      000000C8H.0 SFRSYM    DATA     BIT       PWM0SS
      00000098H.1 SFRSYM    DATA     BIT       TI0
      000000A8H.0 SFRSYM    DATA     BIT       EX0
      000000D0H.0 SFRSYM    DATA     BIT       P
      000000B8H.3 SFRSYM    DATA     BIT       EFCINTEN
      000000A2H   SFRSYM    DATA     BYTE      OINTEN
      00000098H.7 SFRSYM    DATA     BIT       SM0
      00000098H.6 SFRSYM    DATA     BIT       SM1
      000000FEH   SFRSYM    DATA     BYTE      ADCCDR0
      000000FFH   SFRSYM    DATA     BYTE      ADCCDR1
      000000D0H.3 SFRSYM    DATA     BIT       RS0
      000000ACH   SFRSYM    DATA     BYTE      ADCGCR0
      000000D0H.4 SFRSYM    DATA     BIT       RS1
      000000ADH   SFRSYM    DATA     BYTE      ADCGCR1
      000000B4H   SFRSYM    DATA     BYTE      ADCGCR2
      000000B5H   SFRSYM    DATA     BYTE      ADCGCR3
      000000F8H.3 SFRSYM    DATA     BIT       RC32KEN
      000000DEH   SFRSYM    DATA     BYTE      PCLK0
      000000DFH   SFRSYM    DATA     BYTE      PCLK1
      00000083H   SFRSYM    DATA     BYTE      DPH
      000000E9H   SFRSYM    DATA     BYTE      P0IEN
      000000F5H   SFRSYM    DATA     BYTE      ADCHL
      000000F8H.2 SFRSYM    DATA     BIT       RC16MEN
      000000EAH   SFRSYM    DATA     BYTE      P1IEN
      000000EBH   SFRSYM    DATA     BYTE      P2IEN
      000000B6H   SFRSYM    DATA     WORD      ADCDR
      000000B3H   SFRSYM    DATA     BYTE      XTHCTR
      00000082H   SFRSYM    DATA     BYTE      DPL
      00000099H   SFRSYM    DATA     BYTE      S0BUF
      0000009CH   SFRSYM    DATA     BYTE      S1BUF
      000000F9H   SFRSYM    DATA     BYTE      P0OEN
      000000B8H.0 SFRSYM    DATA     BIT       GTIM0INTEN
      000000D9H   SFRSYM    DATA     BYTE      SYSDIV
      00000098H   SFRSYM    DATA     BYTE      S0CON
LX51 LINKER/LOCATER V4.66.97.0                                                        06/12/2025  17:35:51  PAGE 18


      000000FAH   SFRSYM    DATA     BYTE      P1OEN
      000000B8H.2 SFRSYM    DATA     BIT       GTIM1INTEN
      000000A3H   SFRSYM    DATA     BYTE      OINTUS
      000000BEH   SFRSYM    DATA     BYTE      RCHTRIMH
      000000F8H.0 SFRSYM    DATA     BIT       SYSSEL
      0000009BH   SFRSYM    DATA     BYTE      S1CON
      000000FBH   SFRSYM    DATA     BYTE      P2OEN
      000000B8H.6 SFRSYM    DATA     BIT       GTIM2INTEN
      000000BDH   SFRSYM    DATA     BYTE      LDOTRIMH
      00000092H   SFRSYM    DATA     BYTE      DPS
      0000009FH   SFRSYM    DATA     BYTE      RCLTRIMH
      000000BFH   SFRSYM    DATA     BYTE      RCHTRIML
      000000D3H   SFRSYM    DATA     BYTE      ODATA
      00000091H   SFRSYM    DATA     BYTE      LDOTRIML
      000000BCH   SFRSYM    DATA     BYTE      RCLTRIML
      000000E1H   SFRSYM    DATA     BYTE      P0IRQ
      000000B8H.1 SFRSYM    DATA     BIT       SPIINTEN
      000000E2H   SFRSYM    DATA     BYTE      P1IRQ
      000000E3H   SFRSYM    DATA     BYTE      P2IRQ
      000000D2H   SFRSYM    DATA     BYTE      OADRH
      000000B8H.7 SFRSYM    DATA     BIT       UART2INTEN
      000000F0H.0 SFRSYM    DATA     BIT       B0
      000000F0H.1 SFRSYM    DATA     BIT       B1
      000000F0H.2 SFRSYM    DATA     BIT       B2
      000000D1H   SFRSYM    DATA     BYTE      OADRL
      000000F0H.3 SFRSYM    DATA     BIT       B3
      000000F0H.4 SFRSYM    DATA     BIT       B4
      000000D0H.5 SFRSYM    DATA     BIT       F0
      000000F0H.5 SFRSYM    DATA     BIT       B5
      000000D0H.1 SFRSYM    DATA     BIT       F1
      000000AFH   SFRSYM    DATA     BYTE      REMAP
      000000F0H.6 SFRSYM    DATA     BIT       B6
      000000E0H.0 SFRSYM    DATA     BIT       ACC0
      000000A1H   SFRSYM    DATA     BYTE      OUS
      000000C8H.6 SFRSYM    DATA     BIT       PWM0S
      000000F0H.7 SFRSYM    DATA     BIT       B7
      000000E0H.1 SFRSYM    DATA     BIT       ACC1
      000000F8H.4 SFRSYM    DATA     BIT       XCLKF
      000000E0H.2 SFRSYM    DATA     BIT       ACC2
      0000008EH   SFRSYM    DATA     BYTE      PDSEL
      000000E0H.3 SFRSYM    DATA     BIT       ACC3
      000000D0H   SFRSYM    DATA     BYTE      PSW
      000000E0H.4 SFRSYM    DATA     BIT       ACC4
      00000098H.2 SFRSYM    DATA     BIT       RB80
      000000E0H.5 SFRSYM    DATA     BIT       ACC5
      000000FDH   SFRSYM    DATA     BYTE      ADCVREF
      000000E0H.6 SFRSYM    DATA     BIT       ACC6

      01001130H   BLOCK     CODE     ---       LVL=0
      0200025FH   SYMBOL    XDATA    DWORD     system_clk_hz
      01001136H   BLOCK     CODE     NEAR LAB  LVL=1
      02000263H   SYMBOL    XDATA    DWORD     crystal_clk
      ---         BLOCKEND  ---      ---       LVL=1
      01001130H   LINE      CODE     ---       #26
      01001136H   LINE      CODE     ---       #27
      01001136H   LINE      CODE     ---       #28
      01001140H   LINE      CODE     ---       #29
      01001143H   LINE      CODE     ---       #30
      0100114BH   LINE      CODE     ---       #33
      010011B3H   LINE      CODE     ---       #38
      010011DBH   LINE      CODE     ---       #39
      010011DBH   LINE      CODE     ---       #40
      010011DBH   LINE      CODE     ---       #41
      010011DDH   LINE      CODE     ---       #42
      010011EFH   LINE      CODE     ---       #43
LX51 LINKER/LOCATER V4.66.97.0                                                        06/12/2025  17:35:51  PAGE 19


      010011EFH   LINE      CODE     ---       #44
      010011F9H   LINE      CODE     ---       #45
      010011FBH   LINE      CODE     ---       #47
      010011FBH   LINE      CODE     ---       #48
      01001210H   LINE      CODE     ---       #49
      01001210H   LINE      CODE     ---       #50
      0100122FH   LINE      CODE     ---       #51
      0100122FH   LINE      CODE     ---       #52
      0100122FH   LINE      CODE     ---       #53
      01001232H   LINE      CODE     ---       #54
      01001235H   LINE      CODE     ---       #55
      01001237H   LINE      CODE     ---       #56
      01001237H   LINE      CODE     ---       #57
      0100123AH   LINE      CODE     ---       #58
      0100123DH   LINE      CODE     ---       #59
      0100123FH   LINE      CODE     ---       #60
      0100123FH   LINE      CODE     ---       #61
      01001242H   LINE      CODE     ---       #62
      01001245H   LINE      CODE     ---       #63
      01001245H   LINE      CODE     ---       #64
      01001257H   LINE      CODE     ---       #67
      01001257H   LINE      CODE     ---       #69
      01001257H   LINE      CODE     ---       #71
      0100125AH   LINE      CODE     ---       #72
      0100125DH   LINE      CODE     ---       #73
      ---         BLOCKEND  ---      ---       LVL=0

      01001EEFH   BLOCK     CODE     ---       LVL=0
      01001EEFH   LINE      CODE     ---       #82
      01001EEFH   LINE      CODE     ---       #83
      01001EEFH   LINE      CODE     ---       #84
      ---         BLOCKEND  ---      ---       LVL=0

      ---         MODULE    ---      ---       COMMON
      01001C70H   PUBLIC    CODE     ---       _delay_ms
      00000098H.3 SFRSYM    DATA     BIT       TB80
      000000E0H.7 SFRSYM    DATA     BIT       ACC7
      00000080H   SFRSYM    DATA     BYTE      P0
      00000090H   SFRSYM    DATA     BYTE      P1
      000000A0H   SFRSYM    DATA     BYTE      P2
      00000098H.5 SFRSYM    DATA     BIT       SM20
      000000B2H   SFRSYM    DATA     BYTE      ESTCR
      000000B1H   SFRSYM    DATA     BYTE      CLKST
      000000D0H.6 SFRSYM    DATA     BIT       AC
      000000D8H.3 SFRSYM    DATA     BIT       ERSTF
      000000E6H   SFRSYM    DATA     BYTE      PRESET0
      000000D4H   SFRSYM    DATA     BYTE      OCTRL
      000000A8H.7 SFRSYM    DATA     BIT       EA
      0000008FH   SFRSYM    DATA     BYTE      POREN
      000000C8H   SFRSYM    DATA     BYTE      PWM0CON
      000000E7H   SFRSYM    DATA     BYTE      PRESET1
      000000C9H   SFRSYM    DATA     BYTE      PWM1CON
      00000086H   SFRSYM    DATA     BYTE      BEEPCTR
      000000CAH   SFRSYM    DATA     BYTE      PWM2CON
      000000B8H.4 SFRSYM    DATA     BIT       LPTIMINTEN
      000000ABH   SFRSYM    DATA     BYTE      P0AH
      000000B0H   SFRSYM    DATA     BYTE      P1AH
      000000E8H   SFRSYM    DATA     BYTE      P2AH
      000000F8H.6 SFRSYM    DATA     BIT       RC32KF
      000000A8H   SFRSYM    DATA     BYTE      IEN0
      000000A7H   SFRSYM    DATA     BYTE      OPSET
      000000A4H   SFRSYM    DATA     BYTE      P0AL
      000000B8H   SFRSYM    DATA     BYTE      IEN1
      000000A8H.6 SFRSYM    DATA     BIT       EADC
      00000085H   SFRSYM    DATA     BYTE      DPH1
LX51 LINKER/LOCATER V4.66.97.0                                                        06/12/2025  17:35:51  PAGE 20


      000000AEH   SFRSYM    DATA     BYTE      P1AL
      0000009AH   SFRSYM    DATA     BYTE      IEN2
      000000C0H   SFRSYM    DATA     BYTE      P2AL
      000000B6H   SFRSYM    DATA     BYTE      ADCDR0
      000000F8H.5 SFRSYM    DATA     BIT       RC16MF
      000000B7H   SFRSYM    DATA     BYTE      ADCDR1
      00000084H   SFRSYM    DATA     BYTE      DPL1
      000000D6H   SFRSYM    DATA     BYTE      P0OD
      000000DBH   SFRSYM    DATA     BYTE      P1OD
      000000D5H   SFRSYM    DATA     BYTE      P0PD
      00000098H.4 SFRSYM    DATA     BIT       REN0
      000000ECH   SFRSYM    DATA     BYTE      P2OD
      000000DAH   SFRSYM    DATA     BYTE      P1PD
      000000E4H   SFRSYM    DATA     BYTE      P2PD
      000000D7H   SFRSYM    DATA     BYTE      P0CS
      00000097H   SFRSYM    DATA     BYTE      P0DR
      0000009EH   SFRSYM    DATA     BYTE      EUARTEN
      000000DCH   SFRSYM    DATA     BYTE      P1CS
      000000E5H   SFRSYM    DATA     BYTE      P1DR
      000000F4H   SFRSYM    DATA     BYTE      P2CS
      000000FCH   SFRSYM    DATA     BYTE      P2DR
      000000D0H.7 SFRSYM    DATA     BIT       CY
      000000D8H.0 SFRSYM    DATA     BIT       WDT0
      000000D8H.1 SFRSYM    DATA     BIT       WDT1
      000000D8H.2 SFRSYM    DATA     BIT       WDT2
      00000081H   SFRSYM    DATA     BYTE      SP
      000000F1H   SFRSYM    DATA     BYTE      P0PU
      000000F2H   SFRSYM    DATA     BYTE      P1PU
      000000D1H   SFRSYM    DATA     WORD      OADR
      000000F3H   SFRSYM    DATA     BYTE      P2PU
      00000093H   SFRSYM    DATA     BYTE      ADCIER
      000000A5H   SFRSYM    DATA     BYTE      OSEC
      000000D8H.6 SFRSYM    DATA     BIT       WDEN
      000000BAH   SFRSYM    DATA     BYTE      S0RELH
      00000080H.0 SFRSYM    DATA     BIT       P00
      000000D8H.7 SFRSYM    DATA     BIT       WDOF
      000000BBH   SFRSYM    DATA     BYTE      S1RELH
      00000090H.0 SFRSYM    DATA     BIT       P10
      00000080H.1 SFRSYM    DATA     BIT       P01
      00000087H   SFRSYM    DATA     BYTE      PCON
      000000C4H   SFRSYM    DATA     BYTE      PWM0DH
      000000A0H.0 SFRSYM    DATA     BIT       P20
      00000090H.1 SFRSYM    DATA     BIT       P11
      00000080H.2 SFRSYM    DATA     BIT       P02
      000000C6H   SFRSYM    DATA     BYTE      PWM1DH
      00000090H.2 SFRSYM    DATA     BIT       P12
      00000080H.3 SFRSYM    DATA     BIT       P03
      000000C7H   SFRSYM    DATA     BYTE      PWM2DH
      000000C8H.2 SFRSYM    DATA     BIT       PWM0IE
      000000AAH   SFRSYM    DATA     BYTE      S0RELL
      000000A0H.2 SFRSYM    DATA     BIT       P22
      00000090H.3 SFRSYM    DATA     BIT       P13
      00000080H.4 SFRSYM    DATA     BIT       P04
      000000C8H.1 SFRSYM    DATA     BIT       PWM0IF
      0000009DH   SFRSYM    DATA     BYTE      S1RELL
      000000A0H.3 SFRSYM    DATA     BIT       P23
      00000090H.4 SFRSYM    DATA     BIT       P14
      00000080H.5 SFRSYM    DATA     BIT       P05
      000000C3H   SFRSYM    DATA     BYTE      PWM0DL
      00000090H.5 SFRSYM    DATA     BIT       P15
      000000A6H   SFRSYM    DATA     BYTE      OSTATUS
      000000C5H   SFRSYM    DATA     BYTE      PWM1DL
      000000A0H.5 SFRSYM    DATA     BIT       P25
      000000D8H.4 SFRSYM    DATA     BIT       PORF
      000000D8H   SFRSYM    DATA     BYTE      RSTSTAT
LX51 LINKER/LOCATER V4.66.97.0                                                        06/12/2025  17:35:51  PAGE 21


      000000CFH   SFRSYM    DATA     BYTE      PWM2DL
      000000A0H.6 SFRSYM    DATA     BIT       P26
      000000C8H.7 SFRSYM    DATA     BIT       PWM0EN
      000000A0H.7 SFRSYM    DATA     BIT       P27
      000000A8H.5 SFRSYM    DATA     BIT       EPWM
      000000D8H.5 SFRSYM    DATA     BIT       LVRF
      000000F8H   SFRSYM    DATA     BYTE      CLKCON
      000000CCH   SFRSYM    DATA     BYTE      PWM0PH
      000000CEH   SFRSYM    DATA     BYTE      PWM1PH
      000000B8H.5 SFRSYM    DATA     BIT       I2CINTEN
      000000C2H   SFRSYM    DATA     BYTE      PWM2PH
      000000F0H   SFRSYM    DATA     BYTE      B
      000000EEH   SFRSYM    DATA     BYTE      RCHDIV
      000000CBH   SFRSYM    DATA     BYTE      PWM0PL
      000000CDH   SFRSYM    DATA     BYTE      PWM1PL
      000000C1H   SFRSYM    DATA     BYTE      PWM2PL
      000000F7H   SFRSYM    DATA     BYTE      ADCSPW
      000000F8H.1 SFRSYM    DATA     BIT       XCLKEN
      000000E0H   SFRSYM    DATA     BYTE      ACC
      000000DDH   SFRSYM    DATA     BYTE      LVDCON
      000000A8H.4 SFRSYM    DATA     BIT       ES0
      000000A9H   SFRSYM    DATA     BYTE      IP0
      000000A8H.1 SFRSYM    DATA     BIT       ET0
      000000A8H.2 SFRSYM    DATA     BIT       ES1
      000000F6H   SFRSYM    DATA     BYTE      ADCCSTAT
      000000B9H   SFRSYM    DATA     BYTE      IP1
      000000A8H.3 SFRSYM    DATA     BIT       ET1
      00000098H.0 SFRSYM    DATA     BIT       RI0
      000000C8H.0 SFRSYM    DATA     BIT       PWM0SS
      00000098H.1 SFRSYM    DATA     BIT       TI0
      000000A8H.0 SFRSYM    DATA     BIT       EX0
      000000D0H.0 SFRSYM    DATA     BIT       P
      000000B8H.3 SFRSYM    DATA     BIT       EFCINTEN
      000000A2H   SFRSYM    DATA     BYTE      OINTEN
      00000098H.7 SFRSYM    DATA     BIT       SM0
      00000098H.6 SFRSYM    DATA     BIT       SM1
      000000FEH   SFRSYM    DATA     BYTE      ADCCDR0
      000000FFH   SFRSYM    DATA     BYTE      ADCCDR1
      000000D0H.3 SFRSYM    DATA     BIT       RS0
      000000ACH   SFRSYM    DATA     BYTE      ADCGCR0
      000000D0H.4 SFRSYM    DATA     BIT       RS1
      000000ADH   SFRSYM    DATA     BYTE      ADCGCR1
      000000B4H   SFRSYM    DATA     BYTE      ADCGCR2
      000000B5H   SFRSYM    DATA     BYTE      ADCGCR3
      000000F8H.3 SFRSYM    DATA     BIT       RC32KEN
      000000DEH   SFRSYM    DATA     BYTE      PCLK0
      000000DFH   SFRSYM    DATA     BYTE      PCLK1
      00000083H   SFRSYM    DATA     BYTE      DPH
      000000E9H   SFRSYM    DATA     BYTE      P0IEN
      000000F5H   SFRSYM    DATA     BYTE      ADCHL
      000000F8H.2 SFRSYM    DATA     BIT       RC16MEN
      000000EAH   SFRSYM    DATA     BYTE      P1IEN
      000000EBH   SFRSYM    DATA     BYTE      P2IEN
      000000B6H   SFRSYM    DATA     WORD      ADCDR
      000000B3H   SFRSYM    DATA     BYTE      XTHCTR
      00000082H   SFRSYM    DATA     BYTE      DPL
      00000099H   SFRSYM    DATA     BYTE      S0BUF
      0000009CH   SFRSYM    DATA     BYTE      S1BUF
      000000F9H   SFRSYM    DATA     BYTE      P0OEN
      000000B8H.0 SFRSYM    DATA     BIT       GTIM0INTEN
      000000D9H   SFRSYM    DATA     BYTE      SYSDIV
      00000098H   SFRSYM    DATA     BYTE      S0CON
      000000FAH   SFRSYM    DATA     BYTE      P1OEN
      000000B8H.2 SFRSYM    DATA     BIT       GTIM1INTEN
      000000A3H   SFRSYM    DATA     BYTE      OINTUS
LX51 LINKER/LOCATER V4.66.97.0                                                        06/12/2025  17:35:51  PAGE 22


      000000BEH   SFRSYM    DATA     BYTE      RCHTRIMH
      000000F8H.0 SFRSYM    DATA     BIT       SYSSEL
      0000009BH   SFRSYM    DATA     BYTE      S1CON
      000000FBH   SFRSYM    DATA     BYTE      P2OEN
      000000B8H.6 SFRSYM    DATA     BIT       GTIM2INTEN
      000000BDH   SFRSYM    DATA     BYTE      LDOTRIMH
      00000092H   SFRSYM    DATA     BYTE      DPS
      0000009FH   SFRSYM    DATA     BYTE      RCLTRIMH
      000000BFH   SFRSYM    DATA     BYTE      RCHTRIML
      000000D3H   SFRSYM    DATA     BYTE      ODATA
      00000091H   SFRSYM    DATA     BYTE      LDOTRIML
      000000BCH   SFRSYM    DATA     BYTE      RCLTRIML
      000000E1H   SFRSYM    DATA     BYTE      P0IRQ
      000000B8H.1 SFRSYM    DATA     BIT       SPIINTEN
      000000E2H   SFRSYM    DATA     BYTE      P1IRQ
      000000E3H   SFRSYM    DATA     BYTE      P2IRQ
      000000D2H   SFRSYM    DATA     BYTE      OADRH
      000000B8H.7 SFRSYM    DATA     BIT       UART2INTEN
      000000F0H.0 SFRSYM    DATA     BIT       B0
      000000F0H.1 SFRSYM    DATA     BIT       B1
      000000F0H.2 SFRSYM    DATA     BIT       B2
      000000D1H   SFRSYM    DATA     BYTE      OADRL
      000000F0H.3 SFRSYM    DATA     BIT       B3
      000000F0H.4 SFRSYM    DATA     BIT       B4
      000000D0H.5 SFRSYM    DATA     BIT       F0
      000000F0H.5 SFRSYM    DATA     BIT       B5
      000000D0H.1 SFRSYM    DATA     BIT       F1
      000000AFH   SFRSYM    DATA     BYTE      REMAP
      000000F0H.6 SFRSYM    DATA     BIT       B6
      000000E0H.0 SFRSYM    DATA     BIT       ACC0
      000000A1H   SFRSYM    DATA     BYTE      OUS
      000000C8H.6 SFRSYM    DATA     BIT       PWM0S
      000000F0H.7 SFRSYM    DATA     BIT       B7
      000000E0H.1 SFRSYM    DATA     BIT       ACC1
      000000F8H.4 SFRSYM    DATA     BIT       XCLKF
      000000E0H.2 SFRSYM    DATA     BIT       ACC2
      0000008EH   SFRSYM    DATA     BYTE      PDSEL
      000000E0H.3 SFRSYM    DATA     BIT       ACC3
      000000D0H   SFRSYM    DATA     BYTE      PSW
      000000E0H.4 SFRSYM    DATA     BIT       ACC4
      00000098H.2 SFRSYM    DATA     BIT       RB80
      000000E0H.5 SFRSYM    DATA     BIT       ACC5
      000000FDH   SFRSYM    DATA     BYTE      ADCVREF
      000000E0H.6 SFRSYM    DATA     BIT       ACC6

      01001C70H   BLOCK     CODE     ---       LVL=0
      02000261H   SYMBOL    XDATA    DWORD     n
      01001C76H   BLOCK     CODE     NEAR LAB  LVL=1
      02000265H   SYMBOL    XDATA    DWORD     x
      00000007H   SYMBOL    DATA     BYTE      i
      00000006H   SYMBOL    DATA     BYTE      j
      ---         BLOCKEND  ---      ---       LVL=1
      01001C70H   LINE      CODE     ---       #20
      01001C76H   LINE      CODE     ---       #21
      01001C76H   LINE      CODE     ---       #25
      01001C92H   LINE      CODE     ---       #26
      01001C92H   LINE      CODE     ---       #27
      01001C93H   LINE      CODE     ---       #28
      01001C95H   LINE      CODE     ---       #29
      01001C97H   LINE      CODE     ---       #31
      01001C97H   LINE      CODE     ---       #32
      01001C99H   LINE      CODE     ---       #33
      01001C9BH   LINE      CODE     ---       #34
      01001CB6H   LINE      CODE     ---       #35
      ---         BLOCKEND  ---      ---       LVL=0
LX51 LINKER/LOCATER V4.66.97.0                                                        06/12/2025  17:35:51  PAGE 23



      ---         MODULE    ---      ---       UART0
      0200032EH   PUBLIC    XDATA    ---       uart0_func
      0200032DH   PUBLIC    XDATA    BYTE      tx_flag
      01001F1DH   PUBLIC    CODE     ---       _putchar
      01000006H   PUBLIC    CODE     ---       _uart0_send_byte
      01000026H   PUBLIC    CODE     ---       _uart0_init
      01001C26H   PUBLIC    CODE     ---       UART0_IRQHandler
      00000098H.3 SFRSYM    DATA     BIT       TB80
      000000E0H.7 SFRSYM    DATA     BIT       ACC7
      00000080H   SFRSYM    DATA     BYTE      P0
      00000090H   SFRSYM    DATA     BYTE      P1
      000000A0H   SFRSYM    DATA     BYTE      P2
      00000098H.5 SFRSYM    DATA     BIT       SM20
      000000B2H   SFRSYM    DATA     BYTE      ESTCR
      000000B1H   SFRSYM    DATA     BYTE      CLKST
      000000D0H.6 SFRSYM    DATA     BIT       AC
      000000D8H.3 SFRSYM    DATA     BIT       ERSTF
      000000E6H   SFRSYM    DATA     BYTE      PRESET0
      000000D4H   SFRSYM    DATA     BYTE      OCTRL
      000000A8H.7 SFRSYM    DATA     BIT       EA
      0000008FH   SFRSYM    DATA     BYTE      POREN
      000000C8H   SFRSYM    DATA     BYTE      PWM0CON
      000000E7H   SFRSYM    DATA     BYTE      PRESET1
      000000C9H   SFRSYM    DATA     BYTE      PWM1CON
      00000086H   SFRSYM    DATA     BYTE      BEEPCTR
      000000CAH   SFRSYM    DATA     BYTE      PWM2CON
      000000B8H.4 SFRSYM    DATA     BIT       LPTIMINTEN
      000000ABH   SFRSYM    DATA     BYTE      P0AH
      000000B0H   SFRSYM    DATA     BYTE      P1AH
      000000E8H   SFRSYM    DATA     BYTE      P2AH
      000000F8H.6 SFRSYM    DATA     BIT       RC32KF
      000000A8H   SFRSYM    DATA     BYTE      IEN0
      000000A7H   SFRSYM    DATA     BYTE      OPSET
      000000A4H   SFRSYM    DATA     BYTE      P0AL
      000000B8H   SFRSYM    DATA     BYTE      IEN1
      000000A8H.6 SFRSYM    DATA     BIT       EADC
      00000085H   SFRSYM    DATA     BYTE      DPH1
      000000AEH   SFRSYM    DATA     BYTE      P1AL
      0000009AH   SFRSYM    DATA     BYTE      IEN2
      000000C0H   SFRSYM    DATA     BYTE      P2AL
      000000B6H   SFRSYM    DATA     BYTE      ADCDR0
      000000F8H.5 SFRSYM    DATA     BIT       RC16MF
      000000B7H   SFRSYM    DATA     BYTE      ADCDR1
      00000084H   SFRSYM    DATA     BYTE      DPL1
      000000D6H   SFRSYM    DATA     BYTE      P0OD
      000000DBH   SFRSYM    DATA     BYTE      P1OD
      000000D5H   SFRSYM    DATA     BYTE      P0PD
      00000098H.4 SFRSYM    DATA     BIT       REN0
      000000ECH   SFRSYM    DATA     BYTE      P2OD
      000000DAH   SFRSYM    DATA     BYTE      P1PD
      000000E4H   SFRSYM    DATA     BYTE      P2PD
      000000D7H   SFRSYM    DATA     BYTE      P0CS
      00000097H   SFRSYM    DATA     BYTE      P0DR
      0000009EH   SFRSYM    DATA     BYTE      EUARTEN
      000000DCH   SFRSYM    DATA     BYTE      P1CS
      000000E5H   SFRSYM    DATA     BYTE      P1DR
      000000F4H   SFRSYM    DATA     BYTE      P2CS
      000000FCH   SFRSYM    DATA     BYTE      P2DR
      000000D0H.7 SFRSYM    DATA     BIT       CY
      000000D8H.0 SFRSYM    DATA     BIT       WDT0
      000000D8H.1 SFRSYM    DATA     BIT       WDT1
      000000D8H.2 SFRSYM    DATA     BIT       WDT2
      00000081H   SFRSYM    DATA     BYTE      SP
      000000F1H   SFRSYM    DATA     BYTE      P0PU
LX51 LINKER/LOCATER V4.66.97.0                                                        06/12/2025  17:35:51  PAGE 24


      000000F2H   SFRSYM    DATA     BYTE      P1PU
      000000D1H   SFRSYM    DATA     WORD      OADR
      000000F3H   SFRSYM    DATA     BYTE      P2PU
      00000093H   SFRSYM    DATA     BYTE      ADCIER
      000000A5H   SFRSYM    DATA     BYTE      OSEC
      000000D8H.6 SFRSYM    DATA     BIT       WDEN
      000000BAH   SFRSYM    DATA     BYTE      S0RELH
      00000080H.0 SFRSYM    DATA     BIT       P00
      000000D8H.7 SFRSYM    DATA     BIT       WDOF
      000000BBH   SFRSYM    DATA     BYTE      S1RELH
      00000090H.0 SFRSYM    DATA     BIT       P10
      00000080H.1 SFRSYM    DATA     BIT       P01
      00000087H   SFRSYM    DATA     BYTE      PCON
      000000C4H   SFRSYM    DATA     BYTE      PWM0DH
      000000A0H.0 SFRSYM    DATA     BIT       P20
      00000090H.1 SFRSYM    DATA     BIT       P11
      00000080H.2 SFRSYM    DATA     BIT       P02
      000000C6H   SFRSYM    DATA     BYTE      PWM1DH
      00000090H.2 SFRSYM    DATA     BIT       P12
      00000080H.3 SFRSYM    DATA     BIT       P03
      000000C7H   SFRSYM    DATA     BYTE      PWM2DH
      000000C8H.2 SFRSYM    DATA     BIT       PWM0IE
      000000AAH   SFRSYM    DATA     BYTE      S0RELL
      000000A0H.2 SFRSYM    DATA     BIT       P22
      00000090H.3 SFRSYM    DATA     BIT       P13
      00000080H.4 SFRSYM    DATA     BIT       P04
      000000C8H.1 SFRSYM    DATA     BIT       PWM0IF
      0000009DH   SFRSYM    DATA     BYTE      S1RELL
      000000A0H.3 SFRSYM    DATA     BIT       P23
      00000090H.4 SFRSYM    DATA     BIT       P14
      00000080H.5 SFRSYM    DATA     BIT       P05
      000000C3H   SFRSYM    DATA     BYTE      PWM0DL
      00000090H.5 SFRSYM    DATA     BIT       P15
      000000A6H   SFRSYM    DATA     BYTE      OSTATUS
      000000C5H   SFRSYM    DATA     BYTE      PWM1DL
      000000A0H.5 SFRSYM    DATA     BIT       P25
      000000D8H.4 SFRSYM    DATA     BIT       PORF
      000000D8H   SFRSYM    DATA     BYTE      RSTSTAT
      000000CFH   SFRSYM    DATA     BYTE      PWM2DL
      000000A0H.6 SFRSYM    DATA     BIT       P26
      000000C8H.7 SFRSYM    DATA     BIT       PWM0EN
      000000A0H.7 SFRSYM    DATA     BIT       P27
      000000A8H.5 SFRSYM    DATA     BIT       EPWM
      000000D8H.5 SFRSYM    DATA     BIT       LVRF
      000000F8H   SFRSYM    DATA     BYTE      CLKCON
      000000CCH   SFRSYM    DATA     BYTE      PWM0PH
      000000CEH   SFRSYM    DATA     BYTE      PWM1PH
      000000B8H.5 SFRSYM    DATA     BIT       I2CINTEN
      000000C2H   SFRSYM    DATA     BYTE      PWM2PH
      000000F0H   SFRSYM    DATA     BYTE      B
      000000EEH   SFRSYM    DATA     BYTE      RCHDIV
      000000CBH   SFRSYM    DATA     BYTE      PWM0PL
      000000CDH   SFRSYM    DATA     BYTE      PWM1PL
      000000C1H   SFRSYM    DATA     BYTE      PWM2PL
      000000F7H   SFRSYM    DATA     BYTE      ADCSPW
      000000F8H.1 SFRSYM    DATA     BIT       XCLKEN
      000000E0H   SFRSYM    DATA     BYTE      ACC
      000000DDH   SFRSYM    DATA     BYTE      LVDCON
      000000A8H.4 SFRSYM    DATA     BIT       ES0
      000000A9H   SFRSYM    DATA     BYTE      IP0
      000000A8H.1 SFRSYM    DATA     BIT       ET0
      000000A8H.2 SFRSYM    DATA     BIT       ES1
      000000F6H   SFRSYM    DATA     BYTE      ADCCSTAT
      000000B9H   SFRSYM    DATA     BYTE      IP1
      000000A8H.3 SFRSYM    DATA     BIT       ET1
LX51 LINKER/LOCATER V4.66.97.0                                                        06/12/2025  17:35:51  PAGE 25


      00000098H.0 SFRSYM    DATA     BIT       RI0
      000000C8H.0 SFRSYM    DATA     BIT       PWM0SS
      00000098H.1 SFRSYM    DATA     BIT       TI0
      000000A8H.0 SFRSYM    DATA     BIT       EX0
      000000D0H.0 SFRSYM    DATA     BIT       P
      000000B8H.3 SFRSYM    DATA     BIT       EFCINTEN
      000000A2H   SFRSYM    DATA     BYTE      OINTEN
      00000098H.7 SFRSYM    DATA     BIT       SM0
      00000098H.6 SFRSYM    DATA     BIT       SM1
      000000FEH   SFRSYM    DATA     BYTE      ADCCDR0
      000000FFH   SFRSYM    DATA     BYTE      ADCCDR1
      000000D0H.3 SFRSYM    DATA     BIT       RS0
      000000ACH   SFRSYM    DATA     BYTE      ADCGCR0
      000000D0H.4 SFRSYM    DATA     BIT       RS1
      000000ADH   SFRSYM    DATA     BYTE      ADCGCR1
      000000B4H   SFRSYM    DATA     BYTE      ADCGCR2
      000000B5H   SFRSYM    DATA     BYTE      ADCGCR3
      000000F8H.3 SFRSYM    DATA     BIT       RC32KEN
      000000DEH   SFRSYM    DATA     BYTE      PCLK0
      000000DFH   SFRSYM    DATA     BYTE      PCLK1
      00000083H   SFRSYM    DATA     BYTE      DPH
      000000E9H   SFRSYM    DATA     BYTE      P0IEN
      000000F5H   SFRSYM    DATA     BYTE      ADCHL
      000000F8H.2 SFRSYM    DATA     BIT       RC16MEN
      000000EAH   SFRSYM    DATA     BYTE      P1IEN
      000000EBH   SFRSYM    DATA     BYTE      P2IEN
      000000B6H   SFRSYM    DATA     WORD      ADCDR
      000000B3H   SFRSYM    DATA     BYTE      XTHCTR
      00000082H   SFRSYM    DATA     BYTE      DPL
      00000099H   SFRSYM    DATA     BYTE      S0BUF
      0000009CH   SFRSYM    DATA     BYTE      S1BUF
      000000F9H   SFRSYM    DATA     BYTE      P0OEN
      000000B8H.0 SFRSYM    DATA     BIT       GTIM0INTEN
      000000D9H   SFRSYM    DATA     BYTE      SYSDIV
      00000098H   SFRSYM    DATA     BYTE      S0CON
      000000FAH   SFRSYM    DATA     BYTE      P1OEN
      000000B8H.2 SFRSYM    DATA     BIT       GTIM1INTEN
      000000A3H   SFRSYM    DATA     BYTE      OINTUS
      000000BEH   SFRSYM    DATA     BYTE      RCHTRIMH
      000000F8H.0 SFRSYM    DATA     BIT       SYSSEL
      0000009BH   SFRSYM    DATA     BYTE      S1CON
      000000FBH   SFRSYM    DATA     BYTE      P2OEN
      000000B8H.6 SFRSYM    DATA     BIT       GTIM2INTEN
      000000BDH   SFRSYM    DATA     BYTE      LDOTRIMH
      00000092H   SFRSYM    DATA     BYTE      DPS
      0000009FH   SFRSYM    DATA     BYTE      RCLTRIMH
      000000BFH   SFRSYM    DATA     BYTE      RCHTRIML
      000000D3H   SFRSYM    DATA     BYTE      ODATA
      00000091H   SFRSYM    DATA     BYTE      LDOTRIML
      000000BCH   SFRSYM    DATA     BYTE      RCLTRIML
      000000E1H   SFRSYM    DATA     BYTE      P0IRQ
      000000B8H.1 SFRSYM    DATA     BIT       SPIINTEN
      000000E2H   SFRSYM    DATA     BYTE      P1IRQ
      000000E3H   SFRSYM    DATA     BYTE      P2IRQ
      000000D2H   SFRSYM    DATA     BYTE      OADRH
      000000B8H.7 SFRSYM    DATA     BIT       UART2INTEN
      000000F0H.0 SFRSYM    DATA     BIT       B0
      000000F0H.1 SFRSYM    DATA     BIT       B1
      000000F0H.2 SFRSYM    DATA     BIT       B2
      000000D1H   SFRSYM    DATA     BYTE      OADRL
      000000F0H.3 SFRSYM    DATA     BIT       B3
      000000F0H.4 SFRSYM    DATA     BIT       B4
      000000D0H.5 SFRSYM    DATA     BIT       F0
      000000F0H.5 SFRSYM    DATA     BIT       B5
      000000D0H.1 SFRSYM    DATA     BIT       F1
LX51 LINKER/LOCATER V4.66.97.0                                                        06/12/2025  17:35:51  PAGE 26


      000000AFH   SFRSYM    DATA     BYTE      REMAP
      000000F0H.6 SFRSYM    DATA     BIT       B6
      000000E0H.0 SFRSYM    DATA     BIT       ACC0
      000000A1H   SFRSYM    DATA     BYTE      OUS
      000000C8H.6 SFRSYM    DATA     BIT       PWM0S
      000000F0H.7 SFRSYM    DATA     BIT       B7
      000000E0H.1 SFRSYM    DATA     BIT       ACC1
      000000F8H.4 SFRSYM    DATA     BIT       XCLKF
      000000E0H.2 SFRSYM    DATA     BIT       ACC2
      0000008EH   SFRSYM    DATA     BYTE      PDSEL
      000000E0H.3 SFRSYM    DATA     BIT       ACC3
      000000D0H   SFRSYM    DATA     BYTE      PSW
      000000E0H.4 SFRSYM    DATA     BIT       ACC4
      00000098H.2 SFRSYM    DATA     BIT       RB80
      000000E0H.5 SFRSYM    DATA     BIT       ACC5
      000000FDH   SFRSYM    DATA     BYTE      ADCVREF
      000000E0H.6 SFRSYM    DATA     BIT       ACC6
      010019D7H   SYMBOL    CODE     ---       _uart0_set_baud_rate

      01001C26H   BLOCK     CODE     ---       LVL=0
      01001C26H   LINE      CODE     ---       #24
      01001C43H   LINE      CODE     ---       #26
      01001C46H   LINE      CODE     ---       #27
      01001C46H   LINE      CODE     ---       #28
      01001C50H   LINE      CODE     ---       #29
      01001C50H   LINE      CODE     ---       #30
      01001C53H   LINE      CODE     ---       #31
      01001C53H   LINE      CODE     ---       #32
      01001C55H   LINE      CODE     ---       #33
      01001C55H   LINE      CODE     ---       #42
      ---         BLOCKEND  ---      ---       LVL=0

      010019D7H   BLOCK     CODE     ---       LVL=0
      02000263H   SYMBOL    XDATA    DWORD     clk_hz
      02000267H   SYMBOL    XDATA    DWORD     baud_rate
      010019DDH   BLOCK     CODE     NEAR LAB  LVL=1
      0200026BH   SYMBOL    XDATA    DWORD     temp
      00000003H   SYMBOL    DATA     BYTE      MSbyte
      00000007H   SYMBOL    DATA     BYTE      LSbyte
      ---         BLOCKEND  ---      ---       LVL=1
      010019D7H   LINE      CODE     ---       #52
      010019DDH   LINE      CODE     ---       #53
      010019DDH   LINE      CODE     ---       #57
      010019F2H   LINE      CODE     ---       #58
      01001A19H   LINE      CODE     ---       #59
      01001A33H   LINE      CODE     ---       #61
      01001A40H   LINE      CODE     ---       #62
      01001A46H   LINE      CODE     ---       #64
      01001A4BH   LINE      CODE     ---       #65
      01001A4DH   LINE      CODE     ---       #66
      ---         BLOCKEND  ---      ---       LVL=0

      01000026H   BLOCK     CODE     ---       LVL=0
      0200025FH   SYMBOL    XDATA    DWORD     baud_rate
      01000026H   LINE      CODE     ---       #75
      0100002CH   LINE      CODE     ---       #76
      0100002CH   LINE      CODE     ---       #78
      0100002FH   LINE      CODE     ---       #79
      01000032H   LINE      CODE     ---       #80
      01000035H   LINE      CODE     ---       #82
      0100003AH   LINE      CODE     ---       #84
      0100003CH   LINE      CODE     ---       #85
      0100003EH   LINE      CODE     ---       #87
      01000040H   LINE      CODE     ---       #88
      01000042H   LINE      CODE     ---       #90
LX51 LINKER/LOCATER V4.66.97.0                                                        06/12/2025  17:35:51  PAGE 27


      01000057H   LINE      CODE     ---       #91
      01000059H   LINE      CODE     ---       #93
      0100005CH   LINE      CODE     ---       #94
      ---         BLOCKEND  ---      ---       LVL=0
      00000007H   SYMBOL    DATA     BYTE      irqstate
      00000001H   SYMBOL    DATA     ---       pfunc_recv

      01000006H   BLOCK     CODE     ---       LVL=0
      00000007H   SYMBOL    DATA     CHAR      c
      01000006H   BLOCK     CODE     NEAR LAB  LVL=1
      00000004H   SYMBOL    DATA     WORD      timeout
      ---         BLOCKEND  ---      ---       LVL=1
      01000006H   LINE      CODE     ---       #127
      01000006H   LINE      CODE     ---       #128
      01000006H   LINE      CODE     ---       #131
      0100000AH   LINE      CODE     ---       #133
      0100000CH   LINE      CODE     ---       #140
      0100000FH   LINE      CODE     ---       #141
      0100000FH   LINE      CODE     ---       #142
      01000019H   LINE      CODE     ---       #143
      01000019H   LINE      CODE     ---       #144
      01000019H   LINE      CODE     ---       #145
      01000019H   LINE      CODE     ---       #146
      01000019H   LINE      CODE     ---       #147
      0100001BH   LINE      CODE     ---       #149
      ---         BLOCKEND  ---      ---       LVL=0

      01001F1DH   BLOCK     CODE     ---       LVL=0
      00000003H   SYMBOL    DATA     CHAR      c
      01001F1DH   LINE      CODE     ---       #185
      01001F1FH   LINE      CODE     ---       #186
      01001F1FH   LINE      CODE     ---       #187
      ---         BLOCKEND  ---      ---       LVL=0

      ---         MODULE    ---      ---       GPIO
      020002D1H   PUBLIC    XDATA    ---       gpiofunc
      01001CB7H   PUBLIC    CODE     ---       _gpio_irq_clr
      01001420H   PUBLIC    CODE     ---       _gpio_irq_set
      010018D6H   PUBLIC    CODE     ---       _gpio_io_set
      01001D41H   PUBLIC    CODE     ---       _gpio_io_get
      01001855H   PUBLIC    CODE     ---       _gpio_pd_set
      010017D4H   PUBLIC    CODE     ---       _gpio_pu_set
      010014E3H   PUBLIC    CODE     ---       _gpio_in_enable
      01001753H   PUBLIC    CODE     ---       _gpio_dir_set
      01001DC1H   PUBLIC    CODE     ---       _gpio_init
      00000098H.3 SFRSYM    DATA     BIT       TB80
      000000E0H.7 SFRSYM    DATA     BIT       ACC7
      00000080H   SFRSYM    DATA     BYTE      P0
      00000090H   SFRSYM    DATA     BYTE      P1
      000000A0H   SFRSYM    DATA     BYTE      P2
      00000098H.5 SFRSYM    DATA     BIT       SM20
      000000B2H   SFRSYM    DATA     BYTE      ESTCR
      000000B1H   SFRSYM    DATA     BYTE      CLKST
      000000D0H.6 SFRSYM    DATA     BIT       AC
      000000D8H.3 SFRSYM    DATA     BIT       ERSTF
      000000E6H   SFRSYM    DATA     BYTE      PRESET0
      000000D4H   SFRSYM    DATA     BYTE      OCTRL
      000000A8H.7 SFRSYM    DATA     BIT       EA
      0000008FH   SFRSYM    DATA     BYTE      POREN
      000000C8H   SFRSYM    DATA     BYTE      PWM0CON
      000000E7H   SFRSYM    DATA     BYTE      PRESET1
      000000C9H   SFRSYM    DATA     BYTE      PWM1CON
      00000086H   SFRSYM    DATA     BYTE      BEEPCTR
      000000CAH   SFRSYM    DATA     BYTE      PWM2CON
      000000B8H.4 SFRSYM    DATA     BIT       LPTIMINTEN
LX51 LINKER/LOCATER V4.66.97.0                                                        06/12/2025  17:35:51  PAGE 28


      000000ABH   SFRSYM    DATA     BYTE      P0AH
      000000B0H   SFRSYM    DATA     BYTE      P1AH
      000000E8H   SFRSYM    DATA     BYTE      P2AH
      000000F8H.6 SFRSYM    DATA     BIT       RC32KF
      000000A8H   SFRSYM    DATA     BYTE      IEN0
      000000A7H   SFRSYM    DATA     BYTE      OPSET
      000000A4H   SFRSYM    DATA     BYTE      P0AL
      000000B8H   SFRSYM    DATA     BYTE      IEN1
      000000A8H.6 SFRSYM    DATA     BIT       EADC
      00000085H   SFRSYM    DATA     BYTE      DPH1
      000000AEH   SFRSYM    DATA     BYTE      P1AL
      0000009AH   SFRSYM    DATA     BYTE      IEN2
      000000C0H   SFRSYM    DATA     BYTE      P2AL
      000000B6H   SFRSYM    DATA     BYTE      ADCDR0
      000000F8H.5 SFRSYM    DATA     BIT       RC16MF
      000000B7H   SFRSYM    DATA     BYTE      ADCDR1
      00000084H   SFRSYM    DATA     BYTE      DPL1
      000000D6H   SFRSYM    DATA     BYTE      P0OD
      000000DBH   SFRSYM    DATA     BYTE      P1OD
      000000D5H   SFRSYM    DATA     BYTE      P0PD
      00000098H.4 SFRSYM    DATA     BIT       REN0
      000000ECH   SFRSYM    DATA     BYTE      P2OD
      000000DAH   SFRSYM    DATA     BYTE      P1PD
      000000E4H   SFRSYM    DATA     BYTE      P2PD
      000000D7H   SFRSYM    DATA     BYTE      P0CS
      00000097H   SFRSYM    DATA     BYTE      P0DR
      0000009EH   SFRSYM    DATA     BYTE      EUARTEN
      000000DCH   SFRSYM    DATA     BYTE      P1CS
      000000E5H   SFRSYM    DATA     BYTE      P1DR
      000000F4H   SFRSYM    DATA     BYTE      P2CS
      000000FCH   SFRSYM    DATA     BYTE      P2DR
      000000D0H.7 SFRSYM    DATA     BIT       CY
      000000D8H.0 SFRSYM    DATA     BIT       WDT0
      000000D8H.1 SFRSYM    DATA     BIT       WDT1
      000000D8H.2 SFRSYM    DATA     BIT       WDT2
      00000081H   SFRSYM    DATA     BYTE      SP
      000000F1H   SFRSYM    DATA     BYTE      P0PU
      000000F2H   SFRSYM    DATA     BYTE      P1PU
      000000D1H   SFRSYM    DATA     WORD      OADR
      000000F3H   SFRSYM    DATA     BYTE      P2PU
      00000093H   SFRSYM    DATA     BYTE      ADCIER
      000000A5H   SFRSYM    DATA     BYTE      OSEC
      000000D8H.6 SFRSYM    DATA     BIT       WDEN
      000000BAH   SFRSYM    DATA     BYTE      S0RELH
      00000080H.0 SFRSYM    DATA     BIT       P00
      000000D8H.7 SFRSYM    DATA     BIT       WDOF
      000000BBH   SFRSYM    DATA     BYTE      S1RELH
      00000090H.0 SFRSYM    DATA     BIT       P10
      00000080H.1 SFRSYM    DATA     BIT       P01
      00000087H   SFRSYM    DATA     BYTE      PCON
      000000C4H   SFRSYM    DATA     BYTE      PWM0DH
      000000A0H.0 SFRSYM    DATA     BIT       P20
      00000090H.1 SFRSYM    DATA     BIT       P11
      00000080H.2 SFRSYM    DATA     BIT       P02
      000000C6H   SFRSYM    DATA     BYTE      PWM1DH
      00000090H.2 SFRSYM    DATA     BIT       P12
      00000080H.3 SFRSYM    DATA     BIT       P03
      000000C7H   SFRSYM    DATA     BYTE      PWM2DH
      000000C8H.2 SFRSYM    DATA     BIT       PWM0IE
      000000AAH   SFRSYM    DATA     BYTE      S0RELL
      000000A0H.2 SFRSYM    DATA     BIT       P22
      00000090H.3 SFRSYM    DATA     BIT       P13
      00000080H.4 SFRSYM    DATA     BIT       P04
      000000C8H.1 SFRSYM    DATA     BIT       PWM0IF
      0000009DH   SFRSYM    DATA     BYTE      S1RELL
LX51 LINKER/LOCATER V4.66.97.0                                                        06/12/2025  17:35:51  PAGE 29


      000000A0H.3 SFRSYM    DATA     BIT       P23
      00000090H.4 SFRSYM    DATA     BIT       P14
      00000080H.5 SFRSYM    DATA     BIT       P05
      000000C3H   SFRSYM    DATA     BYTE      PWM0DL
      00000090H.5 SFRSYM    DATA     BIT       P15
      000000A6H   SFRSYM    DATA     BYTE      OSTATUS
      000000C5H   SFRSYM    DATA     BYTE      PWM1DL
      000000A0H.5 SFRSYM    DATA     BIT       P25
      000000D8H.4 SFRSYM    DATA     BIT       PORF
      000000D8H   SFRSYM    DATA     BYTE      RSTSTAT
      000000CFH   SFRSYM    DATA     BYTE      PWM2DL
      000000A0H.6 SFRSYM    DATA     BIT       P26
      000000C8H.7 SFRSYM    DATA     BIT       PWM0EN
      000000A0H.7 SFRSYM    DATA     BIT       P27
      000000A8H.5 SFRSYM    DATA     BIT       EPWM
      000000D8H.5 SFRSYM    DATA     BIT       LVRF
      000000F8H   SFRSYM    DATA     BYTE      CLKCON
      000000CCH   SFRSYM    DATA     BYTE      PWM0PH
      000000CEH   SFRSYM    DATA     BYTE      PWM1PH
      000000B8H.5 SFRSYM    DATA     BIT       I2CINTEN
      000000C2H   SFRSYM    DATA     BYTE      PWM2PH
      000000F0H   SFRSYM    DATA     BYTE      B
      000000EEH   SFRSYM    DATA     BYTE      RCHDIV
      000000CBH   SFRSYM    DATA     BYTE      PWM0PL
      000000CDH   SFRSYM    DATA     BYTE      PWM1PL
      000000C1H   SFRSYM    DATA     BYTE      PWM2PL
      000000F7H   SFRSYM    DATA     BYTE      ADCSPW
      000000F8H.1 SFRSYM    DATA     BIT       XCLKEN
      000000E0H   SFRSYM    DATA     BYTE      ACC
      000000DDH   SFRSYM    DATA     BYTE      LVDCON
      000000A8H.4 SFRSYM    DATA     BIT       ES0
      000000A9H   SFRSYM    DATA     BYTE      IP0
      000000A8H.1 SFRSYM    DATA     BIT       ET0
      000000A8H.2 SFRSYM    DATA     BIT       ES1
      000000F6H   SFRSYM    DATA     BYTE      ADCCSTAT
      000000B9H   SFRSYM    DATA     BYTE      IP1
      000000A8H.3 SFRSYM    DATA     BIT       ET1
      00000098H.0 SFRSYM    DATA     BIT       RI0
      000000C8H.0 SFRSYM    DATA     BIT       PWM0SS
      00000098H.1 SFRSYM    DATA     BIT       TI0
      000000A8H.0 SFRSYM    DATA     BIT       EX0
      000000D0H.0 SFRSYM    DATA     BIT       P
      000000B8H.3 SFRSYM    DATA     BIT       EFCINTEN
      000000A2H   SFRSYM    DATA     BYTE      OINTEN
      00000098H.7 SFRSYM    DATA     BIT       SM0
      00000098H.6 SFRSYM    DATA     BIT       SM1
      000000FEH   SFRSYM    DATA     BYTE      ADCCDR0
      000000FFH   SFRSYM    DATA     BYTE      ADCCDR1
      000000D0H.3 SFRSYM    DATA     BIT       RS0
      000000ACH   SFRSYM    DATA     BYTE      ADCGCR0
      000000D0H.4 SFRSYM    DATA     BIT       RS1
      000000ADH   SFRSYM    DATA     BYTE      ADCGCR1
      000000B4H   SFRSYM    DATA     BYTE      ADCGCR2
      000000B5H   SFRSYM    DATA     BYTE      ADCGCR3
      000000F8H.3 SFRSYM    DATA     BIT       RC32KEN
      000000DEH   SFRSYM    DATA     BYTE      PCLK0
      000000DFH   SFRSYM    DATA     BYTE      PCLK1
      00000083H   SFRSYM    DATA     BYTE      DPH
      000000E9H   SFRSYM    DATA     BYTE      P0IEN
      000000F5H   SFRSYM    DATA     BYTE      ADCHL
      000000F8H.2 SFRSYM    DATA     BIT       RC16MEN
      000000EAH   SFRSYM    DATA     BYTE      P1IEN
      000000EBH   SFRSYM    DATA     BYTE      P2IEN
      000000B6H   SFRSYM    DATA     WORD      ADCDR
      000000B3H   SFRSYM    DATA     BYTE      XTHCTR
LX51 LINKER/LOCATER V4.66.97.0                                                        06/12/2025  17:35:51  PAGE 30


      00000082H   SFRSYM    DATA     BYTE      DPL
      00000099H   SFRSYM    DATA     BYTE      S0BUF
      0000009CH   SFRSYM    DATA     BYTE      S1BUF
      000000F9H   SFRSYM    DATA     BYTE      P0OEN
      000000B8H.0 SFRSYM    DATA     BIT       GTIM0INTEN
      000000D9H   SFRSYM    DATA     BYTE      SYSDIV
      00000098H   SFRSYM    DATA     BYTE      S0CON
      000000FAH   SFRSYM    DATA     BYTE      P1OEN
      000000B8H.2 SFRSYM    DATA     BIT       GTIM1INTEN
      000000A3H   SFRSYM    DATA     BYTE      OINTUS
      000000BEH   SFRSYM    DATA     BYTE      RCHTRIMH
      000000F8H.0 SFRSYM    DATA     BIT       SYSSEL
      0000009BH   SFRSYM    DATA     BYTE      S1CON
      000000FBH   SFRSYM    DATA     BYTE      P2OEN
      000000B8H.6 SFRSYM    DATA     BIT       GTIM2INTEN
      000000BDH   SFRSYM    DATA     BYTE      LDOTRIMH
      00000092H   SFRSYM    DATA     BYTE      DPS
      0000009FH   SFRSYM    DATA     BYTE      RCLTRIMH
      000000BFH   SFRSYM    DATA     BYTE      RCHTRIML
      000000D3H   SFRSYM    DATA     BYTE      ODATA
      00000091H   SFRSYM    DATA     BYTE      LDOTRIML
      000000BCH   SFRSYM    DATA     BYTE      RCLTRIML
      000000E1H   SFRSYM    DATA     BYTE      P0IRQ
      000000B8H.1 SFRSYM    DATA     BIT       SPIINTEN
      000000E2H   SFRSYM    DATA     BYTE      P1IRQ
      000000E3H   SFRSYM    DATA     BYTE      P2IRQ
      000000D2H   SFRSYM    DATA     BYTE      OADRH
      000000B8H.7 SFRSYM    DATA     BIT       UART2INTEN
      000000F0H.0 SFRSYM    DATA     BIT       B0
      000000F0H.1 SFRSYM    DATA     BIT       B1
      000000F0H.2 SFRSYM    DATA     BIT       B2
      000000D1H   SFRSYM    DATA     BYTE      OADRL
      000000F0H.3 SFRSYM    DATA     BIT       B3
      000000F0H.4 SFRSYM    DATA     BIT       B4
      000000D0H.5 SFRSYM    DATA     BIT       F0
      000000F0H.5 SFRSYM    DATA     BIT       B5
      000000D0H.1 SFRSYM    DATA     BIT       F1
      000000AFH   SFRSYM    DATA     BYTE      REMAP
      000000F0H.6 SFRSYM    DATA     BIT       B6
      000000E0H.0 SFRSYM    DATA     BIT       ACC0
      000000A1H   SFRSYM    DATA     BYTE      OUS
      000000C8H.6 SFRSYM    DATA     BIT       PWM0S
      000000F0H.7 SFRSYM    DATA     BIT       B7
      000000E0H.1 SFRSYM    DATA     BIT       ACC1
      000000F8H.4 SFRSYM    DATA     BIT       XCLKF
      000000E0H.2 SFRSYM    DATA     BIT       ACC2
      0000008EH   SFRSYM    DATA     BYTE      PDSEL
      000000E0H.3 SFRSYM    DATA     BIT       ACC3
      000000D0H   SFRSYM    DATA     BYTE      PSW
      000000E0H.4 SFRSYM    DATA     BIT       ACC4
      00000098H.2 SFRSYM    DATA     BIT       RB80
      000000E0H.5 SFRSYM    DATA     BIT       ACC5
      000000FDH   SFRSYM    DATA     BYTE      ADCVREF
      000000E0H.6 SFRSYM    DATA     BIT       ACC6

      01001DC1H   BLOCK     CODE     ---       LVL=0
      00000007H   SYMBOL    DATA     BYTE      pin
      01001DC1H   BLOCK     CODE     NEAR LAB  LVL=1
      00000006H   SYMBOL    DATA     BYTE      gpio_pin
      02000261H   SYMBOL    XDATA    BYTE      gpio_num
      ---         BLOCKEND  ---      ---       LVL=1
      01001DC1H   LINE      CODE     ---       #42
      01001DC1H   LINE      CODE     ---       #43
      01001DC1H   LINE      CODE     ---       #44
      01001DC8H   LINE      CODE     ---       #45
LX51 LINKER/LOCATER V4.66.97.0                                                        06/12/2025  17:35:51  PAGE 31


      01001DCFH   LINE      CODE     ---       #48
      01001DD5H   LINE      CODE     ---       #49
      01001DD5H   LINE      CODE     ---       #50
      01001DD8H   LINE      CODE     ---       #51
      01001DDBH   LINE      CODE     ---       #52
      01001DDCH   LINE      CODE     ---       #53
      01001DE2H   LINE      CODE     ---       #54
      01001DE2H   LINE      CODE     ---       #55
      01001DE5H   LINE      CODE     ---       #56
      01001DE8H   LINE      CODE     ---       #57
      01001DE9H   LINE      CODE     ---       #58
      01001DEFH   LINE      CODE     ---       #59
      01001DEFH   LINE      CODE     ---       #60
      01001DF2H   LINE      CODE     ---       #61
      01001DF5H   LINE      CODE     ---       #62
      01001DF5H   LINE      CODE     ---       #63
      ---         BLOCKEND  ---      ---       LVL=0

      01001753H   BLOCK     CODE     ---       LVL=0
      00000007H   SYMBOL    DATA     BYTE      pin
      00000005H   SYMBOL    DATA     BYTE      dir
      01001753H   BLOCK     CODE     NEAR LAB  LVL=1
      00000006H   SYMBOL    DATA     BYTE      gpio_pin
      00000007H   SYMBOL    DATA     BYTE      gpio_num
      ---         BLOCKEND  ---      ---       LVL=1
      01001753H   LINE      CODE     ---       #72
      01001753H   LINE      CODE     ---       #73
      01001753H   LINE      CODE     ---       #74
      0100175AH   LINE      CODE     ---       #75
      0100175EH   LINE      CODE     ---       #77
      01001761H   LINE      CODE     ---       #78
      01001761H   LINE      CODE     ---       #79
      01001767H   LINE      CODE     ---       #80
      01001767H   LINE      CODE     ---       #81
      01001773H   LINE      CODE     ---       #82
      01001774H   LINE      CODE     ---       #83
      0100177AH   LINE      CODE     ---       #84
      0100177AH   LINE      CODE     ---       #85
      01001786H   LINE      CODE     ---       #86
      01001787H   LINE      CODE     ---       #87
      0100178CH   LINE      CODE     ---       #88
      0100178CH   LINE      CODE     ---       #89
      01001798H   LINE      CODE     ---       #90
      01001798H   LINE      CODE     ---       #92
      01001799H   LINE      CODE     ---       #94
      01001799H   LINE      CODE     ---       #95
      0100179FH   LINE      CODE     ---       #96
      0100179FH   LINE      CODE     ---       #97
      010017ACH   LINE      CODE     ---       #98
      010017ADH   LINE      CODE     ---       #99
      010017B3H   LINE      CODE     ---       #100
      010017B3H   LINE      CODE     ---       #101
      010017C0H   LINE      CODE     ---       #103
      010017C1H   LINE      CODE     ---       #104
      010017C6H   LINE      CODE     ---       #105
      010017C6H   LINE      CODE     ---       #106
      010017D3H   LINE      CODE     ---       #107
      010017D3H   LINE      CODE     ---       #108
      010017D3H   LINE      CODE     ---       #109
      ---         BLOCKEND  ---      ---       LVL=0

      010014E3H   BLOCK     CODE     ---       LVL=0
      00000007H   SYMBOL    DATA     BYTE      pin
      00000005H   SYMBOL    DATA     BYTE      mode
      010014E3H   BLOCK     CODE     NEAR LAB  LVL=1
LX51 LINKER/LOCATER V4.66.97.0                                                        06/12/2025  17:35:51  PAGE 32


      00000006H   SYMBOL    DATA     BYTE      gpio_pin
      00000007H   SYMBOL    DATA     BYTE      gpio_num
      ---         BLOCKEND  ---      ---       LVL=1
      010014E3H   LINE      CODE     ---       #117
      010014E3H   LINE      CODE     ---       #118
      010014E3H   LINE      CODE     ---       #119
      010014EAH   LINE      CODE     ---       #120
      010014EEH   LINE      CODE     ---       #122
      010014F1H   LINE      CODE     ---       #123
      010014F1H   LINE      CODE     ---       #124
      010014F7H   LINE      CODE     ---       #125
      010014F7H   LINE      CODE     ---       #126
      0100150BH   LINE      CODE     ---       #127
      0100150DH   LINE      CODE     ---       #128
      01001513H   LINE      CODE     ---       #129
      01001513H   LINE      CODE     ---       #130
      01001527H   LINE      CODE     ---       #131
      01001529H   LINE      CODE     ---       #132
      0100152EH   LINE      CODE     ---       #133
      0100152EH   LINE      CODE     ---       #134
      01001543H   LINE      CODE     ---       #135
      01001543H   LINE      CODE     ---       #137
      01001545H   LINE      CODE     ---       #139
      01001545H   LINE      CODE     ---       #140
      0100154BH   LINE      CODE     ---       #141
      0100154BH   LINE      CODE     ---       #142
      01001561H   LINE      CODE     ---       #143
      01001563H   LINE      CODE     ---       #144
      01001569H   LINE      CODE     ---       #145
      01001569H   LINE      CODE     ---       #146
      0100157FH   LINE      CODE     ---       #147
      01001581H   LINE      CODE     ---       #148
      01001586H   LINE      CODE     ---       #149
      01001586H   LINE      CODE     ---       #150
      010015A1H   LINE      CODE     ---       #151
      010015A1H   LINE      CODE     ---       #153
      010015A1H   LINE      CODE     ---       #154
      ---         BLOCKEND  ---      ---       LVL=0

      010017D4H   BLOCK     CODE     ---       LVL=0
      00000007H   SYMBOL    DATA     BYTE      pin
      00000005H   SYMBOL    DATA     BYTE      mode
      010017D4H   BLOCK     CODE     NEAR LAB  LVL=1
      00000006H   SYMBOL    DATA     BYTE      gpio_pin
      00000007H   SYMBOL    DATA     BYTE      gpio_num
      ---         BLOCKEND  ---      ---       LVL=1
      010017D4H   LINE      CODE     ---       #163
      010017D4H   LINE      CODE     ---       #164
      010017D4H   LINE      CODE     ---       #165
      010017DBH   LINE      CODE     ---       #166
      010017DFH   LINE      CODE     ---       #168
      010017E2H   LINE      CODE     ---       #169
      010017E2H   LINE      CODE     ---       #170
      010017E8H   LINE      CODE     ---       #171
      010017E8H   LINE      CODE     ---       #172
      010017F4H   LINE      CODE     ---       #173
      010017F5H   LINE      CODE     ---       #174
      010017FBH   LINE      CODE     ---       #175
      010017FBH   LINE      CODE     ---       #176
      01001807H   LINE      CODE     ---       #177
      01001808H   LINE      CODE     ---       #178
      0100180DH   LINE      CODE     ---       #179
      0100180DH   LINE      CODE     ---       #180
      01001819H   LINE      CODE     ---       #181
      01001819H   LINE      CODE     ---       #182
LX51 LINKER/LOCATER V4.66.97.0                                                        06/12/2025  17:35:51  PAGE 33


      0100181AH   LINE      CODE     ---       #184
      0100181AH   LINE      CODE     ---       #185
      01001820H   LINE      CODE     ---       #186
      01001820H   LINE      CODE     ---       #187
      0100182DH   LINE      CODE     ---       #188
      0100182EH   LINE      CODE     ---       #189
      01001834H   LINE      CODE     ---       #190
      01001834H   LINE      CODE     ---       #191
      01001841H   LINE      CODE     ---       #192
      01001842H   LINE      CODE     ---       #193
      01001847H   LINE      CODE     ---       #194
      01001847H   LINE      CODE     ---       #195
      01001854H   LINE      CODE     ---       #196
      01001854H   LINE      CODE     ---       #197
      01001854H   LINE      CODE     ---       #198
      ---         BLOCKEND  ---      ---       LVL=0

      01001855H   BLOCK     CODE     ---       LVL=0
      00000007H   SYMBOL    DATA     BYTE      pin
      00000005H   SYMBOL    DATA     BYTE      mode
      01001855H   BLOCK     CODE     NEAR LAB  LVL=1
      00000006H   SYMBOL    DATA     BYTE      gpio_pin
      00000007H   SYMBOL    DATA     BYTE      gpio_num
      ---         BLOCKEND  ---      ---       LVL=1
      01001855H   LINE      CODE     ---       #207
      01001855H   LINE      CODE     ---       #208
      01001855H   LINE      CODE     ---       #209
      0100185CH   LINE      CODE     ---       #210
      01001860H   LINE      CODE     ---       #212
      01001863H   LINE      CODE     ---       #213
      01001863H   LINE      CODE     ---       #214
      01001869H   LINE      CODE     ---       #215
      01001869H   LINE      CODE     ---       #216
      01001875H   LINE      CODE     ---       #217
      01001876H   LINE      CODE     ---       #218
      0100187CH   LINE      CODE     ---       #219
      0100187CH   LINE      CODE     ---       #220
      01001888H   LINE      CODE     ---       #221
      01001889H   LINE      CODE     ---       #222
      0100188EH   LINE      CODE     ---       #223
      0100188EH   LINE      CODE     ---       #224
      0100189AH   LINE      CODE     ---       #225
      0100189AH   LINE      CODE     ---       #226
      0100189BH   LINE      CODE     ---       #228
      0100189BH   LINE      CODE     ---       #229
      010018A1H   LINE      CODE     ---       #230
      010018A1H   LINE      CODE     ---       #231
      010018AEH   LINE      CODE     ---       #232
      010018AFH   LINE      CODE     ---       #233
      010018B5H   LINE      CODE     ---       #234
      010018B5H   LINE      CODE     ---       #235
      010018C2H   LINE      CODE     ---       #236
      010018C3H   LINE      CODE     ---       #237
      010018C8H   LINE      CODE     ---       #238
      010018C8H   LINE      CODE     ---       #239
      010018D5H   LINE      CODE     ---       #240
      010018D5H   LINE      CODE     ---       #241
      010018D5H   LINE      CODE     ---       #242
      ---         BLOCKEND  ---      ---       LVL=0
      00000007H   SYMBOL    DATA     BYTE      pin
      00000005H   SYMBOL    DATA     BYTE      mode
      00000006H   SYMBOL    DATA     BYTE      gpio_pin
      00000007H   SYMBOL    DATA     BYTE      gpio_num
      00000007H   SYMBOL    DATA     BYTE      pin
      00000005H   SYMBOL    DATA     BYTE      mode
LX51 LINKER/LOCATER V4.66.97.0                                                        06/12/2025  17:35:51  PAGE 34


      00000006H   SYMBOL    DATA     BYTE      gpio_pin
      00000007H   SYMBOL    DATA     BYTE      gpio_num
      00000007H   SYMBOL    DATA     BYTE      pin
      00000005H   SYMBOL    DATA     BYTE      mode
      00000006H   SYMBOL    DATA     BYTE      gpio_pin
      00000007H   SYMBOL    DATA     BYTE      gpio_num
      00000007H   SYMBOL    DATA     BYTE      pin
      00000005H   SYMBOL    DATA     BYTE      mode
      00000006H   SYMBOL    DATA     BYTE      gpio_pin
      00000007H   SYMBOL    DATA     BYTE      gpio_num

      01001D41H   BLOCK     CODE     ---       LVL=0
      00000007H   SYMBOL    DATA     BYTE      pin
      01001D41H   BLOCK     CODE     NEAR LAB  LVL=1
      00000006H   SYMBOL    DATA     BYTE      gpio_pin
      00000007H   SYMBOL    DATA     BYTE      gpio_num
      ---         BLOCKEND  ---      ---       LVL=1
      01001D41H   LINE      CODE     ---       #428
      01001D41H   LINE      CODE     ---       #429
      01001D41H   LINE      CODE     ---       #430
      01001D48H   LINE      CODE     ---       #431
      01001D4CH   LINE      CODE     ---       #433
      01001D52H   LINE      CODE     ---       #434
      01001D52H   LINE      CODE     ---       #435
      01001D5FH   LINE      CODE     ---       #436
      01001D5FH   LINE      CODE     ---       #437
      01001D65H   LINE      CODE     ---       #438
      01001D65H   LINE      CODE     ---       #439
      01001D72H   LINE      CODE     ---       #440
      01001D72H   LINE      CODE     ---       #442
      01001D72H   LINE      CODE     ---       #443
      01001D80H   LINE      CODE     ---       #444
      01001D80H   LINE      CODE     ---       #446
      ---         BLOCKEND  ---      ---       LVL=0

      010018D6H   BLOCK     CODE     ---       LVL=0
      00000007H   SYMBOL    DATA     BYTE      pin
      00000005H   SYMBOL    DATA     BYTE      level
      010018D6H   BLOCK     CODE     NEAR LAB  LVL=1
      00000006H   SYMBOL    DATA     BYTE      gpio_pin
      00000007H   SYMBOL    DATA     BYTE      gpio_num
      ---         BLOCKEND  ---      ---       LVL=1
      010018D6H   LINE      CODE     ---       #456
      010018D6H   LINE      CODE     ---       #457
      010018D6H   LINE      CODE     ---       #458
      010018DDH   LINE      CODE     ---       #459
      010018E1H   LINE      CODE     ---       #461
      010018E4H   LINE      CODE     ---       #462
      010018E4H   LINE      CODE     ---       #463
      010018EAH   LINE      CODE     ---       #464
      010018EAH   LINE      CODE     ---       #465
      010018F6H   LINE      CODE     ---       #466
      010018F7H   LINE      CODE     ---       #467
      010018FDH   LINE      CODE     ---       #468
      010018FDH   LINE      CODE     ---       #469
      01001909H   LINE      CODE     ---       #470
      0100190AH   LINE      CODE     ---       #471
      0100190FH   LINE      CODE     ---       #472
      0100190FH   LINE      CODE     ---       #473
      0100191BH   LINE      CODE     ---       #474
      0100191BH   LINE      CODE     ---       #475
      0100191CH   LINE      CODE     ---       #477
      0100191CH   LINE      CODE     ---       #478
      01001922H   LINE      CODE     ---       #479
      01001922H   LINE      CODE     ---       #480
LX51 LINKER/LOCATER V4.66.97.0                                                        06/12/2025  17:35:51  PAGE 35


      0100192FH   LINE      CODE     ---       #481
      01001930H   LINE      CODE     ---       #482
      01001936H   LINE      CODE     ---       #483
      01001936H   LINE      CODE     ---       #484
      01001943H   LINE      CODE     ---       #485
      01001944H   LINE      CODE     ---       #486
      01001949H   LINE      CODE     ---       #487
      01001949H   LINE      CODE     ---       #488
      01001956H   LINE      CODE     ---       #489
      01001956H   LINE      CODE     ---       #490
      01001956H   LINE      CODE     ---       #491
      ---         BLOCKEND  ---      ---       LVL=0

      01001420H   BLOCK     CODE     ---       LVL=0
      00000004H   SYMBOL    DATA     BYTE      pin
      00000005H   SYMBOL    DATA     BYTE      mode
      00000001H   SYMBOL    DATA     ---       pfunc
      01001422H   BLOCK     CODE     NEAR LAB  LVL=1
      0200025FH   SYMBOL    XDATA    BYTE      gpio_pin
      02000260H   SYMBOL    XDATA    BYTE      gpio_num
      ---         BLOCKEND  ---      ---       LVL=1
      01001420H   LINE      CODE     ---       #501
      01001422H   LINE      CODE     ---       #502
      01001422H   LINE      CODE     ---       #503
      0100142CH   LINE      CODE     ---       #505
      01001431H   LINE      CODE     ---       #507
      01001434H   LINE      CODE     ---       #508
      01001434H   LINE      CODE     ---       #509
      01001445H   LINE      CODE     ---       #511
      01001447H   LINE      CODE     ---       #512
      01001449H   LINE      CODE     ---       #513
      0100144CH   LINE      CODE     ---       #514
      01001455H   LINE      CODE     ---       #515
      01001455H   LINE      CODE     ---       #516
      01001464H   LINE      CODE     ---       #517
      01001465H   LINE      CODE     ---       #518
      0100146BH   LINE      CODE     ---       #519
      0100146BH   LINE      CODE     ---       #520
      0100147CH   LINE      CODE     ---       #521
      0100147DH   LINE      CODE     ---       #522
      01001485H   LINE      CODE     ---       #523
      01001485H   LINE      CODE     ---       #524
      01001494H   LINE      CODE     ---       #525
      01001494H   LINE      CODE     ---       #526
      01001495H   LINE      CODE     ---       #528
      01001495H   LINE      CODE     ---       #529
      01001497H   LINE      CODE     ---       #530
      010014A0H   LINE      CODE     ---       #531
      010014A0H   LINE      CODE     ---       #532
      010014B0H   LINE      CODE     ---       #533
      010014B1H   LINE      CODE     ---       #534
      010014B7H   LINE      CODE     ---       #535
      010014B7H   LINE      CODE     ---       #536
      010014C9H   LINE      CODE     ---       #537
      010014CAH   LINE      CODE     ---       #538
      010014D2H   LINE      CODE     ---       #539
      010014D2H   LINE      CODE     ---       #540
      010014E2H   LINE      CODE     ---       #541
      010014E2H   LINE      CODE     ---       #542
      010014E2H   LINE      CODE     ---       #544
      ---         BLOCKEND  ---      ---       LVL=0

      01001CB7H   BLOCK     CODE     ---       LVL=0
      00000007H   SYMBOL    DATA     BYTE      pin
      01001CB7H   BLOCK     CODE     NEAR LAB  LVL=1
LX51 LINKER/LOCATER V4.66.97.0                                                        06/12/2025  17:35:51  PAGE 36


      00000006H   SYMBOL    DATA     BYTE      gpio_pin
      00000007H   SYMBOL    DATA     BYTE      gpio_num
      ---         BLOCKEND  ---      ---       LVL=1
      01001CB7H   LINE      CODE     ---       #553
      01001CB7H   LINE      CODE     ---       #554
      01001CB7H   LINE      CODE     ---       #555
      01001CBEH   LINE      CODE     ---       #556
      01001CC2H   LINE      CODE     ---       #558
      01001CC8H   LINE      CODE     ---       #559
      01001CC8H   LINE      CODE     ---       #560
      01001CD5H   LINE      CODE     ---       #561
      01001CD6H   LINE      CODE     ---       #562
      01001CDCH   LINE      CODE     ---       #563
      01001CDCH   LINE      CODE     ---       #564
      01001CE9H   LINE      CODE     ---       #565
      01001CEAH   LINE      CODE     ---       #566
      01001CEFH   LINE      CODE     ---       #567
      01001CEFH   LINE      CODE     ---       #568
      01001CFCH   LINE      CODE     ---       #569
      01001CFCH   LINE      CODE     ---       #570
      ---         BLOCKEND  ---      ---       LVL=0
      00000007H   SYMBOL    DATA     BYTE      pin
      00000006H   SYMBOL    DATA     BYTE      gpio_pin
      00000007H   SYMBOL    DATA     BYTE      gpio_num

      ---         MODULE    ---      ---       LPTIMER
      02000319H   PUBLIC    XDATA    ---       lptimfunc
      01001F0EH   PUBLIC    CODE     ---       lptimer_start
      01001F05H   PUBLIC    CODE     ---       _lptimer_set_time
      01001E2BH   PUBLIC    CODE     ---       _lptimer_init
      01001358H   PUBLIC    CODE     ---       LPTIMER_IRQHandler
      00000098H.3 SFRSYM    DATA     BIT       TB80
      000000E0H.7 SFRSYM    DATA     BIT       ACC7
      00000080H   SFRSYM    DATA     BYTE      P0
      00000090H   SFRSYM    DATA     BYTE      P1
      000000A0H   SFRSYM    DATA     BYTE      P2
      00000098H.5 SFRSYM    DATA     BIT       SM20
      000000B2H   SFRSYM    DATA     BYTE      ESTCR
      000000B1H   SFRSYM    DATA     BYTE      CLKST
      000000D0H.6 SFRSYM    DATA     BIT       AC
      000000D8H.3 SFRSYM    DATA     BIT       ERSTF
      000000E6H   SFRSYM    DATA     BYTE      PRESET0
      000000D4H   SFRSYM    DATA     BYTE      OCTRL
      000000A8H.7 SFRSYM    DATA     BIT       EA
      0000008FH   SFRSYM    DATA     BYTE      POREN
      000000C8H   SFRSYM    DATA     BYTE      PWM0CON
      000000E7H   SFRSYM    DATA     BYTE      PRESET1
      000000C9H   SFRSYM    DATA     BYTE      PWM1CON
      00000086H   SFRSYM    DATA     BYTE      BEEPCTR
      000000CAH   SFRSYM    DATA     BYTE      PWM2CON
      000000B8H.4 SFRSYM    DATA     BIT       LPTIMINTEN
      000000ABH   SFRSYM    DATA     BYTE      P0AH
      000000B0H   SFRSYM    DATA     BYTE      P1AH
      000000E8H   SFRSYM    DATA     BYTE      P2AH
      000000F8H.6 SFRSYM    DATA     BIT       RC32KF
      000000A8H   SFRSYM    DATA     BYTE      IEN0
      000000A7H   SFRSYM    DATA     BYTE      OPSET
      000000A4H   SFRSYM    DATA     BYTE      P0AL
      000000B8H   SFRSYM    DATA     BYTE      IEN1
      000000A8H.6 SFRSYM    DATA     BIT       EADC
      00000085H   SFRSYM    DATA     BYTE      DPH1
      000000AEH   SFRSYM    DATA     BYTE      P1AL
      0000009AH   SFRSYM    DATA     BYTE      IEN2
      000000C0H   SFRSYM    DATA     BYTE      P2AL
      000000B6H   SFRSYM    DATA     BYTE      ADCDR0
LX51 LINKER/LOCATER V4.66.97.0                                                        06/12/2025  17:35:51  PAGE 37


      000000F8H.5 SFRSYM    DATA     BIT       RC16MF
      000000B7H   SFRSYM    DATA     BYTE      ADCDR1
      00000084H   SFRSYM    DATA     BYTE      DPL1
      000000D6H   SFRSYM    DATA     BYTE      P0OD
      000000DBH   SFRSYM    DATA     BYTE      P1OD
      000000D5H   SFRSYM    DATA     BYTE      P0PD
      00000098H.4 SFRSYM    DATA     BIT       REN0
      000000ECH   SFRSYM    DATA     BYTE      P2OD
      000000DAH   SFRSYM    DATA     BYTE      P1PD
      000000E4H   SFRSYM    DATA     BYTE      P2PD
      000000D7H   SFRSYM    DATA     BYTE      P0CS
      00000097H   SFRSYM    DATA     BYTE      P0DR
      0000009EH   SFRSYM    DATA     BYTE      EUARTEN
      000000DCH   SFRSYM    DATA     BYTE      P1CS
      000000E5H   SFRSYM    DATA     BYTE      P1DR
      000000F4H   SFRSYM    DATA     BYTE      P2CS
      000000FCH   SFRSYM    DATA     BYTE      P2DR
      000000D0H.7 SFRSYM    DATA     BIT       CY
      000000D8H.0 SFRSYM    DATA     BIT       WDT0
      000000D8H.1 SFRSYM    DATA     BIT       WDT1
      000000D8H.2 SFRSYM    DATA     BIT       WDT2
      00000081H   SFRSYM    DATA     BYTE      SP
      000000F1H   SFRSYM    DATA     BYTE      P0PU
      000000F2H   SFRSYM    DATA     BYTE      P1PU
      000000D1H   SFRSYM    DATA     WORD      OADR
      000000F3H   SFRSYM    DATA     BYTE      P2PU
      00000093H   SFRSYM    DATA     BYTE      ADCIER
      000000A5H   SFRSYM    DATA     BYTE      OSEC
      000000D8H.6 SFRSYM    DATA     BIT       WDEN
      000000BAH   SFRSYM    DATA     BYTE      S0RELH
      00000080H.0 SFRSYM    DATA     BIT       P00
      000000D8H.7 SFRSYM    DATA     BIT       WDOF
      000000BBH   SFRSYM    DATA     BYTE      S1RELH
      00000090H.0 SFRSYM    DATA     BIT       P10
      00000080H.1 SFRSYM    DATA     BIT       P01
      00000087H   SFRSYM    DATA     BYTE      PCON
      000000C4H   SFRSYM    DATA     BYTE      PWM0DH
      000000A0H.0 SFRSYM    DATA     BIT       P20
      00000090H.1 SFRSYM    DATA     BIT       P11
      00000080H.2 SFRSYM    DATA     BIT       P02
      000000C6H   SFRSYM    DATA     BYTE      PWM1DH
      00000090H.2 SFRSYM    DATA     BIT       P12
      00000080H.3 SFRSYM    DATA     BIT       P03
      000000C7H   SFRSYM    DATA     BYTE      PWM2DH
      000000C8H.2 SFRSYM    DATA     BIT       PWM0IE
      000000AAH   SFRSYM    DATA     BYTE      S0RELL
      000000A0H.2 SFRSYM    DATA     BIT       P22
      00000090H.3 SFRSYM    DATA     BIT       P13
      00000080H.4 SFRSYM    DATA     BIT       P04
      000000C8H.1 SFRSYM    DATA     BIT       PWM0IF
      0000009DH   SFRSYM    DATA     BYTE      S1RELL
      000000A0H.3 SFRSYM    DATA     BIT       P23
      00000090H.4 SFRSYM    DATA     BIT       P14
      00000080H.5 SFRSYM    DATA     BIT       P05
      000000C3H   SFRSYM    DATA     BYTE      PWM0DL
      00000090H.5 SFRSYM    DATA     BIT       P15
      000000A6H   SFRSYM    DATA     BYTE      OSTATUS
      000000C5H   SFRSYM    DATA     BYTE      PWM1DL
      000000A0H.5 SFRSYM    DATA     BIT       P25
      000000D8H.4 SFRSYM    DATA     BIT       PORF
      000000D8H   SFRSYM    DATA     BYTE      RSTSTAT
      000000CFH   SFRSYM    DATA     BYTE      PWM2DL
      000000A0H.6 SFRSYM    DATA     BIT       P26
      000000C8H.7 SFRSYM    DATA     BIT       PWM0EN
      000000A0H.7 SFRSYM    DATA     BIT       P27
LX51 LINKER/LOCATER V4.66.97.0                                                        06/12/2025  17:35:51  PAGE 38


      000000A8H.5 SFRSYM    DATA     BIT       EPWM
      000000D8H.5 SFRSYM    DATA     BIT       LVRF
      000000F8H   SFRSYM    DATA     BYTE      CLKCON
      000000CCH   SFRSYM    DATA     BYTE      PWM0PH
      000000CEH   SFRSYM    DATA     BYTE      PWM1PH
      000000B8H.5 SFRSYM    DATA     BIT       I2CINTEN
      000000C2H   SFRSYM    DATA     BYTE      PWM2PH
      000000F0H   SFRSYM    DATA     BYTE      B
      000000EEH   SFRSYM    DATA     BYTE      RCHDIV
      000000CBH   SFRSYM    DATA     BYTE      PWM0PL
      000000CDH   SFRSYM    DATA     BYTE      PWM1PL
      000000C1H   SFRSYM    DATA     BYTE      PWM2PL
      000000F7H   SFRSYM    DATA     BYTE      ADCSPW
      000000F8H.1 SFRSYM    DATA     BIT       XCLKEN
      000000E0H   SFRSYM    DATA     BYTE      ACC
      000000DDH   SFRSYM    DATA     BYTE      LVDCON
      000000A8H.4 SFRSYM    DATA     BIT       ES0
      000000A9H   SFRSYM    DATA     BYTE      IP0
      000000A8H.1 SFRSYM    DATA     BIT       ET0
      000000A8H.2 SFRSYM    DATA     BIT       ES1
      000000F6H   SFRSYM    DATA     BYTE      ADCCSTAT
      000000B9H   SFRSYM    DATA     BYTE      IP1
      000000A8H.3 SFRSYM    DATA     BIT       ET1
      00000098H.0 SFRSYM    DATA     BIT       RI0
      000000C8H.0 SFRSYM    DATA     BIT       PWM0SS
      00000098H.1 SFRSYM    DATA     BIT       TI0
      000000A8H.0 SFRSYM    DATA     BIT       EX0
      000000D0H.0 SFRSYM    DATA     BIT       P
      000000B8H.3 SFRSYM    DATA     BIT       EFCINTEN
      000000A2H   SFRSYM    DATA     BYTE      OINTEN
      00000098H.7 SFRSYM    DATA     BIT       SM0
      00000098H.6 SFRSYM    DATA     BIT       SM1
      000000FEH   SFRSYM    DATA     BYTE      ADCCDR0
      000000FFH   SFRSYM    DATA     BYTE      ADCCDR1
      000000D0H.3 SFRSYM    DATA     BIT       RS0
      000000ACH   SFRSYM    DATA     BYTE      ADCGCR0
      000000D0H.4 SFRSYM    DATA     BIT       RS1
      000000ADH   SFRSYM    DATA     BYTE      ADCGCR1
      000000B4H   SFRSYM    DATA     BYTE      ADCGCR2
      000000B5H   SFRSYM    DATA     BYTE      ADCGCR3
      000000F8H.3 SFRSYM    DATA     BIT       RC32KEN
      000000DEH   SFRSYM    DATA     BYTE      PCLK0
      000000DFH   SFRSYM    DATA     BYTE      PCLK1
      00000083H   SFRSYM    DATA     BYTE      DPH
      000000E9H   SFRSYM    DATA     BYTE      P0IEN
      000000F5H   SFRSYM    DATA     BYTE      ADCHL
      000000F8H.2 SFRSYM    DATA     BIT       RC16MEN
      000000EAH   SFRSYM    DATA     BYTE      P1IEN
      000000EBH   SFRSYM    DATA     BYTE      P2IEN
      000000B6H   SFRSYM    DATA     WORD      ADCDR
      000000B3H   SFRSYM    DATA     BYTE      XTHCTR
      00000082H   SFRSYM    DATA     BYTE      DPL
      00000099H   SFRSYM    DATA     BYTE      S0BUF
      0000009CH   SFRSYM    DATA     BYTE      S1BUF
      000000F9H   SFRSYM    DATA     BYTE      P0OEN
      000000B8H.0 SFRSYM    DATA     BIT       GTIM0INTEN
      000000D9H   SFRSYM    DATA     BYTE      SYSDIV
      00000098H   SFRSYM    DATA     BYTE      S0CON
      000000FAH   SFRSYM    DATA     BYTE      P1OEN
      000000B8H.2 SFRSYM    DATA     BIT       GTIM1INTEN
      000000A3H   SFRSYM    DATA     BYTE      OINTUS
      000000BEH   SFRSYM    DATA     BYTE      RCHTRIMH
      000000F8H.0 SFRSYM    DATA     BIT       SYSSEL
      0000009BH   SFRSYM    DATA     BYTE      S1CON
      000000FBH   SFRSYM    DATA     BYTE      P2OEN
LX51 LINKER/LOCATER V4.66.97.0                                                        06/12/2025  17:35:51  PAGE 39


      000000B8H.6 SFRSYM    DATA     BIT       GTIM2INTEN
      000000BDH   SFRSYM    DATA     BYTE      LDOTRIMH
      00000092H   SFRSYM    DATA     BYTE      DPS
      0000009FH   SFRSYM    DATA     BYTE      RCLTRIMH
      000000BFH   SFRSYM    DATA     BYTE      RCHTRIML
      000000D3H   SFRSYM    DATA     BYTE      ODATA
      00000091H   SFRSYM    DATA     BYTE      LDOTRIML
      000000BCH   SFRSYM    DATA     BYTE      RCLTRIML
      000000E1H   SFRSYM    DATA     BYTE      P0IRQ
      000000B8H.1 SFRSYM    DATA     BIT       SPIINTEN
      000000E2H   SFRSYM    DATA     BYTE      P1IRQ
      000000E3H   SFRSYM    DATA     BYTE      P2IRQ
      000000D2H   SFRSYM    DATA     BYTE      OADRH
      000000B8H.7 SFRSYM    DATA     BIT       UART2INTEN
      000000F0H.0 SFRSYM    DATA     BIT       B0
      000000F0H.1 SFRSYM    DATA     BIT       B1
      000000F0H.2 SFRSYM    DATA     BIT       B2
      000000D1H   SFRSYM    DATA     BYTE      OADRL
      000000F0H.3 SFRSYM    DATA     BIT       B3
      000000F0H.4 SFRSYM    DATA     BIT       B4
      000000D0H.5 SFRSYM    DATA     BIT       F0
      000000F0H.5 SFRSYM    DATA     BIT       B5
      000000D0H.1 SFRSYM    DATA     BIT       F1
      000000AFH   SFRSYM    DATA     BYTE      REMAP
      000000F0H.6 SFRSYM    DATA     BIT       B6
      000000E0H.0 SFRSYM    DATA     BIT       ACC0
      000000A1H   SFRSYM    DATA     BYTE      OUS
      000000C8H.6 SFRSYM    DATA     BIT       PWM0S
      000000F0H.7 SFRSYM    DATA     BIT       B7
      000000E0H.1 SFRSYM    DATA     BIT       ACC1
      000000F8H.4 SFRSYM    DATA     BIT       XCLKF
      000000E0H.2 SFRSYM    DATA     BIT       ACC2
      0000008EH   SFRSYM    DATA     BYTE      PDSEL
      000000E0H.3 SFRSYM    DATA     BIT       ACC3
      000000D0H   SFRSYM    DATA     BYTE      PSW
      000000E0H.4 SFRSYM    DATA     BIT       ACC4
      00000098H.2 SFRSYM    DATA     BIT       RB80
      000000E0H.5 SFRSYM    DATA     BIT       ACC5
      000000FDH   SFRSYM    DATA     BYTE      ADCVREF
      000000E0H.6 SFRSYM    DATA     BIT       ACC6

      01001358H   BLOCK     CODE     ---       LVL=0
      01001358H   LINE      CODE     ---       #20
      01001375H   LINE      CODE     ---       #22
      01001389H   LINE      CODE     ---       #23
      01001389H   LINE      CODE     ---       #24
      0100138CH   LINE      CODE     ---       #26
      01001396H   LINE      CODE     ---       #27
      01001396H   LINE      CODE     ---       #28
      01001396H   LINE      CODE     ---       #29
      01001396H   LINE      CODE     ---       #30
      01001398H   LINE      CODE     ---       #31
      010013ACH   LINE      CODE     ---       #32
      010013ACH   LINE      CODE     ---       #33
      010013B0H   LINE      CODE     ---       #35
      010013BAH   LINE      CODE     ---       #36
      010013BAH   LINE      CODE     ---       #37
      010013BAH   LINE      CODE     ---       #38
      010013BAH   LINE      CODE     ---       #39
      010013BCH   LINE      CODE     ---       #40
      010013D0H   LINE      CODE     ---       #41
      010013D0H   LINE      CODE     ---       #42
      010013D4H   LINE      CODE     ---       #44
      010013DEH   LINE      CODE     ---       #45
      010013DEH   LINE      CODE     ---       #46
LX51 LINKER/LOCATER V4.66.97.0                                                        06/12/2025  17:35:51  PAGE 40


      010013DEH   LINE      CODE     ---       #47
      010013DEH   LINE      CODE     ---       #48
      010013E0H   LINE      CODE     ---       #49
      010013F4H   LINE      CODE     ---       #50
      010013F4H   LINE      CODE     ---       #51
      010013F8H   LINE      CODE     ---       #53
      01001402H   LINE      CODE     ---       #54
      01001402H   LINE      CODE     ---       #55
      01001405H   LINE      CODE     ---       #56
      01001405H   LINE      CODE     ---       #57
      01001405H   LINE      CODE     ---       #58
      ---         BLOCKEND  ---      ---       LVL=0

      01001E2BH   BLOCK     CODE     ---       LVL=0
      00000007H   SYMBOL    DATA     BYTE      tmode
      00000005H   SYMBOL    DATA     BYTE      clock_sel
      00000003H   SYMBOL    DATA     BYTE      div
      01001E2BH   LINE      CODE     ---       #69
      01001E2BH   LINE      CODE     ---       #70
      01001E2BH   LINE      CODE     ---       #71
      01001E2EH   LINE      CODE     ---       #72
      01001E31H   LINE      CODE     ---       #74
      01001E42H   LINE      CODE     ---       #75
      01001E47H   LINE      CODE     ---       #76
      01001E54H   LINE      CODE     ---       #78
      01001E58H   LINE      CODE     ---       #80
      01001E5AH   LINE      CODE     ---       #82
      ---         BLOCKEND  ---      ---       LVL=0
      00000007H   SYMBOL    DATA     BYTE      irqstate
      00000005H   SYMBOL    DATA     BYTE      ie
      00000007H   SYMBOL    DATA     BYTE      clock_sel
      00000005H   SYMBOL    DATA     BYTE      div
      00000007H   SYMBOL    DATA     BYTE      channel
      00000005H   SYMBOL    DATA     BYTE      polar

      01001F05H   BLOCK     CODE     ---       LVL=0
      00000006H   SYMBOL    DATA     WORD      target
      01001F05H   LINE      CODE     ---       #228
      01001F05H   LINE      CODE     ---       #229
      01001F05H   LINE      CODE     ---       #230
      01001F0AH   LINE      CODE     ---       #231
      01001F0DH   LINE      CODE     ---       #233
      ---         BLOCKEND  ---      ---       LVL=0
      00000007H   SYMBOL    DATA     BYTE      channel
      00000005H   SYMBOL    DATA     BYTE      edge
      00000007H   SYMBOL    DATA     BYTE      channel

      01001F0EH   BLOCK     CODE     ---       LVL=0
      01001F0EH   LINE      CODE     ---       #276
      01001F0EH   LINE      CODE     ---       #277
      01001F0EH   LINE      CODE     ---       #278
      01001F15H   LINE      CODE     ---       #279
      ---         BLOCKEND  ---      ---       LVL=0
      00000007H   SYMBOL    DATA     BYTE      edge
      00000007H   SYMBOL    DATA     BYTE      edge
      00000007H   SYMBOL    DATA     BYTE      io

      ---         MODULE    ---      ---       RADIO
      01001EE3H   PUBLIC    CODE     ---       radio_init

      01001EE3H   BLOCK     CODE     ---       LVL=0
      01001EE3H   LINE      CODE     ---       #22
      01001EE3H   LINE      CODE     ---       #23
      01001EE3H   LINE      CODE     ---       #24
      01001EE6H   LINE      CODE     ---       #25
LX51 LINKER/LOCATER V4.66.97.0                                                        06/12/2025  17:35:51  PAGE 41


      01001EE9H   LINE      CODE     ---       #26
      01001EECH   LINE      CODE     ---       #28
      01001EEEH   LINE      CODE     ---       #29
      ---         BLOCKEND  ---      ---       LVL=0

      ---         MODULE    ---      ---       UM2006A
      02000000H   PUBLIC    XDATA    ---       rf_config
      01001EC7H   PUBLIC    CODE     ---       um2006A_reset_digit
      010015A2H   PUBLIC    CODE     ---       um2006A_cal_rc32K
      01001EB9H   PUBLIC    CODE     ---       um2006A_into_rx_bpfcal
      01001E92H   PUBLIC    CODE     ---       _um2006A_read_reg
      01001E0AH   PUBLIC    CODE     ---       _um2006A_write_reg
      01001A4EH   PUBLIC    CODE     ---       um2006A_init
      00000098H.3 SFRSYM    DATA     BIT       TB80
      000000E0H.7 SFRSYM    DATA     BIT       ACC7
      00000080H   SFRSYM    DATA     BYTE      P0
      00000090H   SFRSYM    DATA     BYTE      P1
      000000A0H   SFRSYM    DATA     BYTE      P2
      00000098H.5 SFRSYM    DATA     BIT       SM20
      000000B2H   SFRSYM    DATA     BYTE      ESTCR
      000000B1H   SFRSYM    DATA     BYTE      CLKST
      000000D0H.6 SFRSYM    DATA     BIT       AC
      000000D8H.3 SFRSYM    DATA     BIT       ERSTF
      000000E6H   SFRSYM    DATA     BYTE      PRESET0
      000000D4H   SFRSYM    DATA     BYTE      OCTRL
      000000A8H.7 SFRSYM    DATA     BIT       EA
      0000008FH   SFRSYM    DATA     BYTE      POREN
      000000C8H   SFRSYM    DATA     BYTE      PWM0CON
      000000E7H   SFRSYM    DATA     BYTE      PRESET1
      000000C9H   SFRSYM    DATA     BYTE      PWM1CON
      00000086H   SFRSYM    DATA     BYTE      BEEPCTR
      000000CAH   SFRSYM    DATA     BYTE      PWM2CON
      000000B8H.4 SFRSYM    DATA     BIT       LPTIMINTEN
      000000ABH   SFRSYM    DATA     BYTE      P0AH
      000000B0H   SFRSYM    DATA     BYTE      P1AH
      000000E8H   SFRSYM    DATA     BYTE      P2AH
      000000F8H.6 SFRSYM    DATA     BIT       RC32KF
      000000A8H   SFRSYM    DATA     BYTE      IEN0
      000000A7H   SFRSYM    DATA     BYTE      OPSET
      000000A4H   SFRSYM    DATA     BYTE      P0AL
      000000B8H   SFRSYM    DATA     BYTE      IEN1
      000000A8H.6 SFRSYM    DATA     BIT       EADC
      00000085H   SFRSYM    DATA     BYTE      DPH1
      000000AEH   SFRSYM    DATA     BYTE      P1AL
      0000009AH   SFRSYM    DATA     BYTE      IEN2
      000000C0H   SFRSYM    DATA     BYTE      P2AL
      000000B6H   SFRSYM    DATA     BYTE      ADCDR0
      000000F8H.5 SFRSYM    DATA     BIT       RC16MF
      000000B7H   SFRSYM    DATA     BYTE      ADCDR1
      00000084H   SFRSYM    DATA     BYTE      DPL1
      000000D6H   SFRSYM    DATA     BYTE      P0OD
      000000DBH   SFRSYM    DATA     BYTE      P1OD
      000000D5H   SFRSYM    DATA     BYTE      P0PD
      00000098H.4 SFRSYM    DATA     BIT       REN0
      000000ECH   SFRSYM    DATA     BYTE      P2OD
      000000DAH   SFRSYM    DATA     BYTE      P1PD
      000000E4H   SFRSYM    DATA     BYTE      P2PD
      000000D7H   SFRSYM    DATA     BYTE      P0CS
      00000097H   SFRSYM    DATA     BYTE      P0DR
      0000009EH   SFRSYM    DATA     BYTE      EUARTEN
      000000DCH   SFRSYM    DATA     BYTE      P1CS
      000000E5H   SFRSYM    DATA     BYTE      P1DR
      000000F4H   SFRSYM    DATA     BYTE      P2CS
      000000FCH   SFRSYM    DATA     BYTE      P2DR
      000000D0H.7 SFRSYM    DATA     BIT       CY
LX51 LINKER/LOCATER V4.66.97.0                                                        06/12/2025  17:35:51  PAGE 42


      000000D8H.0 SFRSYM    DATA     BIT       WDT0
      000000D8H.1 SFRSYM    DATA     BIT       WDT1
      000000D8H.2 SFRSYM    DATA     BIT       WDT2
      00000081H   SFRSYM    DATA     BYTE      SP
      000000F1H   SFRSYM    DATA     BYTE      P0PU
      000000F2H   SFRSYM    DATA     BYTE      P1PU
      000000D1H   SFRSYM    DATA     WORD      OADR
      000000F3H   SFRSYM    DATA     BYTE      P2PU
      00000093H   SFRSYM    DATA     BYTE      ADCIER
      000000A5H   SFRSYM    DATA     BYTE      OSEC
      000000D8H.6 SFRSYM    DATA     BIT       WDEN
      000000BAH   SFRSYM    DATA     BYTE      S0RELH
      00000080H.0 SFRSYM    DATA     BIT       P00
      000000D8H.7 SFRSYM    DATA     BIT       WDOF
      000000BBH   SFRSYM    DATA     BYTE      S1RELH
      00000090H.0 SFRSYM    DATA     BIT       P10
      00000080H.1 SFRSYM    DATA     BIT       P01
      00000087H   SFRSYM    DATA     BYTE      PCON
      000000C4H   SFRSYM    DATA     BYTE      PWM0DH
      000000A0H.0 SFRSYM    DATA     BIT       P20
      00000090H.1 SFRSYM    DATA     BIT       P11
      00000080H.2 SFRSYM    DATA     BIT       P02
      000000C6H   SFRSYM    DATA     BYTE      PWM1DH
      00000090H.2 SFRSYM    DATA     BIT       P12
      00000080H.3 SFRSYM    DATA     BIT       P03
      000000C7H   SFRSYM    DATA     BYTE      PWM2DH
      000000C8H.2 SFRSYM    DATA     BIT       PWM0IE
      000000AAH   SFRSYM    DATA     BYTE      S0RELL
      000000A0H.2 SFRSYM    DATA     BIT       P22
      00000090H.3 SFRSYM    DATA     BIT       P13
      00000080H.4 SFRSYM    DATA     BIT       P04
      000000C8H.1 SFRSYM    DATA     BIT       PWM0IF
      0000009DH   SFRSYM    DATA     BYTE      S1RELL
      000000A0H.3 SFRSYM    DATA     BIT       P23
      00000090H.4 SFRSYM    DATA     BIT       P14
      00000080H.5 SFRSYM    DATA     BIT       P05
      000000C3H   SFRSYM    DATA     BYTE      PWM0DL
      00000090H.5 SFRSYM    DATA     BIT       P15
      000000A6H   SFRSYM    DATA     BYTE      OSTATUS
      000000C5H   SFRSYM    DATA     BYTE      PWM1DL
      000000A0H.5 SFRSYM    DATA     BIT       P25
      000000D8H.4 SFRSYM    DATA     BIT       PORF
      000000D8H   SFRSYM    DATA     BYTE      RSTSTAT
      000000CFH   SFRSYM    DATA     BYTE      PWM2DL
      000000A0H.6 SFRSYM    DATA     BIT       P26
      000000C8H.7 SFRSYM    DATA     BIT       PWM0EN
      000000A0H.7 SFRSYM    DATA     BIT       P27
      000000A8H.5 SFRSYM    DATA     BIT       EPWM
      000000D8H.5 SFRSYM    DATA     BIT       LVRF
      000000F8H   SFRSYM    DATA     BYTE      CLKCON
      000000CCH   SFRSYM    DATA     BYTE      PWM0PH
      000000CEH   SFRSYM    DATA     BYTE      PWM1PH
      000000B8H.5 SFRSYM    DATA     BIT       I2CINTEN
      000000C2H   SFRSYM    DATA     BYTE      PWM2PH
      000000F0H   SFRSYM    DATA     BYTE      B
      000000EEH   SFRSYM    DATA     BYTE      RCHDIV
      000000CBH   SFRSYM    DATA     BYTE      PWM0PL
      000000CDH   SFRSYM    DATA     BYTE      PWM1PL
      000000C1H   SFRSYM    DATA     BYTE      PWM2PL
      000000F7H   SFRSYM    DATA     BYTE      ADCSPW
      000000F8H.1 SFRSYM    DATA     BIT       XCLKEN
      000000E0H   SFRSYM    DATA     BYTE      ACC
      000000DDH   SFRSYM    DATA     BYTE      LVDCON
      000000A8H.4 SFRSYM    DATA     BIT       ES0
      000000A9H   SFRSYM    DATA     BYTE      IP0
LX51 LINKER/LOCATER V4.66.97.0                                                        06/12/2025  17:35:51  PAGE 43


      000000A8H.1 SFRSYM    DATA     BIT       ET0
      000000A8H.2 SFRSYM    DATA     BIT       ES1
      000000F6H   SFRSYM    DATA     BYTE      ADCCSTAT
      000000B9H   SFRSYM    DATA     BYTE      IP1
      000000A8H.3 SFRSYM    DATA     BIT       ET1
      00000098H.0 SFRSYM    DATA     BIT       RI0
      000000C8H.0 SFRSYM    DATA     BIT       PWM0SS
      00000098H.1 SFRSYM    DATA     BIT       TI0
      000000A8H.0 SFRSYM    DATA     BIT       EX0
      000000D0H.0 SFRSYM    DATA     BIT       P
      000000B8H.3 SFRSYM    DATA     BIT       EFCINTEN
      000000A2H   SFRSYM    DATA     BYTE      OINTEN
      00000098H.7 SFRSYM    DATA     BIT       SM0
      00000098H.6 SFRSYM    DATA     BIT       SM1
      000000FEH   SFRSYM    DATA     BYTE      ADCCDR0
      000000FFH   SFRSYM    DATA     BYTE      ADCCDR1
      000000D0H.3 SFRSYM    DATA     BIT       RS0
      000000ACH   SFRSYM    DATA     BYTE      ADCGCR0
      000000D0H.4 SFRSYM    DATA     BIT       RS1
      000000ADH   SFRSYM    DATA     BYTE      ADCGCR1
      000000B4H   SFRSYM    DATA     BYTE      ADCGCR2
      000000B5H   SFRSYM    DATA     BYTE      ADCGCR3
      000000F8H.3 SFRSYM    DATA     BIT       RC32KEN
      000000DEH   SFRSYM    DATA     BYTE      PCLK0
      000000DFH   SFRSYM    DATA     BYTE      PCLK1
      00000083H   SFRSYM    DATA     BYTE      DPH
      000000E9H   SFRSYM    DATA     BYTE      P0IEN
      000000F5H   SFRSYM    DATA     BYTE      ADCHL
      000000F8H.2 SFRSYM    DATA     BIT       RC16MEN
      000000EAH   SFRSYM    DATA     BYTE      P1IEN
      000000EBH   SFRSYM    DATA     BYTE      P2IEN
      000000B6H   SFRSYM    DATA     WORD      ADCDR
      000000B3H   SFRSYM    DATA     BYTE      XTHCTR
      00000082H   SFRSYM    DATA     BYTE      DPL
      00000099H   SFRSYM    DATA     BYTE      S0BUF
      0000009CH   SFRSYM    DATA     BYTE      S1BUF
      000000F9H   SFRSYM    DATA     BYTE      P0OEN
      000000B8H.0 SFRSYM    DATA     BIT       GTIM0INTEN
      000000D9H   SFRSYM    DATA     BYTE      SYSDIV
      00000098H   SFRSYM    DATA     BYTE      S0CON
      000000FAH   SFRSYM    DATA     BYTE      P1OEN
      000000B8H.2 SFRSYM    DATA     BIT       GTIM1INTEN
      000000A3H   SFRSYM    DATA     BYTE      OINTUS
      000000BEH   SFRSYM    DATA     BYTE      RCHTRIMH
      000000F8H.0 SFRSYM    DATA     BIT       SYSSEL
      0000009BH   SFRSYM    DATA     BYTE      S1CON
      000000FBH   SFRSYM    DATA     BYTE      P2OEN
      000000B8H.6 SFRSYM    DATA     BIT       GTIM2INTEN
      000000BDH   SFRSYM    DATA     BYTE      LDOTRIMH
      00000092H   SFRSYM    DATA     BYTE      DPS
      0000009FH   SFRSYM    DATA     BYTE      RCLTRIMH
      000000BFH   SFRSYM    DATA     BYTE      RCHTRIML
      000000D3H   SFRSYM    DATA     BYTE      ODATA
      00000091H   SFRSYM    DATA     BYTE      LDOTRIML
      000000BCH   SFRSYM    DATA     BYTE      RCLTRIML
      000000E1H   SFRSYM    DATA     BYTE      P0IRQ
      000000B8H.1 SFRSYM    DATA     BIT       SPIINTEN
      000000E2H   SFRSYM    DATA     BYTE      P1IRQ
      000000E3H   SFRSYM    DATA     BYTE      P2IRQ
      000000D2H   SFRSYM    DATA     BYTE      OADRH
      000000B8H.7 SFRSYM    DATA     BIT       UART2INTEN
      000000F0H.0 SFRSYM    DATA     BIT       B0
      000000F0H.1 SFRSYM    DATA     BIT       B1
      000000F0H.2 SFRSYM    DATA     BIT       B2
      000000D1H   SFRSYM    DATA     BYTE      OADRL
LX51 LINKER/LOCATER V4.66.97.0                                                        06/12/2025  17:35:51  PAGE 44


      000000F0H.3 SFRSYM    DATA     BIT       B3
      000000F0H.4 SFRSYM    DATA     BIT       B4
      000000D0H.5 SFRSYM    DATA     BIT       F0
      000000F0H.5 SFRSYM    DATA     BIT       B5
      000000D0H.1 SFRSYM    DATA     BIT       F1
      000000AFH   SFRSYM    DATA     BYTE      REMAP
      000000F0H.6 SFRSYM    DATA     BIT       B6
      000000E0H.0 SFRSYM    DATA     BIT       ACC0
      000000A1H   SFRSYM    DATA     BYTE      OUS
      000000C8H.6 SFRSYM    DATA     BIT       PWM0S
      000000F0H.7 SFRSYM    DATA     BIT       B7
      000000E0H.1 SFRSYM    DATA     BIT       ACC1
      000000F8H.4 SFRSYM    DATA     BIT       XCLKF
      000000E0H.2 SFRSYM    DATA     BIT       ACC2
      0000008EH   SFRSYM    DATA     BYTE      PDSEL
      000000E0H.3 SFRSYM    DATA     BIT       ACC3
      000000D0H   SFRSYM    DATA     BYTE      PSW
      000000E0H.4 SFRSYM    DATA     BIT       ACC4
      00000098H.2 SFRSYM    DATA     BIT       RB80
      000000E0H.5 SFRSYM    DATA     BIT       ACC5
      000000FDH   SFRSYM    DATA     BYTE      ADCVREF
      000000E0H.6 SFRSYM    DATA     BIT       ACC6
      02000078H   SYMBOL    XDATA    ---       wor_sleep
      020000A8H   SYMBOL    XDATA    ---       wor_t1
      020000D8H   SYMBOL    XDATA    ---       wor_t2
      02000108H   SYMBOL    XDATA    ---       wor_t3
      02000138H   SYMBOL    XDATA    ---       shape_if_offset_200K
      02000148H   SYMBOL    XDATA    ---       shape_if_offset_340K

      01001A4EH   BLOCK     CODE     ---       LVL=0
      01001A4EH   BLOCK     CODE     NEAR LAB  LVL=1
      0200025FH   SYMBOL    XDATA    BYTE      i
      02000260H   SYMBOL    XDATA    BYTE      len
      ---         BLOCKEND  ---      ---       LVL=1
      01001A4EH   LINE      CODE     ---       #25
      01001A4EH   LINE      CODE     ---       #26
      01001A4EH   LINE      CODE     ---       #27
      01001A53H   LINE      CODE     ---       #28
      01001A55H   LINE      CODE     ---       #30
      01001A58H   LINE      CODE     ---       #32
      01001A5BH   LINE      CODE     ---       #33
      01001A66H   LINE      CODE     ---       #35
      01001A6DH   LINE      CODE     ---       #36
      01001A73H   LINE      CODE     ---       #37
      01001A86H   LINE      CODE     ---       #38
      01001A86H   LINE      CODE     ---       #39
      01001A97H   LINE      CODE     ---       #40
      01001A97H   LINE      CODE     ---       #41
      01001A97H   LINE      CODE     ---       #42
      01001A97H   LINE      CODE     ---       #43
      01001AABH   LINE      CODE     ---       #44
      01001AB3H   LINE      CODE     ---       #46
      ---         BLOCKEND  ---      ---       LVL=0

      01001DF6H   BLOCK     CODE     VOID      LVL=0
      ---         BLOCKEND  ---      ---       LVL=0

      01001E0AH   BLOCK     CODE     ---       LVL=0
      02000268H   SYMBOL    XDATA    BYTE      addr
      02000269H   SYMBOL    XDATA    BYTE      value
      01001E0AH   LINE      CODE     ---       #56
      01001E12H   LINE      CODE     ---       #57
      01001E12H   LINE      CODE     ---       #58
      01001E15H   LINE      CODE     ---       #59
      01001E1DH   LINE      CODE     ---       #60
LX51 LINKER/LOCATER V4.66.97.0                                                        06/12/2025  17:35:51  PAGE 45


      01001E20H   LINE      CODE     ---       #61
      01001E28H   LINE      CODE     ---       #62
      ---         BLOCKEND  ---      ---       LVL=0

      01001E8BH   BLOCK     CODE     VOID      LVL=0
      ---         BLOCKEND  ---      ---       LVL=0

      01001E92H   BLOCK     CODE     ---       LVL=0
      02000268H   SYMBOL    XDATA    BYTE      addr
      02000269H   SYMBOL    XDATA    BYTE      value
      01001E97H   BLOCK     CODE     NEAR LAB  LVL=1
      02000269H   SYMBOL    XDATA    BYTE      value
      ---         BLOCKEND  ---      ---       LVL=1
      01001E92H   LINE      CODE     ---       #92
      01001E97H   LINE      CODE     ---       #93
      01001E97H   LINE      CODE     ---       #94
      01001E9AH   LINE      CODE     ---       #95
      01001E9DH   LINE      CODE     ---       #96
      01001EA5H   LINE      CODE     ---       #97
      01001EA8H   LINE      CODE     ---       #98
      01001EB0H   LINE      CODE     ---       #99
      01001EB3H   LINE      CODE     ---       #100
      01001EB8H   LINE      CODE     ---       #101
      ---         BLOCKEND  ---      ---       LVL=0
      00000001H   SYMBOL    DATA     ---       dat
      00000005H   SYMBOL    DATA     BYTE      len

      01001EB9H   BLOCK     CODE     ---       LVL=0
      01001EB9H   LINE      CODE     ---       #196
      01001EB9H   LINE      CODE     ---       #197
      01001EB9H   LINE      CODE     ---       #198
      01001EC0H   LINE      CODE     ---       #199
      ---         BLOCKEND  ---      ---       LVL=0
      00000007H   SYMBOL    DATA     BYTE      tmp
      00000007H   SYMBOL    DATA     BYTE      tmp
      00000007H   SYMBOL    DATA     BYTE      tmp
      00000007H   SYMBOL    DATA     BYTE      reg09

      010015A2H   BLOCK     CODE     ---       LVL=0
      010015A2H   BLOCK     CODE     NEAR LAB  LVL=1
      02000261H   SYMBOL    XDATA    DWORD     count
      02000265H   SYMBOL    XDATA    BYTE      reg03
      02000266H   SYMBOL    XDATA    BYTE      reg07
      02000267H   SYMBOL    XDATA    BYTE      reg51
      ---         BLOCKEND  ---      ---       LVL=1
      010015A2H   LINE      CODE     ---       #313
      010015A2H   LINE      CODE     ---       #314
      010015A2H   LINE      CODE     ---       #315
      010015ACH   LINE      CODE     ---       #317
      010015B6H   LINE      CODE     ---       #318
      010015C0H   LINE      CODE     ---       #319
      010015CAH   LINE      CODE     ---       #321
      010015D1H   LINE      CODE     ---       #322
      010015DDH   LINE      CODE     ---       #323
      010015E9H   LINE      CODE     ---       #324
      010015F0H   LINE      CODE     ---       #325
      010015FAH   LINE      CODE     ---       #326
      01001608H   LINE      CODE     ---       #327
      01001608H   LINE      CODE     ---       #328
      01001611H   LINE      CODE     ---       #329
      01001611H   LINE      CODE     ---       #330
      01001611H   LINE      CODE     ---       #331
      01001611H   LINE      CODE     ---       #332
      01001612H   LINE      CODE     ---       #333
      01001613H   LINE      CODE     ---       #334
LX51 LINKER/LOCATER V4.66.97.0                                                        06/12/2025  17:35:51  PAGE 46


      01001614H   LINE      CODE     ---       #335
      01001615H   LINE      CODE     ---       #336
      01001616H   LINE      CODE     ---       #337
      01001618H   LINE      CODE     ---       #339
      0100161FH   LINE      CODE     ---       #340
      01001629H   LINE      CODE     ---       #341
      01001633H   LINE      CODE     ---       #342
      ---         BLOCKEND  ---      ---       LVL=0
      00000007H   SYMBOL    DATA     BYTE      value
      00000007H   SYMBOL    DATA     BYTE      value
      00000004H   SYMBOL    DATA     FLOAT     rssithr
      00000007H   SYMBOL    DATA     BYTE      rssi
      00000007H   SYMBOL    DATA     BYTE      reg03
      00000001H   SYMBOL    DATA     ---       array
      00000005H   SYMBOL    DATA     BYTE      rows
      00000007H   SYMBOL    DATA     BYTE      reg0E
      00000005H   SYMBOL    DATA     BYTE      reg0E
      00000005H   SYMBOL    DATA     BYTE      reg0E

      01001EC7H   BLOCK     CODE     ---       LVL=0
      01001EC7H   LINE      CODE     ---       #1102
      01001EC7H   LINE      CODE     ---       #1103
      01001EC7H   LINE      CODE     ---       #1104
      01001ECEH   LINE      CODE     ---       #1105
      ---         BLOCKEND  ---      ---       LVL=0
      00000007H   SYMBOL    DATA     BYTE      reg13

      ---         MODULE    ---      ---       UM2006A_HAL
      01001AB6H   PUBLIC    CODE     ---       spi_read_byte
      01001B7BH   PUBLIC    CODE     ---       _spi_write_byte
      01001ED5H   PUBLIC    CODE     ---       spi_cs_disable
      01001F16H   PUBLIC    CODE     ---       spi_cs_enable
      01001BD6H   PUBLIC    CODE     ---       spi_init
      01001E5BH   PUBLIC    CODE     ---       um2006A_hal_init
      0100001CH   PUBLIC    CODE     ---       um2006A_hal_irq
      00000098H.3 SFRSYM    DATA     BIT       TB80
      000000E0H.7 SFRSYM    DATA     BIT       ACC7
      00000080H   SFRSYM    DATA     BYTE      P0
      00000090H   SFRSYM    DATA     BYTE      P1
      000000A0H   SFRSYM    DATA     BYTE      P2
      00000098H.5 SFRSYM    DATA     BIT       SM20
      000000B2H   SFRSYM    DATA     BYTE      ESTCR
      000000B1H   SFRSYM    DATA     BYTE      CLKST
      000000D0H.6 SFRSYM    DATA     BIT       AC
      000000D8H.3 SFRSYM    DATA     BIT       ERSTF
      000000E6H   SFRSYM    DATA     BYTE      PRESET0
      000000D4H   SFRSYM    DATA     BYTE      OCTRL
      000000A8H.7 SFRSYM    DATA     BIT       EA
      0000008FH   SFRSYM    DATA     BYTE      POREN
      000000C8H   SFRSYM    DATA     BYTE      PWM0CON
      000000E7H   SFRSYM    DATA     BYTE      PRESET1
      000000C9H   SFRSYM    DATA     BYTE      PWM1CON
      00000086H   SFRSYM    DATA     BYTE      BEEPCTR
      000000CAH   SFRSYM    DATA     BYTE      PWM2CON
      000000B8H.4 SFRSYM    DATA     BIT       LPTIMINTEN
      000000ABH   SFRSYM    DATA     BYTE      P0AH
      000000B0H   SFRSYM    DATA     BYTE      P1AH
      000000E8H   SFRSYM    DATA     BYTE      P2AH
      000000F8H.6 SFRSYM    DATA     BIT       RC32KF
      000000A8H   SFRSYM    DATA     BYTE      IEN0
      000000A7H   SFRSYM    DATA     BYTE      OPSET
      000000A4H   SFRSYM    DATA     BYTE      P0AL
      000000B8H   SFRSYM    DATA     BYTE      IEN1
      000000A8H.6 SFRSYM    DATA     BIT       EADC
      00000085H   SFRSYM    DATA     BYTE      DPH1
LX51 LINKER/LOCATER V4.66.97.0                                                        06/12/2025  17:35:51  PAGE 47


      000000AEH   SFRSYM    DATA     BYTE      P1AL
      0000009AH   SFRSYM    DATA     BYTE      IEN2
      000000C0H   SFRSYM    DATA     BYTE      P2AL
      000000B6H   SFRSYM    DATA     BYTE      ADCDR0
      000000F8H.5 SFRSYM    DATA     BIT       RC16MF
      000000B7H   SFRSYM    DATA     BYTE      ADCDR1
      00000084H   SFRSYM    DATA     BYTE      DPL1
      000000D6H   SFRSYM    DATA     BYTE      P0OD
      000000DBH   SFRSYM    DATA     BYTE      P1OD
      000000D5H   SFRSYM    DATA     BYTE      P0PD
      00000098H.4 SFRSYM    DATA     BIT       REN0
      000000ECH   SFRSYM    DATA     BYTE      P2OD
      000000DAH   SFRSYM    DATA     BYTE      P1PD
      000000E4H   SFRSYM    DATA     BYTE      P2PD
      000000D7H   SFRSYM    DATA     BYTE      P0CS
      00000097H   SFRSYM    DATA     BYTE      P0DR
      0000009EH   SFRSYM    DATA     BYTE      EUARTEN
      000000DCH   SFRSYM    DATA     BYTE      P1CS
      000000E5H   SFRSYM    DATA     BYTE      P1DR
      000000F4H   SFRSYM    DATA     BYTE      P2CS
      000000FCH   SFRSYM    DATA     BYTE      P2DR
      000000D0H.7 SFRSYM    DATA     BIT       CY
      000000D8H.0 SFRSYM    DATA     BIT       WDT0
      000000D8H.1 SFRSYM    DATA     BIT       WDT1
      000000D8H.2 SFRSYM    DATA     BIT       WDT2
      00000081H   SFRSYM    DATA     BYTE      SP
      000000F1H   SFRSYM    DATA     BYTE      P0PU
      000000F2H   SFRSYM    DATA     BYTE      P1PU
      000000D1H   SFRSYM    DATA     WORD      OADR
      000000F3H   SFRSYM    DATA     BYTE      P2PU
      00000093H   SFRSYM    DATA     BYTE      ADCIER
      000000A5H   SFRSYM    DATA     BYTE      OSEC
      000000D8H.6 SFRSYM    DATA     BIT       WDEN
      000000BAH   SFRSYM    DATA     BYTE      S0RELH
      00000080H.0 SFRSYM    DATA     BIT       P00
      000000D8H.7 SFRSYM    DATA     BIT       WDOF
      000000BBH   SFRSYM    DATA     BYTE      S1RELH
      00000090H.0 SFRSYM    DATA     BIT       P10
      00000080H.1 SFRSYM    DATA     BIT       P01
      00000087H   SFRSYM    DATA     BYTE      PCON
      000000C4H   SFRSYM    DATA     BYTE      PWM0DH
      000000A0H.0 SFRSYM    DATA     BIT       P20
      00000090H.1 SFRSYM    DATA     BIT       P11
      00000080H.2 SFRSYM    DATA     BIT       P02
      000000C6H   SFRSYM    DATA     BYTE      PWM1DH
      00000090H.2 SFRSYM    DATA     BIT       P12
      00000080H.3 SFRSYM    DATA     BIT       P03
      000000C7H   SFRSYM    DATA     BYTE      PWM2DH
      000000C8H.2 SFRSYM    DATA     BIT       PWM0IE
      000000AAH   SFRSYM    DATA     BYTE      S0RELL
      000000A0H.2 SFRSYM    DATA     BIT       P22
      00000090H.3 SFRSYM    DATA     BIT       P13
      00000080H.4 SFRSYM    DATA     BIT       P04
      000000C8H.1 SFRSYM    DATA     BIT       PWM0IF
      0000009DH   SFRSYM    DATA     BYTE      S1RELL
      000000A0H.3 SFRSYM    DATA     BIT       P23
      00000090H.4 SFRSYM    DATA     BIT       P14
      00000080H.5 SFRSYM    DATA     BIT       P05
      000000C3H   SFRSYM    DATA     BYTE      PWM0DL
      00000090H.5 SFRSYM    DATA     BIT       P15
      000000A6H   SFRSYM    DATA     BYTE      OSTATUS
      000000C5H   SFRSYM    DATA     BYTE      PWM1DL
      000000A0H.5 SFRSYM    DATA     BIT       P25
      000000D8H.4 SFRSYM    DATA     BIT       PORF
      000000D8H   SFRSYM    DATA     BYTE      RSTSTAT
LX51 LINKER/LOCATER V4.66.97.0                                                        06/12/2025  17:35:51  PAGE 48


      000000CFH   SFRSYM    DATA     BYTE      PWM2DL
      000000A0H.6 SFRSYM    DATA     BIT       P26
      000000C8H.7 SFRSYM    DATA     BIT       PWM0EN
      000000A0H.7 SFRSYM    DATA     BIT       P27
      000000A8H.5 SFRSYM    DATA     BIT       EPWM
      000000D8H.5 SFRSYM    DATA     BIT       LVRF
      000000F8H   SFRSYM    DATA     BYTE      CLKCON
      000000CCH   SFRSYM    DATA     BYTE      PWM0PH
      000000CEH   SFRSYM    DATA     BYTE      PWM1PH
      000000B8H.5 SFRSYM    DATA     BIT       I2CINTEN
      000000C2H   SFRSYM    DATA     BYTE      PWM2PH
      000000F0H   SFRSYM    DATA     BYTE      B
      000000EEH   SFRSYM    DATA     BYTE      RCHDIV
      000000CBH   SFRSYM    DATA     BYTE      PWM0PL
      000000CDH   SFRSYM    DATA     BYTE      PWM1PL
      000000C1H   SFRSYM    DATA     BYTE      PWM2PL
      000000F7H   SFRSYM    DATA     BYTE      ADCSPW
      000000F8H.1 SFRSYM    DATA     BIT       XCLKEN
      000000E0H   SFRSYM    DATA     BYTE      ACC
      000000DDH   SFRSYM    DATA     BYTE      LVDCON
      000000A8H.4 SFRSYM    DATA     BIT       ES0
      000000A9H   SFRSYM    DATA     BYTE      IP0
      000000A8H.1 SFRSYM    DATA     BIT       ET0
      000000A8H.2 SFRSYM    DATA     BIT       ES1
      000000F6H   SFRSYM    DATA     BYTE      ADCCSTAT
      000000B9H   SFRSYM    DATA     BYTE      IP1
      000000A8H.3 SFRSYM    DATA     BIT       ET1
      00000098H.0 SFRSYM    DATA     BIT       RI0
      000000C8H.0 SFRSYM    DATA     BIT       PWM0SS
      00000098H.1 SFRSYM    DATA     BIT       TI0
      000000A8H.0 SFRSYM    DATA     BIT       EX0
      000000D0H.0 SFRSYM    DATA     BIT       P
      000000B8H.3 SFRSYM    DATA     BIT       EFCINTEN
      000000A2H   SFRSYM    DATA     BYTE      OINTEN
      00000098H.7 SFRSYM    DATA     BIT       SM0
      00000098H.6 SFRSYM    DATA     BIT       SM1
      000000FEH   SFRSYM    DATA     BYTE      ADCCDR0
      000000FFH   SFRSYM    DATA     BYTE      ADCCDR1
      000000D0H.3 SFRSYM    DATA     BIT       RS0
      000000ACH   SFRSYM    DATA     BYTE      ADCGCR0
      000000D0H.4 SFRSYM    DATA     BIT       RS1
      000000ADH   SFRSYM    DATA     BYTE      ADCGCR1
      000000B4H   SFRSYM    DATA     BYTE      ADCGCR2
      000000B5H   SFRSYM    DATA     BYTE      ADCGCR3
      000000F8H.3 SFRSYM    DATA     BIT       RC32KEN
      000000DEH   SFRSYM    DATA     BYTE      PCLK0
      000000DFH   SFRSYM    DATA     BYTE      PCLK1
      00000083H   SFRSYM    DATA     BYTE      DPH
      000000E9H   SFRSYM    DATA     BYTE      P0IEN
      000000F5H   SFRSYM    DATA     BYTE      ADCHL
      000000F8H.2 SFRSYM    DATA     BIT       RC16MEN
      000000EAH   SFRSYM    DATA     BYTE      P1IEN
      000000EBH   SFRSYM    DATA     BYTE      P2IEN
      000000B6H   SFRSYM    DATA     WORD      ADCDR
      000000B3H   SFRSYM    DATA     BYTE      XTHCTR
      00000082H   SFRSYM    DATA     BYTE      DPL
      00000099H   SFRSYM    DATA     BYTE      S0BUF
      0000009CH   SFRSYM    DATA     BYTE      S1BUF
      000000F9H   SFRSYM    DATA     BYTE      P0OEN
      000000B8H.0 SFRSYM    DATA     BIT       GTIM0INTEN
      000000D9H   SFRSYM    DATA     BYTE      SYSDIV
      00000098H   SFRSYM    DATA     BYTE      S0CON
      000000FAH   SFRSYM    DATA     BYTE      P1OEN
      000000B8H.2 SFRSYM    DATA     BIT       GTIM1INTEN
      000000A3H   SFRSYM    DATA     BYTE      OINTUS
LX51 LINKER/LOCATER V4.66.97.0                                                        06/12/2025  17:35:51  PAGE 49


      000000BEH   SFRSYM    DATA     BYTE      RCHTRIMH
      000000F8H.0 SFRSYM    DATA     BIT       SYSSEL
      0000009BH   SFRSYM    DATA     BYTE      S1CON
      000000FBH   SFRSYM    DATA     BYTE      P2OEN
      000000B8H.6 SFRSYM    DATA     BIT       GTIM2INTEN
      000000BDH   SFRSYM    DATA     BYTE      LDOTRIMH
      00000092H   SFRSYM    DATA     BYTE      DPS
      0000009FH   SFRSYM    DATA     BYTE      RCLTRIMH
      000000BFH   SFRSYM    DATA     BYTE      RCHTRIML
      000000D3H   SFRSYM    DATA     BYTE      ODATA
      00000091H   SFRSYM    DATA     BYTE      LDOTRIML
      000000BCH   SFRSYM    DATA     BYTE      RCLTRIML
      000000E1H   SFRSYM    DATA     BYTE      P0IRQ
      000000B8H.1 SFRSYM    DATA     BIT       SPIINTEN
      000000E2H   SFRSYM    DATA     BYTE      P1IRQ
      000000E3H   SFRSYM    DATA     BYTE      P2IRQ
      000000D2H   SFRSYM    DATA     BYTE      OADRH
      000000B8H.7 SFRSYM    DATA     BIT       UART2INTEN
      000000F0H.0 SFRSYM    DATA     BIT       B0
      000000F0H.1 SFRSYM    DATA     BIT       B1
      000000F0H.2 SFRSYM    DATA     BIT       B2
      000000D1H   SFRSYM    DATA     BYTE      OADRL
      000000F0H.3 SFRSYM    DATA     BIT       B3
      000000F0H.4 SFRSYM    DATA     BIT       B4
      000000D0H.5 SFRSYM    DATA     BIT       F0
      000000F0H.5 SFRSYM    DATA     BIT       B5
      000000D0H.1 SFRSYM    DATA     BIT       F1
      000000AFH   SFRSYM    DATA     BYTE      REMAP
      000000F0H.6 SFRSYM    DATA     BIT       B6
      000000E0H.0 SFRSYM    DATA     BIT       ACC0
      000000A1H   SFRSYM    DATA     BYTE      OUS
      000000C8H.6 SFRSYM    DATA     BIT       PWM0S
      000000F0H.7 SFRSYM    DATA     BIT       B7
      000000E0H.1 SFRSYM    DATA     BIT       ACC1
      000000F8H.4 SFRSYM    DATA     BIT       XCLKF
      000000E0H.2 SFRSYM    DATA     BIT       ACC2
      0000008EH   SFRSYM    DATA     BYTE      PDSEL
      000000E0H.3 SFRSYM    DATA     BIT       ACC3
      000000D0H   SFRSYM    DATA     BYTE      PSW
      000000E0H.4 SFRSYM    DATA     BIT       ACC4
      00000098H.2 SFRSYM    DATA     BIT       RB80
      000000E0H.5 SFRSYM    DATA     BIT       ACC5
      000000FDH   SFRSYM    DATA     BYTE      ADCVREF
      000000E0H.6 SFRSYM    DATA     BIT       ACC6
      02000331H   SYMBOL    XDATA    BYTE      g_rxbyte_flag

      0100001CH   BLOCK     CODE     ---       LVL=0
      0100001CH   LINE      CODE     ---       #37
      0100001CH   LINE      CODE     ---       #38
      0100001CH   LINE      CODE     ---       #39
      01000022H   LINE      CODE     ---       #40
      ---         BLOCKEND  ---      ---       LVL=0

      01001E5BH   BLOCK     CODE     ---       LVL=0
      01001E5BH   LINE      CODE     ---       #73
      01001E5BH   LINE      CODE     ---       #74
      01001E5BH   LINE      CODE     ---       #75
      01001E60H   LINE      CODE     ---       #76
      01001E67H   LINE      CODE     ---       #77
      01001E6EH   LINE      CODE     ---       #78
      01001E75H   LINE      CODE     ---       #80
      01001E82H   LINE      CODE     ---       #81
      01001E85H   LINE      CODE     ---       #82
      01001E88H   LINE      CODE     ---       #84
      01001E8AH   LINE      CODE     ---       #85
LX51 LINKER/LOCATER V4.66.97.0                                                        06/12/2025  17:35:51  PAGE 50


      ---         BLOCKEND  ---      ---       LVL=0

      01001BD6H   BLOCK     CODE     ---       LVL=0
      01001BD6H   LINE      CODE     ---       #94
      01001BD6H   LINE      CODE     ---       #95
      01001BD6H   LINE      CODE     ---       #96
      01001BDBH   LINE      CODE     ---       #97
      01001BE0H   LINE      CODE     ---       #99
      01001BE7H   LINE      CODE     ---       #100
      01001BEEH   LINE      CODE     ---       #101
      01001BF5H   LINE      CODE     ---       #103
      01001BFCH   LINE      CODE     ---       #104
      01001C03H   LINE      CODE     ---       #105
      01001C0AH   LINE      CODE     ---       #107
      01001C11H   LINE      CODE     ---       #108
      01001C18H   LINE      CODE     ---       #109
      01001C1FH   LINE      CODE     ---       #110
      ---         BLOCKEND  ---      ---       LVL=0

      01001F16H   BLOCK     CODE     ---       LVL=0
      01001F16H   LINE      CODE     ---       #120
      01001F16H   LINE      CODE     ---       #121
      01001F16H   LINE      CODE     ---       #122
      ---         BLOCKEND  ---      ---       LVL=0

      01001ED5H   BLOCK     CODE     ---       LVL=0
      01001ED5H   LINE      CODE     ---       #132
      01001ED5H   LINE      CODE     ---       #133
      01001ED5H   LINE      CODE     ---       #134
      01001EDCH   LINE      CODE     ---       #135
      ---         BLOCKEND  ---      ---       LVL=0

      01001B7BH   BLOCK     CODE     ---       LVL=0
      0200026AH   SYMBOL    XDATA    BYTE      byte
      01001B80H   BLOCK     CODE     NEAR LAB  LVL=1
      0200026BH   SYMBOL    XDATA    BYTE      i
      ---         BLOCKEND  ---      ---       LVL=1
      01001B7BH   LINE      CODE     ---       #145
      01001B80H   LINE      CODE     ---       #146
      01001B80H   LINE      CODE     ---       #147
      01001B83H   LINE      CODE     ---       #148
      01001B89H   LINE      CODE     ---       #149
      01001B9BH   LINE      CODE     ---       #150
      01001B9BH   LINE      CODE     ---       #151
      01001BA2H   LINE      CODE     ---       #152
      01001BA9H   LINE      CODE     ---       #153
      01001BA9H   LINE      CODE     ---       #154
      01001BABH   LINE      CODE     ---       #155
      01001BADH   LINE      CODE     ---       #157
      01001BADH   LINE      CODE     ---       #158
      01001BB4H   LINE      CODE     ---       #159
      01001BB4H   LINE      CODE     ---       #160
      01001BBBH   LINE      CODE     ---       #161
      01001BC2H   LINE      CODE     ---       #162
      01001BC8H   LINE      CODE     ---       #163
      01001BCFH   LINE      CODE     ---       #164
      ---         BLOCKEND  ---      ---       LVL=0

      01001AB6H   BLOCK     CODE     ---       LVL=0
      01001AB6H   BLOCK     CODE     NEAR LAB  LVL=1
      0200026AH   SYMBOL    XDATA    BYTE      i
      0200026BH   SYMBOL    XDATA    BYTE      value
      ---         BLOCKEND  ---      ---       LVL=1
      01001AB6H   LINE      CODE     ---       #174
      01001AB6H   LINE      CODE     ---       #175
LX51 LINKER/LOCATER V4.66.97.0                                                        06/12/2025  17:35:51  PAGE 51


      01001AB6H   LINE      CODE     ---       #176
      01001ABBH   LINE      CODE     ---       #177
      01001ABDH   LINE      CODE     ---       #178
      01001AC4H   LINE      CODE     ---       #179
      01001AD6H   LINE      CODE     ---       #180
      01001AD6H   LINE      CODE     ---       #181
      01001ADBH   LINE      CODE     ---       #182
      01001AE2H   LINE      CODE     ---       #183
      01001AEAH   LINE      CODE     ---       #184
      01001AEAH   LINE      CODE     ---       #185
      01001AF0H   LINE      CODE     ---       #186
      01001AF0H   LINE      CODE     ---       #188
      01001AF7H   LINE      CODE     ---       #189
      01001AFFH   LINE      CODE     ---       #190
      01001B06H   LINE      CODE     ---       #191
      01001B0DH   LINE      CODE     ---       #192
      01001B14H   LINE      CODE     ---       #193
      01001B19H   LINE      CODE     ---       #194
      ---         BLOCKEND  ---      ---       LVL=0

      ---         MODULE    ---      ---       MAIN
      01001EFAH   PUBLIC    CODE     ---       main
      00000098H.3 SFRSYM    DATA     BIT       TB80
      000000E0H.7 SFRSYM    DATA     BIT       ACC7
      00000080H   SFRSYM    DATA     BYTE      P0
      00000090H   SFRSYM    DATA     BYTE      P1
      000000A0H   SFRSYM    DATA     BYTE      P2
      00000098H.5 SFRSYM    DATA     BIT       SM20
      000000B2H   SFRSYM    DATA     BYTE      ESTCR
      000000B1H   SFRSYM    DATA     BYTE      CLKST
      000000D0H.6 SFRSYM    DATA     BIT       AC
      000000D8H.3 SFRSYM    DATA     BIT       ERSTF
      000000E6H   SFRSYM    DATA     BYTE      PRESET0
      000000D4H   SFRSYM    DATA     BYTE      OCTRL
      000000A8H.7 SFRSYM    DATA     BIT       EA
      0000008FH   SFRSYM    DATA     BYTE      POREN
      000000C8H   SFRSYM    DATA     BYTE      PWM0CON
      000000E7H   SFRSYM    DATA     BYTE      PRESET1
      000000C9H   SFRSYM    DATA     BYTE      PWM1CON
      00000086H   SFRSYM    DATA     BYTE      BEEPCTR
      000000CAH   SFRSYM    DATA     BYTE      PWM2CON
      000000B8H.4 SFRSYM    DATA     BIT       LPTIMINTEN
      000000ABH   SFRSYM    DATA     BYTE      P0AH
      000000B0H   SFRSYM    DATA     BYTE      P1AH
      000000E8H   SFRSYM    DATA     BYTE      P2AH
      000000F8H.6 SFRSYM    DATA     BIT       RC32KF
      000000A8H   SFRSYM    DATA     BYTE      IEN0
      000000A7H   SFRSYM    DATA     BYTE      OPSET
      000000A4H   SFRSYM    DATA     BYTE      P0AL
      000000B8H   SFRSYM    DATA     BYTE      IEN1
      000000A8H.6 SFRSYM    DATA     BIT       EADC
      00000085H   SFRSYM    DATA     BYTE      DPH1
      000000AEH   SFRSYM    DATA     BYTE      P1AL
      0000009AH   SFRSYM    DATA     BYTE      IEN2
      000000C0H   SFRSYM    DATA     BYTE      P2AL
      000000B6H   SFRSYM    DATA     BYTE      ADCDR0
      000000F8H.5 SFRSYM    DATA     BIT       RC16MF
      000000B7H   SFRSYM    DATA     BYTE      ADCDR1
      00000084H   SFRSYM    DATA     BYTE      DPL1
      000000D6H   SFRSYM    DATA     BYTE      P0OD
      000000DBH   SFRSYM    DATA     BYTE      P1OD
      000000D5H   SFRSYM    DATA     BYTE      P0PD
      00000098H.4 SFRSYM    DATA     BIT       REN0
      000000ECH   SFRSYM    DATA     BYTE      P2OD
      000000DAH   SFRSYM    DATA     BYTE      P1PD
LX51 LINKER/LOCATER V4.66.97.0                                                        06/12/2025  17:35:51  PAGE 52


      000000E4H   SFRSYM    DATA     BYTE      P2PD
      000000D7H   SFRSYM    DATA     BYTE      P0CS
      00000097H   SFRSYM    DATA     BYTE      P0DR
      0000009EH   SFRSYM    DATA     BYTE      EUARTEN
      000000DCH   SFRSYM    DATA     BYTE      P1CS
      000000E5H   SFRSYM    DATA     BYTE      P1DR
      000000F4H   SFRSYM    DATA     BYTE      P2CS
      000000FCH   SFRSYM    DATA     BYTE      P2DR
      000000D0H.7 SFRSYM    DATA     BIT       CY
      000000D8H.0 SFRSYM    DATA     BIT       WDT0
      000000D8H.1 SFRSYM    DATA     BIT       WDT1
      000000D8H.2 SFRSYM    DATA     BIT       WDT2
      00000081H   SFRSYM    DATA     BYTE      SP
      000000F1H   SFRSYM    DATA     BYTE      P0PU
      000000F2H   SFRSYM    DATA     BYTE      P1PU
      000000D1H   SFRSYM    DATA     WORD      OADR
      000000F3H   SFRSYM    DATA     BYTE      P2PU
      00000093H   SFRSYM    DATA     BYTE      ADCIER
      000000A5H   SFRSYM    DATA     BYTE      OSEC
      000000D8H.6 SFRSYM    DATA     BIT       WDEN
      000000BAH   SFRSYM    DATA     BYTE      S0RELH
      00000080H.0 SFRSYM    DATA     BIT       P00
      000000D8H.7 SFRSYM    DATA     BIT       WDOF
      000000BBH   SFRSYM    DATA     BYTE      S1RELH
      00000090H.0 SFRSYM    DATA     BIT       P10
      00000080H.1 SFRSYM    DATA     BIT       P01
      00000087H   SFRSYM    DATA     BYTE      PCON
      000000C4H   SFRSYM    DATA     BYTE      PWM0DH
      000000A0H.0 SFRSYM    DATA     BIT       P20
      00000090H.1 SFRSYM    DATA     BIT       P11
      00000080H.2 SFRSYM    DATA     BIT       P02
      000000C6H   SFRSYM    DATA     BYTE      PWM1DH
      00000090H.2 SFRSYM    DATA     BIT       P12
      00000080H.3 SFRSYM    DATA     BIT       P03
      000000C7H   SFRSYM    DATA     BYTE      PWM2DH
      000000C8H.2 SFRSYM    DATA     BIT       PWM0IE
      000000AAH   SFRSYM    DATA     BYTE      S0RELL
      000000A0H.2 SFRSYM    DATA     BIT       P22
      00000090H.3 SFRSYM    DATA     BIT       P13
      00000080H.4 SFRSYM    DATA     BIT       P04
      000000C8H.1 SFRSYM    DATA     BIT       PWM0IF
      0000009DH   SFRSYM    DATA     BYTE      S1RELL
      000000A0H.3 SFRSYM    DATA     BIT       P23
      00000090H.4 SFRSYM    DATA     BIT       P14
      00000080H.5 SFRSYM    DATA     BIT       P05
      000000C3H   SFRSYM    DATA     BYTE      PWM0DL
      00000090H.5 SFRSYM    DATA     BIT       P15
      000000A6H   SFRSYM    DATA     BYTE      OSTATUS
      000000C5H   SFRSYM    DATA     BYTE      PWM1DL
      000000A0H.5 SFRSYM    DATA     BIT       P25
      000000D8H.4 SFRSYM    DATA     BIT       PORF
      000000D8H   SFRSYM    DATA     BYTE      RSTSTAT
      000000CFH   SFRSYM    DATA     BYTE      PWM2DL
      000000A0H.6 SFRSYM    DATA     BIT       P26
      000000C8H.7 SFRSYM    DATA     BIT       PWM0EN
      000000A0H.7 SFRSYM    DATA     BIT       P27
      000000A8H.5 SFRSYM    DATA     BIT       EPWM
      000000D8H.5 SFRSYM    DATA     BIT       LVRF
      000000F8H   SFRSYM    DATA     BYTE      CLKCON
      000000CCH   SFRSYM    DATA     BYTE      PWM0PH
      000000CEH   SFRSYM    DATA     BYTE      PWM1PH
      000000B8H.5 SFRSYM    DATA     BIT       I2CINTEN
      000000C2H   SFRSYM    DATA     BYTE      PWM2PH
      000000F0H   SFRSYM    DATA     BYTE      B
      000000EEH   SFRSYM    DATA     BYTE      RCHDIV
LX51 LINKER/LOCATER V4.66.97.0                                                        06/12/2025  17:35:51  PAGE 53


      000000CBH   SFRSYM    DATA     BYTE      PWM0PL
      000000CDH   SFRSYM    DATA     BYTE      PWM1PL
      000000C1H   SFRSYM    DATA     BYTE      PWM2PL
      000000F7H   SFRSYM    DATA     BYTE      ADCSPW
      000000F8H.1 SFRSYM    DATA     BIT       XCLKEN
      000000E0H   SFRSYM    DATA     BYTE      ACC
      000000DDH   SFRSYM    DATA     BYTE      LVDCON
      000000A8H.4 SFRSYM    DATA     BIT       ES0
      000000A9H   SFRSYM    DATA     BYTE      IP0
      000000A8H.1 SFRSYM    DATA     BIT       ET0
      000000A8H.2 SFRSYM    DATA     BIT       ES1
      000000F6H   SFRSYM    DATA     BYTE      ADCCSTAT
      000000B9H   SFRSYM    DATA     BYTE      IP1
      000000A8H.3 SFRSYM    DATA     BIT       ET1
      00000098H.0 SFRSYM    DATA     BIT       RI0
      000000C8H.0 SFRSYM    DATA     BIT       PWM0SS
      00000098H.1 SFRSYM    DATA     BIT       TI0
      000000A8H.0 SFRSYM    DATA     BIT       EX0
      000000D0H.0 SFRSYM    DATA     BIT       P
      000000B8H.3 SFRSYM    DATA     BIT       EFCINTEN
      000000A2H   SFRSYM    DATA     BYTE      OINTEN
      00000098H.7 SFRSYM    DATA     BIT       SM0
      00000098H.6 SFRSYM    DATA     BIT       SM1
      000000FEH   SFRSYM    DATA     BYTE      ADCCDR0
      000000FFH   SFRSYM    DATA     BYTE      ADCCDR1
      000000D0H.3 SFRSYM    DATA     BIT       RS0
      000000ACH   SFRSYM    DATA     BYTE      ADCGCR0
      000000D0H.4 SFRSYM    DATA     BIT       RS1
      000000ADH   SFRSYM    DATA     BYTE      ADCGCR1
      000000B4H   SFRSYM    DATA     BYTE      ADCGCR2
      000000B5H   SFRSYM    DATA     BYTE      ADCGCR3
      000000F8H.3 SFRSYM    DATA     BIT       RC32KEN
      000000DEH   SFRSYM    DATA     BYTE      PCLK0
      000000DFH   SFRSYM    DATA     BYTE      PCLK1
      00000083H   SFRSYM    DATA     BYTE      DPH
      000000E9H   SFRSYM    DATA     BYTE      P0IEN
      000000F5H   SFRSYM    DATA     BYTE      ADCHL
      000000F8H.2 SFRSYM    DATA     BIT       RC16MEN
      000000EAH   SFRSYM    DATA     BYTE      P1IEN
      000000EBH   SFRSYM    DATA     BYTE      P2IEN
      000000B6H   SFRSYM    DATA     WORD      ADCDR
      000000B3H   SFRSYM    DATA     BYTE      XTHCTR
      00000082H   SFRSYM    DATA     BYTE      DPL
      00000099H   SFRSYM    DATA     BYTE      S0BUF
      0000009CH   SFRSYM    DATA     BYTE      S1BUF
      000000F9H   SFRSYM    DATA     BYTE      P0OEN
      000000B8H.0 SFRSYM    DATA     BIT       GTIM0INTEN
      000000D9H   SFRSYM    DATA     BYTE      SYSDIV
      00000098H   SFRSYM    DATA     BYTE      S0CON
      000000FAH   SFRSYM    DATA     BYTE      P1OEN
      000000B8H.2 SFRSYM    DATA     BIT       GTIM1INTEN
      000000A3H   SFRSYM    DATA     BYTE      OINTUS
      000000BEH   SFRSYM    DATA     BYTE      RCHTRIMH
      000000F8H.0 SFRSYM    DATA     BIT       SYSSEL
      0000009BH   SFRSYM    DATA     BYTE      S1CON
      000000FBH   SFRSYM    DATA     BYTE      P2OEN
      000000B8H.6 SFRSYM    DATA     BIT       GTIM2INTEN
      000000BDH   SFRSYM    DATA     BYTE      LDOTRIMH
      00000092H   SFRSYM    DATA     BYTE      DPS
      0000009FH   SFRSYM    DATA     BYTE      RCLTRIMH
      000000BFH   SFRSYM    DATA     BYTE      RCHTRIML
      000000D3H   SFRSYM    DATA     BYTE      ODATA
      00000091H   SFRSYM    DATA     BYTE      LDOTRIML
      000000BCH   SFRSYM    DATA     BYTE      RCLTRIML
      000000E1H   SFRSYM    DATA     BYTE      P0IRQ
LX51 LINKER/LOCATER V4.66.97.0                                                        06/12/2025  17:35:51  PAGE 54


      000000B8H.1 SFRSYM    DATA     BIT       SPIINTEN
      000000E2H   SFRSYM    DATA     BYTE      P1IRQ
      000000E3H   SFRSYM    DATA     BYTE      P2IRQ
      000000D2H   SFRSYM    DATA     BYTE      OADRH
      000000B8H.7 SFRSYM    DATA     BIT       UART2INTEN
      000000F0H.0 SFRSYM    DATA     BIT       B0
      000000F0H.1 SFRSYM    DATA     BIT       B1
      000000F0H.2 SFRSYM    DATA     BIT       B2
      000000D1H   SFRSYM    DATA     BYTE      OADRL
      000000F0H.3 SFRSYM    DATA     BIT       B3
      000000F0H.4 SFRSYM    DATA     BIT       B4
      000000D0H.5 SFRSYM    DATA     BIT       F0
      000000F0H.5 SFRSYM    DATA     BIT       B5
      000000D0H.1 SFRSYM    DATA     BIT       F1
      000000AFH   SFRSYM    DATA     BYTE      REMAP
      000000F0H.6 SFRSYM    DATA     BIT       B6
      000000E0H.0 SFRSYM    DATA     BIT       ACC0
      000000A1H   SFRSYM    DATA     BYTE      OUS
      000000C8H.6 SFRSYM    DATA     BIT       PWM0S
      000000F0H.7 SFRSYM    DATA     BIT       B7
      000000E0H.1 SFRSYM    DATA     BIT       ACC1
      000000F8H.4 SFRSYM    DATA     BIT       XCLKF
      000000E0H.2 SFRSYM    DATA     BIT       ACC2
      0000008EH   SFRSYM    DATA     BYTE      PDSEL
      000000E0H.3 SFRSYM    DATA     BIT       ACC3
      000000D0H   SFRSYM    DATA     BYTE      PSW
      000000E0H.4 SFRSYM    DATA     BIT       ACC4
      00000098H.2 SFRSYM    DATA     BIT       RB80
      000000E0H.5 SFRSYM    DATA     BIT       ACC5
      000000FDH   SFRSYM    DATA     BYTE      ADCVREF
      000000E0H.6 SFRSYM    DATA     BIT       ACC6

      01001EFAH   BLOCK     CODE     ---       LVL=0
      01001EFAH   LINE      CODE     ---       #20
      01001EFAH   LINE      CODE     ---       #21
      01001EFAH   LINE      CODE     ---       #22
      01001EFDH   LINE      CODE     ---       #23
      01001F00H   LINE      CODE     ---       #24
      01001F00H   LINE      CODE     ---       #25
      01001F00H   LINE      CODE     ---       #26
      01001F03H   LINE      CODE     ---       #27
      ---         BLOCKEND  ---      ---       LVL=0

      ---         MODULE    ---      ---       APP
      01001F22H   PUBLIC    CODE     ---       app_run
      01001B1AH   PUBLIC    CODE     ---       app_init
      00000098H.3 SFRSYM    DATA     BIT       TB80
      000000E0H.7 SFRSYM    DATA     BIT       ACC7
      00000080H   SFRSYM    DATA     BYTE      P0
      00000090H   SFRSYM    DATA     BYTE      P1
      000000A0H   SFRSYM    DATA     BYTE      P2
      00000098H.5 SFRSYM    DATA     BIT       SM20
      000000B2H   SFRSYM    DATA     BYTE      ESTCR
      000000B1H   SFRSYM    DATA     BYTE      CLKST
      000000D0H.6 SFRSYM    DATA     BIT       AC
      000000D8H.3 SFRSYM    DATA     BIT       ERSTF
      000000E6H   SFRSYM    DATA     BYTE      PRESET0
      000000D4H   SFRSYM    DATA     BYTE      OCTRL
      000000A8H.7 SFRSYM    DATA     BIT       EA
      0000008FH   SFRSYM    DATA     BYTE      POREN
      000000C8H   SFRSYM    DATA     BYTE      PWM0CON
      000000E7H   SFRSYM    DATA     BYTE      PRESET1
      000000C9H   SFRSYM    DATA     BYTE      PWM1CON
      00000086H   SFRSYM    DATA     BYTE      BEEPCTR
      000000CAH   SFRSYM    DATA     BYTE      PWM2CON
LX51 LINKER/LOCATER V4.66.97.0                                                        06/12/2025  17:35:51  PAGE 55


      000000B8H.4 SFRSYM    DATA     BIT       LPTIMINTEN
      000000ABH   SFRSYM    DATA     BYTE      P0AH
      000000B0H   SFRSYM    DATA     BYTE      P1AH
      000000E8H   SFRSYM    DATA     BYTE      P2AH
      000000F8H.6 SFRSYM    DATA     BIT       RC32KF
      000000A8H   SFRSYM    DATA     BYTE      IEN0
      000000A7H   SFRSYM    DATA     BYTE      OPSET
      000000A4H   SFRSYM    DATA     BYTE      P0AL
      000000B8H   SFRSYM    DATA     BYTE      IEN1
      000000A8H.6 SFRSYM    DATA     BIT       EADC
      00000085H   SFRSYM    DATA     BYTE      DPH1
      000000AEH   SFRSYM    DATA     BYTE      P1AL
      0000009AH   SFRSYM    DATA     BYTE      IEN2
      000000C0H   SFRSYM    DATA     BYTE      P2AL
      000000B6H   SFRSYM    DATA     BYTE      ADCDR0
      000000F8H.5 SFRSYM    DATA     BIT       RC16MF
      000000B7H   SFRSYM    DATA     BYTE      ADCDR1
      00000084H   SFRSYM    DATA     BYTE      DPL1
      000000D6H   SFRSYM    DATA     BYTE      P0OD
      000000DBH   SFRSYM    DATA     BYTE      P1OD
      000000D5H   SFRSYM    DATA     BYTE      P0PD
      00000098H.4 SFRSYM    DATA     BIT       REN0
      000000ECH   SFRSYM    DATA     BYTE      P2OD
      000000DAH   SFRSYM    DATA     BYTE      P1PD
      000000E4H   SFRSYM    DATA     BYTE      P2PD
      000000D7H   SFRSYM    DATA     BYTE      P0CS
      00000097H   SFRSYM    DATA     BYTE      P0DR
      0000009EH   SFRSYM    DATA     BYTE      EUARTEN
      000000DCH   SFRSYM    DATA     BYTE      P1CS
      000000E5H   SFRSYM    DATA     BYTE      P1DR
      000000F4H   SFRSYM    DATA     BYTE      P2CS
      000000FCH   SFRSYM    DATA     BYTE      P2DR
      000000D0H.7 SFRSYM    DATA     BIT       CY
      000000D8H.0 SFRSYM    DATA     BIT       WDT0
      000000D8H.1 SFRSYM    DATA     BIT       WDT1
      000000D8H.2 SFRSYM    DATA     BIT       WDT2
      00000081H   SFRSYM    DATA     BYTE      SP
      000000F1H   SFRSYM    DATA     BYTE      P0PU
      000000F2H   SFRSYM    DATA     BYTE      P1PU
      000000D1H   SFRSYM    DATA     WORD      OADR
      000000F3H   SFRSYM    DATA     BYTE      P2PU
      00000093H   SFRSYM    DATA     BYTE      ADCIER
      000000A5H   SFRSYM    DATA     BYTE      OSEC
      000000D8H.6 SFRSYM    DATA     BIT       WDEN
      000000BAH   SFRSYM    DATA     BYTE      S0RELH
      00000080H.0 SFRSYM    DATA     BIT       P00
      000000D8H.7 SFRSYM    DATA     BIT       WDOF
      000000BBH   SFRSYM    DATA     BYTE      S1RELH
      00000090H.0 SFRSYM    DATA     BIT       P10
      00000080H.1 SFRSYM    DATA     BIT       P01
      00000087H   SFRSYM    DATA     BYTE      PCON
      000000C4H   SFRSYM    DATA     BYTE      PWM0DH
      000000A0H.0 SFRSYM    DATA     BIT       P20
      00000090H.1 SFRSYM    DATA     BIT       P11
      00000080H.2 SFRSYM    DATA     BIT       P02
      000000C6H   SFRSYM    DATA     BYTE      PWM1DH
      00000090H.2 SFRSYM    DATA     BIT       P12
      00000080H.3 SFRSYM    DATA     BIT       P03
      000000C7H   SFRSYM    DATA     BYTE      PWM2DH
      000000C8H.2 SFRSYM    DATA     BIT       PWM0IE
      000000AAH   SFRSYM    DATA     BYTE      S0RELL
      000000A0H.2 SFRSYM    DATA     BIT       P22
      00000090H.3 SFRSYM    DATA     BIT       P13
      00000080H.4 SFRSYM    DATA     BIT       P04
      000000C8H.1 SFRSYM    DATA     BIT       PWM0IF
LX51 LINKER/LOCATER V4.66.97.0                                                        06/12/2025  17:35:51  PAGE 56


      0000009DH   SFRSYM    DATA     BYTE      S1RELL
      000000A0H.3 SFRSYM    DATA     BIT       P23
      00000090H.4 SFRSYM    DATA     BIT       P14
      00000080H.5 SFRSYM    DATA     BIT       P05
      000000C3H   SFRSYM    DATA     BYTE      PWM0DL
      00000090H.5 SFRSYM    DATA     BIT       P15
      000000A6H   SFRSYM    DATA     BYTE      OSTATUS
      000000C5H   SFRSYM    DATA     BYTE      PWM1DL
      000000A0H.5 SFRSYM    DATA     BIT       P25
      000000D8H.4 SFRSYM    DATA     BIT       PORF
      000000D8H   SFRSYM    DATA     BYTE      RSTSTAT
      000000CFH   SFRSYM    DATA     BYTE      PWM2DL
      000000A0H.6 SFRSYM    DATA     BIT       P26
      000000C8H.7 SFRSYM    DATA     BIT       PWM0EN
      000000A0H.7 SFRSYM    DATA     BIT       P27
      000000A8H.5 SFRSYM    DATA     BIT       EPWM
      000000D8H.5 SFRSYM    DATA     BIT       LVRF
      000000F8H   SFRSYM    DATA     BYTE      CLKCON
      000000CCH   SFRSYM    DATA     BYTE      PWM0PH
      000000CEH   SFRSYM    DATA     BYTE      PWM1PH
      000000B8H.5 SFRSYM    DATA     BIT       I2CINTEN
      000000C2H   SFRSYM    DATA     BYTE      PWM2PH
      000000F0H   SFRSYM    DATA     BYTE      B
      000000EEH   SFRSYM    DATA     BYTE      RCHDIV
      000000CBH   SFRSYM    DATA     BYTE      PWM0PL
      000000CDH   SFRSYM    DATA     BYTE      PWM1PL
      000000C1H   SFRSYM    DATA     BYTE      PWM2PL
      000000F7H   SFRSYM    DATA     BYTE      ADCSPW
      000000F8H.1 SFRSYM    DATA     BIT       XCLKEN
      000000E0H   SFRSYM    DATA     BYTE      ACC
      000000DDH   SFRSYM    DATA     BYTE      LVDCON
      000000A8H.4 SFRSYM    DATA     BIT       ES0
      000000A9H   SFRSYM    DATA     BYTE      IP0
      000000A8H.1 SFRSYM    DATA     BIT       ET0
      000000A8H.2 SFRSYM    DATA     BIT       ES1
      000000F6H   SFRSYM    DATA     BYTE      ADCCSTAT
      000000B9H   SFRSYM    DATA     BYTE      IP1
      000000A8H.3 SFRSYM    DATA     BIT       ET1
      00000098H.0 SFRSYM    DATA     BIT       RI0
      000000C8H.0 SFRSYM    DATA     BIT       PWM0SS
      00000098H.1 SFRSYM    DATA     BIT       TI0
      000000A8H.0 SFRSYM    DATA     BIT       EX0
      000000D0H.0 SFRSYM    DATA     BIT       P
      000000B8H.3 SFRSYM    DATA     BIT       EFCINTEN
      000000A2H   SFRSYM    DATA     BYTE      OINTEN
      00000098H.7 SFRSYM    DATA     BIT       SM0
      00000098H.6 SFRSYM    DATA     BIT       SM1
      000000FEH   SFRSYM    DATA     BYTE      ADCCDR0
      000000FFH   SFRSYM    DATA     BYTE      ADCCDR1
      000000D0H.3 SFRSYM    DATA     BIT       RS0
      000000ACH   SFRSYM    DATA     BYTE      ADCGCR0
      000000D0H.4 SFRSYM    DATA     BIT       RS1
      000000ADH   SFRSYM    DATA     BYTE      ADCGCR1
      000000B4H   SFRSYM    DATA     BYTE      ADCGCR2
      000000B5H   SFRSYM    DATA     BYTE      ADCGCR3
      000000F8H.3 SFRSYM    DATA     BIT       RC32KEN
      000000DEH   SFRSYM    DATA     BYTE      PCLK0
      000000DFH   SFRSYM    DATA     BYTE      PCLK1
      00000083H   SFRSYM    DATA     BYTE      DPH
      000000E9H   SFRSYM    DATA     BYTE      P0IEN
      000000F5H   SFRSYM    DATA     BYTE      ADCHL
      000000F8H.2 SFRSYM    DATA     BIT       RC16MEN
      000000EAH   SFRSYM    DATA     BYTE      P1IEN
      000000EBH   SFRSYM    DATA     BYTE      P2IEN
      000000B6H   SFRSYM    DATA     WORD      ADCDR
LX51 LINKER/LOCATER V4.66.97.0                                                        06/12/2025  17:35:51  PAGE 57


      000000B3H   SFRSYM    DATA     BYTE      XTHCTR
      00000082H   SFRSYM    DATA     BYTE      DPL
      00000099H   SFRSYM    DATA     BYTE      S0BUF
      0000009CH   SFRSYM    DATA     BYTE      S1BUF
      000000F9H   SFRSYM    DATA     BYTE      P0OEN
      000000B8H.0 SFRSYM    DATA     BIT       GTIM0INTEN
      000000D9H   SFRSYM    DATA     BYTE      SYSDIV
      00000098H   SFRSYM    DATA     BYTE      S0CON
      000000FAH   SFRSYM    DATA     BYTE      P1OEN
      000000B8H.2 SFRSYM    DATA     BIT       GTIM1INTEN
      000000A3H   SFRSYM    DATA     BYTE      OINTUS
      000000BEH   SFRSYM    DATA     BYTE      RCHTRIMH
      000000F8H.0 SFRSYM    DATA     BIT       SYSSEL
      0000009BH   SFRSYM    DATA     BYTE      S1CON
      000000FBH   SFRSYM    DATA     BYTE      P2OEN
      000000B8H.6 SFRSYM    DATA     BIT       GTIM2INTEN
      000000BDH   SFRSYM    DATA     BYTE      LDOTRIMH
      00000092H   SFRSYM    DATA     BYTE      DPS
      0000009FH   SFRSYM    DATA     BYTE      RCLTRIMH
      000000BFH   SFRSYM    DATA     BYTE      RCHTRIML
      000000D3H   SFRSYM    DATA     BYTE      ODATA
      00000091H   SFRSYM    DATA     BYTE      LDOTRIML
      000000BCH   SFRSYM    DATA     BYTE      RCLTRIML
      000000E1H   SFRSYM    DATA     BYTE      P0IRQ
      000000B8H.1 SFRSYM    DATA     BIT       SPIINTEN
      000000E2H   SFRSYM    DATA     BYTE      P1IRQ
      000000E3H   SFRSYM    DATA     BYTE      P2IRQ
      000000D2H   SFRSYM    DATA     BYTE      OADRH
      000000B8H.7 SFRSYM    DATA     BIT       UART2INTEN
      000000F0H.0 SFRSYM    DATA     BIT       B0
      000000F0H.1 SFRSYM    DATA     BIT       B1
      000000F0H.2 SFRSYM    DATA     BIT       B2
      000000D1H   SFRSYM    DATA     BYTE      OADRL
      000000F0H.3 SFRSYM    DATA     BIT       B3
      000000F0H.4 SFRSYM    DATA     BIT       B4
      000000D0H.5 SFRSYM    DATA     BIT       F0
      000000F0H.5 SFRSYM    DATA     BIT       B5
      000000D0H.1 SFRSYM    DATA     BIT       F1
      000000AFH   SFRSYM    DATA     BYTE      REMAP
      000000F0H.6 SFRSYM    DATA     BIT       B6
      000000E0H.0 SFRSYM    DATA     BIT       ACC0
      000000A1H   SFRSYM    DATA     BYTE      OUS
      000000C8H.6 SFRSYM    DATA     BIT       PWM0S
      000000F0H.7 SFRSYM    DATA     BIT       B7
      000000E0H.1 SFRSYM    DATA     BIT       ACC1
      000000F8H.4 SFRSYM    DATA     BIT       XCLKF
      000000E0H.2 SFRSYM    DATA     BIT       ACC2
      0000008EH   SFRSYM    DATA     BYTE      PDSEL
      000000E0H.3 SFRSYM    DATA     BIT       ACC3
      000000D0H   SFRSYM    DATA     BYTE      PSW
      000000E0H.4 SFRSYM    DATA     BIT       ACC4
      00000098H.2 SFRSYM    DATA     BIT       RB80
      000000E0H.5 SFRSYM    DATA     BIT       ACC5
      000000FDH   SFRSYM    DATA     BYTE      ADCVREF
      000000E0H.6 SFRSYM    DATA     BIT       ACC6

      01001B1AH   BLOCK     CODE     ---       LVL=0
      01001B1AH   LINE      CODE     ---       #21
      01001B1AH   LINE      CODE     ---       #22
      01001B1AH   LINE      CODE     ---       #23
      01001B25H   LINE      CODE     ---       #24
      01001B2EH   LINE      CODE     ---       #25
      01001B37H   LINE      CODE     ---       #26
      01001B40H   LINE      CODE     ---       #27
      01001B53H   LINE      CODE     ---       #28
LX51 LINKER/LOCATER V4.66.97.0                                                        06/12/2025  17:35:51  PAGE 58


      01001B66H   LINE      CODE     ---       #29
      01001B6FH   LINE      CODE     ---       #30
      01001B78H   LINE      CODE     ---       #32
      ---         BLOCKEND  ---      ---       LVL=0

      01001F22H   BLOCK     CODE     ---       LVL=0
      01001F22H   LINE      CODE     ---       #42
      01001F22H   LINE      CODE     ---       #43
      01001F22H   LINE      CODE     ---       #44
      ---         BLOCKEND  ---      ---       LVL=0

      ---         MODULE    ---      ---       APP_UM2006A
      01001957H   PUBLIC    CODE     ---       app_um2006A_run
      0100005DH   PUBLIC    CODE     ---       app_um2006A_init
      00000098H.3 SFRSYM    DATA     BIT       TB80
      000000E0H.7 SFRSYM    DATA     BIT       ACC7
      00000080H   SFRSYM    DATA     BYTE      P0
      00000090H   SFRSYM    DATA     BYTE      P1
      000000A0H   SFRSYM    DATA     BYTE      P2
      00000098H.5 SFRSYM    DATA     BIT       SM20
      000000B2H   SFRSYM    DATA     BYTE      ESTCR
      000000B1H   SFRSYM    DATA     BYTE      CLKST
      000000D0H.6 SFRSYM    DATA     BIT       AC
      000000D8H.3 SFRSYM    DATA     BIT       ERSTF
      000000E6H   SFRSYM    DATA     BYTE      PRESET0
      000000D4H   SFRSYM    DATA     BYTE      OCTRL
      000000A8H.7 SFRSYM    DATA     BIT       EA
      0000008FH   SFRSYM    DATA     BYTE      POREN
      000000C8H   SFRSYM    DATA     BYTE      PWM0CON
      000000E7H   SFRSYM    DATA     BYTE      PRESET1
      000000C9H   SFRSYM    DATA     BYTE      PWM1CON
      00000086H   SFRSYM    DATA     BYTE      BEEPCTR
      000000CAH   SFRSYM    DATA     BYTE      PWM2CON
      000000B8H.4 SFRSYM    DATA     BIT       LPTIMINTEN
      000000ABH   SFRSYM    DATA     BYTE      P0AH
      000000B0H   SFRSYM    DATA     BYTE      P1AH
      000000E8H   SFRSYM    DATA     BYTE      P2AH
      000000F8H.6 SFRSYM    DATA     BIT       RC32KF
      000000A8H   SFRSYM    DATA     BYTE      IEN0
      000000A7H   SFRSYM    DATA     BYTE      OPSET
      000000A4H   SFRSYM    DATA     BYTE      P0AL
      000000B8H   SFRSYM    DATA     BYTE      IEN1
      000000A8H.6 SFRSYM    DATA     BIT       EADC
      00000085H   SFRSYM    DATA     BYTE      DPH1
      000000AEH   SFRSYM    DATA     BYTE      P1AL
      0000009AH   SFRSYM    DATA     BYTE      IEN2
      000000C0H   SFRSYM    DATA     BYTE      P2AL
      000000B6H   SFRSYM    DATA     BYTE      ADCDR0
      000000F8H.5 SFRSYM    DATA     BIT       RC16MF
      000000B7H   SFRSYM    DATA     BYTE      ADCDR1
      00000084H   SFRSYM    DATA     BYTE      DPL1
      000000D6H   SFRSYM    DATA     BYTE      P0OD
      000000DBH   SFRSYM    DATA     BYTE      P1OD
      000000D5H   SFRSYM    DATA     BYTE      P0PD
      00000098H.4 SFRSYM    DATA     BIT       REN0
      000000ECH   SFRSYM    DATA     BYTE      P2OD
      000000DAH   SFRSYM    DATA     BYTE      P1PD
      000000E4H   SFRSYM    DATA     BYTE      P2PD
      000000D7H   SFRSYM    DATA     BYTE      P0CS
      00000097H   SFRSYM    DATA     BYTE      P0DR
      0000009EH   SFRSYM    DATA     BYTE      EUARTEN
      000000DCH   SFRSYM    DATA     BYTE      P1CS
      000000E5H   SFRSYM    DATA     BYTE      P1DR
      000000F4H   SFRSYM    DATA     BYTE      P2CS
      000000FCH   SFRSYM    DATA     BYTE      P2DR
LX51 LINKER/LOCATER V4.66.97.0                                                        06/12/2025  17:35:51  PAGE 59


      000000D0H.7 SFRSYM    DATA     BIT       CY
      000000D8H.0 SFRSYM    DATA     BIT       WDT0
      000000D8H.1 SFRSYM    DATA     BIT       WDT1
      000000D8H.2 SFRSYM    DATA     BIT       WDT2
      00000081H   SFRSYM    DATA     BYTE      SP
      000000F1H   SFRSYM    DATA     BYTE      P0PU
      000000F2H   SFRSYM    DATA     BYTE      P1PU
      000000D1H   SFRSYM    DATA     WORD      OADR
      000000F3H   SFRSYM    DATA     BYTE      P2PU
      00000093H   SFRSYM    DATA     BYTE      ADCIER
      000000A5H   SFRSYM    DATA     BYTE      OSEC
      000000D8H.6 SFRSYM    DATA     BIT       WDEN
      000000BAH   SFRSYM    DATA     BYTE      S0RELH
      00000080H.0 SFRSYM    DATA     BIT       P00
      000000D8H.7 SFRSYM    DATA     BIT       WDOF
      000000BBH   SFRSYM    DATA     BYTE      S1RELH
      00000090H.0 SFRSYM    DATA     BIT       P10
      00000080H.1 SFRSYM    DATA     BIT       P01
      00000087H   SFRSYM    DATA     BYTE      PCON
      000000C4H   SFRSYM    DATA     BYTE      PWM0DH
      000000A0H.0 SFRSYM    DATA     BIT       P20
      00000090H.1 SFRSYM    DATA     BIT       P11
      00000080H.2 SFRSYM    DATA     BIT       P02
      000000C6H   SFRSYM    DATA     BYTE      PWM1DH
      00000090H.2 SFRSYM    DATA     BIT       P12
      00000080H.3 SFRSYM    DATA     BIT       P03
      000000C7H   SFRSYM    DATA     BYTE      PWM2DH
      000000C8H.2 SFRSYM    DATA     BIT       PWM0IE
      000000AAH   SFRSYM    DATA     BYTE      S0RELL
      000000A0H.2 SFRSYM    DATA     BIT       P22
      00000090H.3 SFRSYM    DATA     BIT       P13
      00000080H.4 SFRSYM    DATA     BIT       P04
      000000C8H.1 SFRSYM    DATA     BIT       PWM0IF
      0000009DH   SFRSYM    DATA     BYTE      S1RELL
      000000A0H.3 SFRSYM    DATA     BIT       P23
      00000090H.4 SFRSYM    DATA     BIT       P14
      00000080H.5 SFRSYM    DATA     BIT       P05
      000000C3H   SFRSYM    DATA     BYTE      PWM0DL
      00000090H.5 SFRSYM    DATA     BIT       P15
      000000A6H   SFRSYM    DATA     BYTE      OSTATUS
      000000C5H   SFRSYM    DATA     BYTE      PWM1DL
      000000A0H.5 SFRSYM    DATA     BIT       P25
      000000D8H.4 SFRSYM    DATA     BIT       PORF
      000000D8H   SFRSYM    DATA     BYTE      RSTSTAT
      000000CFH   SFRSYM    DATA     BYTE      PWM2DL
      000000A0H.6 SFRSYM    DATA     BIT       P26
      000000C8H.7 SFRSYM    DATA     BIT       PWM0EN
      000000A0H.7 SFRSYM    DATA     BIT       P27
      000000A8H.5 SFRSYM    DATA     BIT       EPWM
      000000D8H.5 SFRSYM    DATA     BIT       LVRF
      000000F8H   SFRSYM    DATA     BYTE      CLKCON
      000000CCH   SFRSYM    DATA     BYTE      PWM0PH
      000000CEH   SFRSYM    DATA     BYTE      PWM1PH
      000000B8H.5 SFRSYM    DATA     BIT       I2CINTEN
      000000C2H   SFRSYM    DATA     BYTE      PWM2PH
      000000F0H   SFRSYM    DATA     BYTE      B
      000000EEH   SFRSYM    DATA     BYTE      RCHDIV
      000000CBH   SFRSYM    DATA     BYTE      PWM0PL
      000000CDH   SFRSYM    DATA     BYTE      PWM1PL
      000000C1H   SFRSYM    DATA     BYTE      PWM2PL
      000000F7H   SFRSYM    DATA     BYTE      ADCSPW
      000000F8H.1 SFRSYM    DATA     BIT       XCLKEN
      000000E0H   SFRSYM    DATA     BYTE      ACC
      000000DDH   SFRSYM    DATA     BYTE      LVDCON
      000000A8H.4 SFRSYM    DATA     BIT       ES0
LX51 LINKER/LOCATER V4.66.97.0                                                        06/12/2025  17:35:51  PAGE 60


      000000A9H   SFRSYM    DATA     BYTE      IP0
      000000A8H.1 SFRSYM    DATA     BIT       ET0
      000000A8H.2 SFRSYM    DATA     BIT       ES1
      000000F6H   SFRSYM    DATA     BYTE      ADCCSTAT
      000000B9H   SFRSYM    DATA     BYTE      IP1
      000000A8H.3 SFRSYM    DATA     BIT       ET1
      00000098H.0 SFRSYM    DATA     BIT       RI0
      000000C8H.0 SFRSYM    DATA     BIT       PWM0SS
      00000098H.1 SFRSYM    DATA     BIT       TI0
      000000A8H.0 SFRSYM    DATA     BIT       EX0
      000000D0H.0 SFRSYM    DATA     BIT       P
      000000B8H.3 SFRSYM    DATA     BIT       EFCINTEN
      000000A2H   SFRSYM    DATA     BYTE      OINTEN
      00000098H.7 SFRSYM    DATA     BIT       SM0
      00000098H.6 SFRSYM    DATA     BIT       SM1
      000000FEH   SFRSYM    DATA     BYTE      ADCCDR0
      000000FFH   SFRSYM    DATA     BYTE      ADCCDR1
      000000D0H.3 SFRSYM    DATA     BIT       RS0
      000000ACH   SFRSYM    DATA     BYTE      ADCGCR0
      000000D0H.4 SFRSYM    DATA     BIT       RS1
      000000ADH   SFRSYM    DATA     BYTE      ADCGCR1
      000000B4H   SFRSYM    DATA     BYTE      ADCGCR2
      000000B5H   SFRSYM    DATA     BYTE      ADCGCR3
      000000F8H.3 SFRSYM    DATA     BIT       RC32KEN
      000000DEH   SFRSYM    DATA     BYTE      PCLK0
      000000DFH   SFRSYM    DATA     BYTE      PCLK1
      00000083H   SFRSYM    DATA     BYTE      DPH
      000000E9H   SFRSYM    DATA     BYTE      P0IEN
      000000F5H   SFRSYM    DATA     BYTE      ADCHL
      000000F8H.2 SFRSYM    DATA     BIT       RC16MEN
      000000EAH   SFRSYM    DATA     BYTE      P1IEN
      000000EBH   SFRSYM    DATA     BYTE      P2IEN
      000000B6H   SFRSYM    DATA     WORD      ADCDR
      000000B3H   SFRSYM    DATA     BYTE      XTHCTR
      00000082H   SFRSYM    DATA     BYTE      DPL
      00000099H   SFRSYM    DATA     BYTE      S0BUF
      0000009CH   SFRSYM    DATA     BYTE      S1BUF
      000000F9H   SFRSYM    DATA     BYTE      P0OEN
      000000B8H.0 SFRSYM    DATA     BIT       GTIM0INTEN
      000000D9H   SFRSYM    DATA     BYTE      SYSDIV
      00000098H   SFRSYM    DATA     BYTE      S0CON
      000000FAH   SFRSYM    DATA     BYTE      P1OEN
      000000B8H.2 SFRSYM    DATA     BIT       GTIM1INTEN
      000000A3H   SFRSYM    DATA     BYTE      OINTUS
      000000BEH   SFRSYM    DATA     BYTE      RCHTRIMH
      000000F8H.0 SFRSYM    DATA     BIT       SYSSEL
      0000009BH   SFRSYM    DATA     BYTE      S1CON
      000000FBH   SFRSYM    DATA     BYTE      P2OEN
      000000B8H.6 SFRSYM    DATA     BIT       GTIM2INTEN
      000000BDH   SFRSYM    DATA     BYTE      LDOTRIMH
      00000092H   SFRSYM    DATA     BYTE      DPS
      0000009FH   SFRSYM    DATA     BYTE      RCLTRIMH
      000000BFH   SFRSYM    DATA     BYTE      RCHTRIML
      000000D3H   SFRSYM    DATA     BYTE      ODATA
      00000091H   SFRSYM    DATA     BYTE      LDOTRIML
      000000BCH   SFRSYM    DATA     BYTE      RCLTRIML
      000000E1H   SFRSYM    DATA     BYTE      P0IRQ
      000000B8H.1 SFRSYM    DATA     BIT       SPIINTEN
      000000E2H   SFRSYM    DATA     BYTE      P1IRQ
      000000E3H   SFRSYM    DATA     BYTE      P2IRQ
      000000D2H   SFRSYM    DATA     BYTE      OADRH
      000000B8H.7 SFRSYM    DATA     BIT       UART2INTEN
      000000F0H.0 SFRSYM    DATA     BIT       B0
      000000F0H.1 SFRSYM    DATA     BIT       B1
      000000F0H.2 SFRSYM    DATA     BIT       B2
LX51 LINKER/LOCATER V4.66.97.0                                                        06/12/2025  17:35:51  PAGE 61


      000000D1H   SFRSYM    DATA     BYTE      OADRL
      000000F0H.3 SFRSYM    DATA     BIT       B3
      000000F0H.4 SFRSYM    DATA     BIT       B4
      000000D0H.5 SFRSYM    DATA     BIT       F0
      000000F0H.5 SFRSYM    DATA     BIT       B5
      000000D0H.1 SFRSYM    DATA     BIT       F1
      000000AFH   SFRSYM    DATA     BYTE      REMAP
      000000F0H.6 SFRSYM    DATA     BIT       B6
      000000E0H.0 SFRSYM    DATA     BIT       ACC0
      000000A1H   SFRSYM    DATA     BYTE      OUS
      000000C8H.6 SFRSYM    DATA     BIT       PWM0S
      000000F0H.7 SFRSYM    DATA     BIT       B7
      000000E0H.1 SFRSYM    DATA     BIT       ACC1
      000000F8H.4 SFRSYM    DATA     BIT       XCLKF
      000000E0H.2 SFRSYM    DATA     BIT       ACC2
      0000008EH   SFRSYM    DATA     BYTE      PDSEL
      000000E0H.3 SFRSYM    DATA     BIT       ACC3
      000000D0H   SFRSYM    DATA     BYTE      PSW
      000000E0H.4 SFRSYM    DATA     BIT       ACC4
      00000098H.2 SFRSYM    DATA     BIT       RB80
      000000E0H.5 SFRSYM    DATA     BIT       ACC5
      000000FDH   SFRSYM    DATA     BYTE      ADCVREF
      000000E0H.6 SFRSYM    DATA     BIT       ACC6
      01002092H   SYMBOL    CONST    ---       _?ix1000

      0100005DH   BLOCK     CODE     ---       LVL=0
      0100005DH   LINE      CODE     ---       #23
      0100005DH   LINE      CODE     ---       #24
      0100005DH   LINE      CODE     ---       #25
      01000060H   LINE      CODE     ---       #27
      ---         BLOCKEND  ---      ---       LVL=0

      01001957H   BLOCK     CODE     ---       LVL=0
      01001957H   BLOCK     CODE     NEAR LAB  LVL=1
      0200025FH   SYMBOL    XDATA    BYTE      i
      02000260H   SYMBOL    XDATA    ---       recv_data
      020002A0H   SYMBOL    XDATA    BYTE      len
      ---         BLOCKEND  ---      ---       LVL=1
      01001957H   LINE      CODE     ---       #37
      01001957H   LINE      CODE     ---       #38
      01001957H   LINE      CODE     ---       #39
      0100195CH   LINE      CODE     ---       #40
      0100196EH   LINE      CODE     ---       #41
      01001973H   LINE      CODE     ---       #42
      01001989H   LINE      CODE     ---       #43
      01001989H   LINE      CODE     ---       #44
      0100199AH   LINE      CODE     ---       #45
      010019ADH   LINE      CODE     ---       #46
      010019ADH   LINE      CODE     ---       #47
      010019C5H   LINE      CODE     ---       #48
      010019CDH   LINE      CODE     ---       #49
      010019D6H   LINE      CODE     ---       #50
      010019D6H   LINE      CODE     ---       #51
      ---         BLOCKEND  ---      ---       LVL=0

      ---         MODULE    ---      ---       APP_EV1527
      0200015FH   PUBLIC    XDATA    ---       g_recv_data
      0200015EH   PUBLIC    XDATA    BYTE      g_recv_index
      0200015CH   PUBLIC    XDATA    WORD      high_time
      0200015AH   PUBLIC    XDATA    WORD      time
      02000158H   PUBLIC    XDATA    WORD      cycle
      020002A1H   PUBLIC    XDATA    BYTE      ?_app_ev1527_recv_data?BYTE
      010016C9H   PUBLIC    CODE     ---       _app_ev1527_recv_data
      01001D81H   PUBLIC    CODE     ---       app_ev1527_init
      0100125EH   PUBLIC    CODE     ---       GPIO_IRQHandler
LX51 LINKER/LOCATER V4.66.97.0                                                        06/12/2025  17:35:51  PAGE 62


      00000098H.3 SFRSYM    DATA     BIT       TB80
      000000E0H.7 SFRSYM    DATA     BIT       ACC7
      00000080H   SFRSYM    DATA     BYTE      P0
      00000090H   SFRSYM    DATA     BYTE      P1
      000000A0H   SFRSYM    DATA     BYTE      P2
      00000098H.5 SFRSYM    DATA     BIT       SM20
      000000B2H   SFRSYM    DATA     BYTE      ESTCR
      000000B1H   SFRSYM    DATA     BYTE      CLKST
      000000D0H.6 SFRSYM    DATA     BIT       AC
      000000D8H.3 SFRSYM    DATA     BIT       ERSTF
      000000E6H   SFRSYM    DATA     BYTE      PRESET0
      000000D4H   SFRSYM    DATA     BYTE      OCTRL
      000000A8H.7 SFRSYM    DATA     BIT       EA
      0000008FH   SFRSYM    DATA     BYTE      POREN
      000000C8H   SFRSYM    DATA     BYTE      PWM0CON
      000000E7H   SFRSYM    DATA     BYTE      PRESET1
      000000C9H   SFRSYM    DATA     BYTE      PWM1CON
      00000086H   SFRSYM    DATA     BYTE      BEEPCTR
      000000CAH   SFRSYM    DATA     BYTE      PWM2CON
      000000B8H.4 SFRSYM    DATA     BIT       LPTIMINTEN
      000000ABH   SFRSYM    DATA     BYTE      P0AH
      000000B0H   SFRSYM    DATA     BYTE      P1AH
      000000E8H   SFRSYM    DATA     BYTE      P2AH
      000000F8H.6 SFRSYM    DATA     BIT       RC32KF
      000000A8H   SFRSYM    DATA     BYTE      IEN0
      000000A7H   SFRSYM    DATA     BYTE      OPSET
      000000A4H   SFRSYM    DATA     BYTE      P0AL
      000000B8H   SFRSYM    DATA     BYTE      IEN1
      000000A8H.6 SFRSYM    DATA     BIT       EADC
      00000085H   SFRSYM    DATA     BYTE      DPH1
      000000AEH   SFRSYM    DATA     BYTE      P1AL
      0000009AH   SFRSYM    DATA     BYTE      IEN2
      000000C0H   SFRSYM    DATA     BYTE      P2AL
      000000B6H   SFRSYM    DATA     BYTE      ADCDR0
      000000F8H.5 SFRSYM    DATA     BIT       RC16MF
      000000B7H   SFRSYM    DATA     BYTE      ADCDR1
      00000084H   SFRSYM    DATA     BYTE      DPL1
      000000D6H   SFRSYM    DATA     BYTE      P0OD
      000000DBH   SFRSYM    DATA     BYTE      P1OD
      000000D5H   SFRSYM    DATA     BYTE      P0PD
      00000098H.4 SFRSYM    DATA     BIT       REN0
      000000ECH   SFRSYM    DATA     BYTE      P2OD
      000000DAH   SFRSYM    DATA     BYTE      P1PD
      000000E4H   SFRSYM    DATA     BYTE      P2PD
      000000D7H   SFRSYM    DATA     BYTE      P0CS
      00000097H   SFRSYM    DATA     BYTE      P0DR
      0000009EH   SFRSYM    DATA     BYTE      EUARTEN
      000000DCH   SFRSYM    DATA     BYTE      P1CS
      000000E5H   SFRSYM    DATA     BYTE      P1DR
      000000F4H   SFRSYM    DATA     BYTE      P2CS
      000000FCH   SFRSYM    DATA     BYTE      P2DR
      000000D0H.7 SFRSYM    DATA     BIT       CY
      000000D8H.0 SFRSYM    DATA     BIT       WDT0
      000000D8H.1 SFRSYM    DATA     BIT       WDT1
      000000D8H.2 SFRSYM    DATA     BIT       WDT2
      00000081H   SFRSYM    DATA     BYTE      SP
      000000F1H   SFRSYM    DATA     BYTE      P0PU
      000000F2H   SFRSYM    DATA     BYTE      P1PU
      000000D1H   SFRSYM    DATA     WORD      OADR
      000000F3H   SFRSYM    DATA     BYTE      P2PU
      00000093H   SFRSYM    DATA     BYTE      ADCIER
      000000A5H   SFRSYM    DATA     BYTE      OSEC
      000000D8H.6 SFRSYM    DATA     BIT       WDEN
      000000BAH   SFRSYM    DATA     BYTE      S0RELH
      00000080H.0 SFRSYM    DATA     BIT       P00
LX51 LINKER/LOCATER V4.66.97.0                                                        06/12/2025  17:35:51  PAGE 63


      000000D8H.7 SFRSYM    DATA     BIT       WDOF
      000000BBH   SFRSYM    DATA     BYTE      S1RELH
      00000090H.0 SFRSYM    DATA     BIT       P10
      00000080H.1 SFRSYM    DATA     BIT       P01
      00000087H   SFRSYM    DATA     BYTE      PCON
      000000C4H   SFRSYM    DATA     BYTE      PWM0DH
      000000A0H.0 SFRSYM    DATA     BIT       P20
      00000090H.1 SFRSYM    DATA     BIT       P11
      00000080H.2 SFRSYM    DATA     BIT       P02
      000000C6H   SFRSYM    DATA     BYTE      PWM1DH
      00000090H.2 SFRSYM    DATA     BIT       P12
      00000080H.3 SFRSYM    DATA     BIT       P03
      000000C7H   SFRSYM    DATA     BYTE      PWM2DH
      000000C8H.2 SFRSYM    DATA     BIT       PWM0IE
      000000AAH   SFRSYM    DATA     BYTE      S0RELL
      000000A0H.2 SFRSYM    DATA     BIT       P22
      00000090H.3 SFRSYM    DATA     BIT       P13
      00000080H.4 SFRSYM    DATA     BIT       P04
      000000C8H.1 SFRSYM    DATA     BIT       PWM0IF
      0000009DH   SFRSYM    DATA     BYTE      S1RELL
      000000A0H.3 SFRSYM    DATA     BIT       P23
      00000090H.4 SFRSYM    DATA     BIT       P14
      00000080H.5 SFRSYM    DATA     BIT       P05
      000000C3H   SFRSYM    DATA     BYTE      PWM0DL
      00000090H.5 SFRSYM    DATA     BIT       P15
      000000A6H   SFRSYM    DATA     BYTE      OSTATUS
      000000C5H   SFRSYM    DATA     BYTE      PWM1DL
      000000A0H.5 SFRSYM    DATA     BIT       P25
      000000D8H.4 SFRSYM    DATA     BIT       PORF
      000000D8H   SFRSYM    DATA     BYTE      RSTSTAT
      000000CFH   SFRSYM    DATA     BYTE      PWM2DL
      000000A0H.6 SFRSYM    DATA     BIT       P26
      000000C8H.7 SFRSYM    DATA     BIT       PWM0EN
      000000A0H.7 SFRSYM    DATA     BIT       P27
      000000A8H.5 SFRSYM    DATA     BIT       EPWM
      000000D8H.5 SFRSYM    DATA     BIT       LVRF
      000000F8H   SFRSYM    DATA     BYTE      CLKCON
      000000CCH   SFRSYM    DATA     BYTE      PWM0PH
      000000CEH   SFRSYM    DATA     BYTE      PWM1PH
      000000B8H.5 SFRSYM    DATA     BIT       I2CINTEN
      000000C2H   SFRSYM    DATA     BYTE      PWM2PH
      000000F0H   SFRSYM    DATA     BYTE      B
      000000EEH   SFRSYM    DATA     BYTE      RCHDIV
      000000CBH   SFRSYM    DATA     BYTE      PWM0PL
      000000CDH   SFRSYM    DATA     BYTE      PWM1PL
      000000C1H   SFRSYM    DATA     BYTE      PWM2PL
      000000F7H   SFRSYM    DATA     BYTE      ADCSPW
      000000F8H.1 SFRSYM    DATA     BIT       XCLKEN
      000000E0H   SFRSYM    DATA     BYTE      ACC
      000000DDH   SFRSYM    DATA     BYTE      LVDCON
      000000A8H.4 SFRSYM    DATA     BIT       ES0
      000000A9H   SFRSYM    DATA     BYTE      IP0
      000000A8H.1 SFRSYM    DATA     BIT       ET0
      000000A8H.2 SFRSYM    DATA     BIT       ES1
      000000F6H   SFRSYM    DATA     BYTE      ADCCSTAT
      000000B9H   SFRSYM    DATA     BYTE      IP1
      000000A8H.3 SFRSYM    DATA     BIT       ET1
      00000098H.0 SFRSYM    DATA     BIT       RI0
      000000C8H.0 SFRSYM    DATA     BIT       PWM0SS
      00000098H.1 SFRSYM    DATA     BIT       TI0
      000000A8H.0 SFRSYM    DATA     BIT       EX0
      000000D0H.0 SFRSYM    DATA     BIT       P
      000000B8H.3 SFRSYM    DATA     BIT       EFCINTEN
      000000A2H   SFRSYM    DATA     BYTE      OINTEN
      00000098H.7 SFRSYM    DATA     BIT       SM0
LX51 LINKER/LOCATER V4.66.97.0                                                        06/12/2025  17:35:51  PAGE 64


      00000098H.6 SFRSYM    DATA     BIT       SM1
      000000FEH   SFRSYM    DATA     BYTE      ADCCDR0
      000000FFH   SFRSYM    DATA     BYTE      ADCCDR1
      000000D0H.3 SFRSYM    DATA     BIT       RS0
      000000ACH   SFRSYM    DATA     BYTE      ADCGCR0
      000000D0H.4 SFRSYM    DATA     BIT       RS1
      000000ADH   SFRSYM    DATA     BYTE      ADCGCR1
      000000B4H   SFRSYM    DATA     BYTE      ADCGCR2
      000000B5H   SFRSYM    DATA     BYTE      ADCGCR3
      000000F8H.3 SFRSYM    DATA     BIT       RC32KEN
      000000DEH   SFRSYM    DATA     BYTE      PCLK0
      000000DFH   SFRSYM    DATA     BYTE      PCLK1
      00000083H   SFRSYM    DATA     BYTE      DPH
      000000E9H   SFRSYM    DATA     BYTE      P0IEN
      000000F5H   SFRSYM    DATA     BYTE      ADCHL
      000000F8H.2 SFRSYM    DATA     BIT       RC16MEN
      000000EAH   SFRSYM    DATA     BYTE      P1IEN
      000000EBH   SFRSYM    DATA     BYTE      P2IEN
      000000B6H   SFRSYM    DATA     WORD      ADCDR
      000000B3H   SFRSYM    DATA     BYTE      XTHCTR
      00000082H   SFRSYM    DATA     BYTE      DPL
      00000099H   SFRSYM    DATA     BYTE      S0BUF
      0000009CH   SFRSYM    DATA     BYTE      S1BUF
      000000F9H   SFRSYM    DATA     BYTE      P0OEN
      000000B8H.0 SFRSYM    DATA     BIT       GTIM0INTEN
      000000D9H   SFRSYM    DATA     BYTE      SYSDIV
      00000098H   SFRSYM    DATA     BYTE      S0CON
      000000FAH   SFRSYM    DATA     BYTE      P1OEN
      000000B8H.2 SFRSYM    DATA     BIT       GTIM1INTEN
      000000A3H   SFRSYM    DATA     BYTE      OINTUS
      000000BEH   SFRSYM    DATA     BYTE      RCHTRIMH
      000000F8H.0 SFRSYM    DATA     BIT       SYSSEL
      0000009BH   SFRSYM    DATA     BYTE      S1CON
      000000FBH   SFRSYM    DATA     BYTE      P2OEN
      000000B8H.6 SFRSYM    DATA     BIT       GTIM2INTEN
      000000BDH   SFRSYM    DATA     BYTE      LDOTRIMH
      00000092H   SFRSYM    DATA     BYTE      DPS
      0000009FH   SFRSYM    DATA     BYTE      RCLTRIMH
      000000BFH   SFRSYM    DATA     BYTE      RCHTRIML
      000000D3H   SFRSYM    DATA     BYTE      ODATA
      00000091H   SFRSYM    DATA     BYTE      LDOTRIML
      000000BCH   SFRSYM    DATA     BYTE      RCLTRIML
      000000E1H   SFRSYM    DATA     BYTE      P0IRQ
      000000B8H.1 SFRSYM    DATA     BIT       SPIINTEN
      000000E2H   SFRSYM    DATA     BYTE      P1IRQ
      000000E3H   SFRSYM    DATA     BYTE      P2IRQ
      000000D2H   SFRSYM    DATA     BYTE      OADRH
      000000B8H.7 SFRSYM    DATA     BIT       UART2INTEN
      000000F0H.0 SFRSYM    DATA     BIT       B0
      000000F0H.1 SFRSYM    DATA     BIT       B1
      000000F0H.2 SFRSYM    DATA     BIT       B2
      000000D1H   SFRSYM    DATA     BYTE      OADRL
      000000F0H.3 SFRSYM    DATA     BIT       B3
      000000F0H.4 SFRSYM    DATA     BIT       B4
      000000D0H.5 SFRSYM    DATA     BIT       F0
      000000F0H.5 SFRSYM    DATA     BIT       B5
      000000D0H.1 SFRSYM    DATA     BIT       F1
      000000AFH   SFRSYM    DATA     BYTE      REMAP
      000000F0H.6 SFRSYM    DATA     BIT       B6
      000000E0H.0 SFRSYM    DATA     BIT       ACC0
      000000A1H   SFRSYM    DATA     BYTE      OUS
      000000C8H.6 SFRSYM    DATA     BIT       PWM0S
      000000F0H.7 SFRSYM    DATA     BIT       B7
      000000E0H.1 SFRSYM    DATA     BIT       ACC1
      000000F8H.4 SFRSYM    DATA     BIT       XCLKF
LX51 LINKER/LOCATER V4.66.97.0                                                        06/12/2025  17:35:51  PAGE 65


      000000E0H.2 SFRSYM    DATA     BIT       ACC2
      0000008EH   SFRSYM    DATA     BYTE      PDSEL
      000000E0H.3 SFRSYM    DATA     BIT       ACC3
      000000D0H   SFRSYM    DATA     BYTE      PSW
      000000E0H.4 SFRSYM    DATA     BIT       ACC4
      00000098H.2 SFRSYM    DATA     BIT       RB80
      000000E0H.5 SFRSYM    DATA     BIT       ACC5
      000000FDH   SFRSYM    DATA     BYTE      ADCVREF
      000000E0H.6 SFRSYM    DATA     BIT       ACC6

      0100125EH   BLOCK     CODE     ---       LVL=0
      0100125EH   LINE      CODE     ---       #39
      01001269H   LINE      CODE     ---       #41
      01001274H   LINE      CODE     ---       #42
      01001274H   LINE      CODE     ---       #44
      01001288H   LINE      CODE     ---       #45
      0100128FH   LINE      CODE     ---       #46
      01001293H   LINE      CODE     ---       #48
      0100129EH   LINE      CODE     ---       #49
      0100129EH   LINE      CODE     ---       #51
      010012B8H   LINE      CODE     ---       #52
      010012C0H   LINE      CODE     ---       #53
      010012C0H   LINE      CODE     ---       #54
      010012C2H   LINE      CODE     ---       #56
      010012C2H   LINE      CODE     ---       #58
      010012D1H   LINE      CODE     ---       #59
      010012D1H   LINE      CODE     ---       #60
      010012D8H   LINE      CODE     ---       #62
      010012D8H   LINE      CODE     ---       #64
      010012DFH   LINE      CODE     ---       #65
      010012DFH   LINE      CODE     ---       #66
      01001307H   LINE      CODE     ---       #67
      01001307H   LINE      CODE     ---       #68
      01001309H   LINE      CODE     ---       #70
      01001309H   LINE      CODE     ---       #71
      01001337H   LINE      CODE     ---       #72
      0100133DH   LINE      CODE     ---       #73
      0100133DH   LINE      CODE     ---       #74
      0100133FH   LINE      CODE     ---       #76
      0100133FH   LINE      CODE     ---       #78
      0100134CH   LINE      CODE     ---       #79
      0100134CH   LINE      CODE     ---       #80
      0100134FH   LINE      CODE     ---       #81
      0100134FH   LINE      CODE     ---       #82
      ---         BLOCKEND  ---      ---       LVL=0

      01001D81H   BLOCK     CODE     ---       LVL=0
      01001D81H   LINE      CODE     ---       #91
      01001D81H   LINE      CODE     ---       #92
      01001D81H   LINE      CODE     ---       #93
      01001D86H   LINE      CODE     ---       #94
      01001D8DH   LINE      CODE     ---       #95
      01001D94H   LINE      CODE     ---       #96
      01001D9BH   LINE      CODE     ---       #97
      01001DA8H   LINE      CODE     ---       #98
      01001DABH   LINE      CODE     ---       #99
      01001DAEH   LINE      CODE     ---       #101
      01001DB7H   LINE      CODE     ---       #102
      01001DBEH   LINE      CODE     ---       #103
      ---         BLOCKEND  ---      ---       LVL=0

      010016C9H   BLOCK     CODE     ---       LVL=0
      020002A1H   SYMBOL    XDATA    ---       dat
      020002A4H   SYMBOL    XDATA    ---       len
      010016CFH   BLOCK     CODE     NEAR LAB  LVL=1
LX51 LINKER/LOCATER V4.66.97.0                                                        06/12/2025  17:35:51  PAGE 66


      020002A7H   SYMBOL    XDATA    BYTE      i
      ---         BLOCKEND  ---      ---       LVL=1
      010016C9H   LINE      CODE     ---       #113
      010016CFH   LINE      CODE     ---       #114
      010016CFH   LINE      CODE     ---       #115
      010016D4H   LINE      CODE     ---       #116
      010016E1H   LINE      CODE     ---       #117
      010016E1H   LINE      CODE     ---       #118
      010016EEH   LINE      CODE     ---       #119
      0100170EH   LINE      CODE     ---       #120
      0100170EH   LINE      CODE     ---       #121
      01001726H   LINE      CODE     ---       #122
      01001726H   LINE      CODE     ---       #123
      01001741H   LINE      CODE     ---       #124
      01001749H   LINE      CODE     ---       #125
      0100174EH   LINE      CODE     ---       #126
      01001750H   LINE      CODE     ---       #127
      01001750H   LINE      CODE     ---       #128
      01001750H   LINE      CODE     ---       #129
      01001752H   LINE      CODE     ---       #130
      ---         BLOCKEND  ---      ---       LVL=0

      ---         MODULE    ---      ---       ?C?FPADD
      0100006DH   PUBLIC    CODE     ---       ?C?FPADD
      01000069H   PUBLIC    CODE     ---       ?C?FPSUB

      ---         MODULE    ---      ---       ?C?FPMUL
      0100015EH   PUBLIC    CODE     ---       ?C?FPMUL

      ---         MODULE    ---      ---       ?C?FPDIV
      01000267H   PUBLIC    CODE     ---       ?C?FPDIV

      ---         MODULE    ---      ---       ?C?FPCMP
      01000306H   PUBLIC    CODE     ---       ?C?FPCMP
      01000304H   PUBLIC    CODE     ---       ?C?FPCMP3

      ---         MODULE    ---      ---       ?C?FPNEG
      0100037DH   PUBLIC    CODE     ---       ?C?FPNEG

      ---         MODULE    ---      ---       ?C?FCAST
      01000398H   PUBLIC    CODE     ---       ?C?FCASTC
      01000393H   PUBLIC    CODE     ---       ?C?FCASTI
      0100038EH   PUBLIC    CODE     ---       ?C?FCASTL

      ---         MODULE    ---      ---       ?C?CASTF
      010003CCH   PUBLIC    CODE     ---       ?C?CASTF

      ---         MODULE    ---      ---       PRINTF
      020002A1H   PUBLIC    XDATA    ---       ?_PRINTF?BYTE
      020002A1H   PUBLIC    XDATA    ---       ?_SPRINTF?BYTE
      01000B1BH   PUBLIC    CODE     ---       _PRINTF
      01000B15H   PUBLIC    CODE     ---       _SPRINTF

      ---         MODULE    ---      ---       FABS

      ---         MODULE    ---      ---       ?C?FPGETOPN
      01000403H   PUBLIC    CODE     ---       ?C?FPGETOPN2
      01000438H   PUBLIC    CODE     ---       ?C?FPNANRESULT
      01000442H   PUBLIC    CODE     ---       ?C?FPOVERFLOW
      0100041AH   PUBLIC    CODE     ---       ?C?FPRESULT
      0100042EH   PUBLIC    CODE     ---       ?C?FPRESULT2
      0100043FH   PUBLIC    CODE     ---       ?C?FPUNDERFLOW

      ---         MODULE    ---      ---       ?C?FPROUND
      0100044DH   PUBLIC    CODE     ---       ?C?FPROUND
LX51 LINKER/LOCATER V4.66.97.0                                                        06/12/2025  17:35:51  PAGE 67



      ---         MODULE    ---      ---       ?C?FPCONVERT
      0100048AH   PUBLIC    CODE     ---       ?C?FPCONVERT

      ---         MODULE    ---      ---       ?C?FTNPWR
      010005BFH   PUBLIC    CODE     ---       ?C?FTNPWR

      ---         MODULE    ---      ---       ?C_INIT
      01001684H   PUBLIC    CODE     ---       ?C_START

      ---         MODULE    ---      ---       ?C?COPY
      010006CFH   PUBLIC    CODE     ---       ?C?COPY

      ---         MODULE    ---      ---       ?C?CLDPTR
      010006F5H   PUBLIC    CODE     ---       ?C?CLDPTR

      ---         MODULE    ---      ---       ?C?CLDOPTR
      0100070EH   PUBLIC    CODE     ---       ?C?CLDOPTR

      ---         MODULE    ---      ---       ?C?CSTPTR
      0100073BH   PUBLIC    CODE     ---       ?C?CSTPTR

      ---         MODULE    ---      ---       ?C?CSTOPTR
      0100074DH   PUBLIC    CODE     ---       ?C?CSTOPTR

      ---         MODULE    ---      ---       ?C?IMUL
      0100076FH   PUBLIC    CODE     ---       ?C?IMUL

      ---         MODULE    ---      ---       ?C?LADD
      01000781H   PUBLIC    CODE     ---       ?C?LADD

      ---         MODULE    ---      ---       ?C?LMUL
      0100078EH   PUBLIC    CODE     ---       ?C?LMUL

      ---         MODULE    ---      ---       ?C?ULDIV
      01000819H   PUBLIC    CODE     ---       ?C?ULDIV

      ---         MODULE    ---      ---       ?C?SLDIV
      01001CFDH   PUBLIC    CODE     ---       ?C?SLDIV

      ---         MODULE    ---      ---       ?C?LOR
      010008ABH   PUBLIC    CODE     ---       ?C?LOR

      ---         MODULE    ---      ---       ?C?LNEG
      010008B8H   PUBLIC    CODE     ---       ?C?LNEG

      ---         MODULE    ---      ---       ?C?SLCMP
      010008C6H   PUBLIC    CODE     ---       ?C?SLCMP

      ---         MODULE    ---      ---       ?C?ULCMP
      010008DCH   PUBLIC    CODE     ---       ?C?ULCMP

      ---         MODULE    ---      ---       ?C?ULSHR
      010008EDH   PUBLIC    CODE     ---       ?C?ULSHR

      ---         MODULE    ---      ---       ?C?LSHL
      01000900H   PUBLIC    CODE     ---       ?C?LSHL

      ---         MODULE    ---      ---       ?C?LLDOPTR
      01000913H   PUBLIC    CODE     ---       ?C?LLDOPTR

      ---         MODULE    ---      ---       ?C?LLDXDATA
      01000943H   PUBLIC    CODE     ---       ?C?LLDXDATA

      ---         MODULE    ---      ---       ?C?LLDXDATA0
LX51 LINKER/LOCATER V4.66.97.0                                                        06/12/2025  17:35:51  PAGE 68


      0100094FH   PUBLIC    CODE     ---       ?C?LLDXDATA0

      ---         MODULE    ---      ---       ?C?LLDIXDATA
      01000964H   PUBLIC    CODE     ---       ?C?LLDIXDATA
      0100095BH   PUBLIC    CODE     ---       ?C?LLDIXDATA1
      0100095DH   PUBLIC    CODE     ---       ?C?LLDIXDATA8

      ---         MODULE    ---      ---       ?C?LSTXDATA
      01000990H   PUBLIC    CODE     ---       ?C?LSTXDATA

      ---         MODULE    ---      ---       ?C?LSTKXDATA
      0100099CH   PUBLIC    CODE     ---       ?C?LSTKXDATA

      ---         MODULE    ---      ---       ?C?PLDXDATA
      010009CDH   PUBLIC    CODE     ---       ?C?PLDXDATA

      ---         MODULE    ---      ---       ?C?PLDIXDATA
      010009D6H   PUBLIC    CODE     ---       ?C?PLDIXDATA

      ---         MODULE    ---      ---       ?C?PSTXDATA
      010009EDH   PUBLIC    CODE     ---       ?C?PSTXDATA

      ---         MODULE    ---      ---       ?C?CCASE
      010009F6H   PUBLIC    CODE     ---       ?C?CCASE

      ---         MODULE    ---      ---       ?C?LCASE
      01000A1CH   PUBLIC    CODE     ---       ?C?LCASE

      ---         MODULE    ---      ---       ?C?ICALL
      01000A56H   PUBLIC    CODE     ---       ?C?ICALL
      01000A5AH   PUBLIC    CODE     ---       ?C?ICALL2

      ---         MODULE    ---      ---       ?C?MEMSET
      01000A5CH   PUBLIC    CODE     ---       ?C?MEMSET

      ---         MODULE    ---      ---       ?C?LLDIDATA
      01000A88H   PUBLIC    CODE     ---       ?C?LLDIDATA

      ---         MODULE    ---      ---       ?C?LLDPDATA
      01000A94H   PUBLIC    CODE     ---       ?C?LLDPDATA

      ---         MODULE    ---      ---       ?C?LLDCODE
      01000AA0H   PUBLIC    CODE     ---       ?C?LLDCODE

Program Size: data=23.1 xdata=818 const=429 code=7973
LX51 RUN COMPLETE.  0 WARNING(S),  0 ERROR(S)
